:100000000C94B0040C94F6040C94F6040C94F604CE
:100010000C94F6040C94F6040C94F6040C94F60478
:100020000C94F6040C9456180C94F6040C94F604F4
:100030000C94782E0C94F6040C94F6040C94F604AC
:100040000C94F6040C94F6040C9479140C94F604B5
:100050000C94100B0C94F6040C94DA0A0C94F6042D
:100060000C94261A0C94F6040C946D290C94F60446
:100070000C94F0720C94F6040C944F6D4B1A501AB9
:10008000551A5E1A751A8C1A9C1AAC1AF01ADB1CD7
:100090008C1AC61BD71BEB1B091C261C711CBD1C14
:1000A000CE1E9B1F0E208720BF20622121227E2290
:1000B000F9222A23A023CE23FB236F627563FA6300
:1000C00013634E648064AE6242630A0D3D3D3D3D64
:1000D0003D3D3D3D3D3D3D3D3D3D3D3D3D3D3D3D50
:1000E0003D3D3D3D3D3D3D3D3D3D3D3D3D3D3D007D
:1000F0000A0D426174743A002025642043656C6CDB
:10010000732000204C6F77207761726E696E673ABA
:100110002025642E2564560020204175746F2D43E0
:10012000483A2025642E2564560020204175746FBE
:100130006C616E64696E673A2025642E25645600F2
:100140000A0D4F6C642046432048617264776172E7
:1001500065206E6F7420737570706F7274656420A3
:1001600062792074686973204672696D776172657F
:1001700021000A0D466F756E6420424C2D43747247
:100180006C3A20002564000A0D0A0D2121204D49FA
:100190005353494E4720424C2D4354524C3A20254C
:1001A00064202121000A0D43616C696272617469E7
:1001B0006E672070726573737572652073656E73F8
:1001C0006F722E2E004F4B0A0D000A0D466C6967A8
:1001D00068742D74696D65202575206D696E2054D5
:1001E0006F74616C3A2575206D696E00416E676CA5
:1001F000654E69636B20202020202020416E676CB3
:1002000065526F6C6C202020202020204163634EBB
:1002100069636B202020202020202020416363522E
:100220006F6C6C20202020202020202059617747EF
:1002300079726F202020202020202020416C7469BA
:1002400074756465205B302E316D5D204163635AA7
:1002500020202020202020202020202047617320E3
:10026000202020202020202020202020436F6D707F
:100270006173732056616C7565202020566F6C7415
:10028000616765205B302E31565D202052656365C5
:1002900069766572204C6576656C20204779726FAF
:1002A00020436F6D70617373202020204D6F746F39
:1002B0007220312020202020202020204D6F746FBC
:1002C0007220322020202020202020204D6F746FAB
:1002D0007220332020202020202020204D6F746F9A
:1002E0007220342020202020202020203136202081
:1002F00020202020202020202020202031372020D6
:1003000020202020202020202020202031382020C4
:1003100020202020202020202020202031392020B3
:1003200020202020202020202020202053657276AD
:100330006F2020202020202020202020486F76655C
:100340007267617320202020202020204375727264
:10035000656E74205B302E31415D202043617061F9
:1003600063697479205B6D41685D20204865696729
:10037000687420536574706F696E74203235202064
:100380002020202020202020202020203236202045
:100390002020202020202020202020203237202034
:1003A0002020202020202020202020204932432DE2
:1003B0004572726F7220202020202020424C204C59
:1003C000696D697420202020202020204750535F31
:1003D0004E69636B20202020202020204750535F4F
:1003E000526F6C6C202020202020202021212120F1
:1003F000494E434F4D50415449424C452021212103
:10040000002E005B25695D005B25695D002B204D9A
:10041000696B726F4B6F70746572202B0048573A8E
:100420005625642E25642053573A25642E253032F4
:10043000642563200053657474696E673A256420EF
:100440002573004D69786572204572726F722100C4
:100450004861726477617265204572726F722031F3
:100460003A2564202121004D697373696E6720422B
:100470004C2D4374726C3A25642021210021204EBA
:10048000432D4552523A2025326420212000493222
:1004900043204552524F5221212100424C2D536599
:1004A0006C6674657374204572723A253264004834
:1004B00065696768743A2020253569005365747052
:1004C0006F696E743A253569005072657373757281
:1004D000653A253569004F66667365743A202025B4
:1004E0003569006163742E2062656172696E670010
:1004F0004E69636B3A202020202020253569005268
:100500006F6C6C3A20202020202025356900436F35
:100510006D706173733A202020253569004B256981
:100520003A25346920204B25693A25346920004E4C
:10053000693A2534692020526F3A253469200047F2
:10054000733A253469202047693A253469200050E0
:10055000313A253469202050323A25346920005040
:10056000333A253469202050343A25346920004735
:1005700079726F202D2053656E736F72004E696320
:100580006B2025346920282533692E2578290052CF
:100590006F6C6C2025346920282533692E25782935
:1005A00000596177202025346920282533692900E6
:1005B000414343202D2053656E736F72004E696373
:1005C0006B2025346920282533692900526F6C6C13
:1005D00020253469202825336929005A202020202D
:1005E00025346920282533692900566F6C746167AA
:1005F000653A2020202533692E2531695600437540
:100600007272656E743A2020202533692E25316977
:100610004100506F7765723A2020202020253469F0
:1006200057004469736368617267653A20253569CC
:100630006D41680052656365697665720052432DAD
:100640005175616C6974793A202534690052432DE3
:100650004368616E6E656C733A25346900556E644B
:100660006572766F6C7461676573202000576172E4
:100670006E3A202532642E25645600486F6D653A27
:10068000202532642E256456004C616E643A202584
:1006900032642E25645600506F746925693A202013
:1006A00025336900506F746925693A202025336924
:1006B00000466C696768742D54696D65202000548C
:1006C0006F74616C3A2535756D696E004163743ADB
:1006D00020202535756D696E002872657365742953
:1006E000000A0D47656E65726174696E6720646506
:1006F0006661756C7420506172616D6574657220FD
:10070000536574202564000A0D5573696E67205087
:100710006172616D65746572205365742025640093
:100720000A0D47656E65726174696E67206465665F
:1007300061756C74204D69786572205461626C65D6
:10074000000A0D4D697865722D436F6E6669673AD0
:10075000202725732720282575204D6F746F72730D
:1007600029000A0D414343206E6F742063616C6958
:10077000627261746564210D0A0000008F001E0121
:10078000AD013B02CA025803E603740402058F055B
:100790001B06A7063307BE074808D2085B09E30912
:1007A0006B0AF20A780BFD0B810C040D860D070E07
:1007B000870E060F840F00107B10F5106E11E511E7
:1007C0005B12CF124213B31323149214FE146A1552
:1007D000D3153B16A11605176717C81727188318D6
:1007E000DE1837198E19E319361A871AD61A231B01
:1007F0006E1BB61BFD1B411C831CC31C001D3C1D36
:10080000751DAB1DE01D121E421E6F1E9A1EC31EDB
:10081000E91E0D1F2E1F4D1F691F841F9B1FB01F38
:10082000C31FD31FE11FEC1FF51FFB1FFF1F00207D
:100830000A0D7777772E4D696B726F4B6F70746509
:10084000722E646520286329204869537973746582
:100850006D7320476D6248000A0D746865207573DA
:1008600065206F66207468697320736F66747761A2
:100870007265206973206F6E6C79207065726D6986
:1008800074746564200A0D6F6E206F726967696EFB
:10089000616C204D696B726F4B6F707465722D487F
:1008A00061726477617265005573657200486F54B8
:1008B00054205634004143542044534C004A65743C
:1008C00069005370656B7472756D0050504D000A6D
:1008D0000D52656365697665723A2000756E6B6EC0
:1008E0006F776E2E205573696E672050504D2E2EF7
:1008F0002E006E6F7420737570706F727465642053
:10090000627920686172647761726521000A0D2046
:100910002D204C4942204E4F5420434F4D504154BE
:1009200049424C452021212121000A0D466C69676E
:100930006874436F6E74726F6C0A0D4861726477ED
:100940006172653A25642E25640A0D536F667477CB
:100950006172653A5625642E253032642563200085
:1009600011241FBECFEFD0E1DEBFCDBF11E0A0E06C
:10097000B1E0EAE7FBEE02C005900D92AE3AB10796
:10098000D9F719E0AEEAB1E001C01D92AE38B10767
:10099000E1F74AEAE2E0F0E081E280935700549107
:1009A00020EF37EFACE9B3E09FE0F9012F5F3F4F55
:1009B00084918D93915097FFF8CF573911F400002F
:1009C000FECFECE9F3E09EE08191482740959150FD
:1009D00097FFFACF8091AB03481721F0573911F4F4
:1009E0000000FECF0E942B060C94BC750C940000F6
:1009F0008AEC90E09F938F938CE891E19F938F9383
:100A0000E091AF03F091B00309950F900F900F9014
:100A10000F90089580915406E82FFF27EE0FFF1FD7
:100A2000E552F84F808191818D5E9F4F14F01092B6
:100A30000401808191818A5B9F4FCCF480910401F5
:100A40008823A9F481E0809304018091E3038F5F00
:100A50008093E303853038F088EE93E09093E701CC
:100A60008093E601089566E970E00E945030089591
:100A7000CF93DF93C82F882311F180EF90E09F93ED
:100A80008F938CE891E19F938F93E091AF03F09166
:100A9000B003099580912301909124016BE270E0ED
:100AA0000E942F75CB018F5F809300010F900F90F4
:100AB0000F900F90873018F086E0809300018091AE
:100AC0007706823328F590910001989F802D11249C
:100AD00080930201CC23F1F068EC70E0892F0E9432
:100AE00050308091000199279F938F9388EF90E079
:100AF0009F938F938CE891E19F938F93E091AF0345
:100B0000F091B00309958DB79EB706968DBF02C0D0
:100B1000809302019091C706923340F480910001C6
:100B2000899F802D11248093B80102C09093B80151
:100B30003091C806323340F480910001839F802DAC
:100B400011248093B70102C03093B7018091B8019E
:100B500090910201981720F491509093B8019F5FF3
:100B60008091B701891720F091509093B7019F5F52
:100B70008091B8012091B701821728F0332319F032
:100B800021502093B801CC2309F462C0892F6AE078
:100B90000E940F75892F99279F938F93809102014F
:100BA0000E940F7599279F938F9383E091E09F9305
:100BB0008F93CCE8D1E1DF93CF93E091AF03F09135
:100BC000B00309958DB79EB708968DBF8091B70188
:100BD0008823E9F06AE00E940F75892F99279F9377
:100BE0008F938091B7010E940F7599279F938F93E0
:100BF00088E191E09F938F93DF93CF93E091AF03D0
:100C0000F091B00309958DB79EB708968DBF80917E
:100C1000B8018823E9F06AE00E940F75892F9927AF
:100C20009F938F938091B8010E940F7599279F938E
:100C30008F938AE291E09F938F93DF93CF93E0911C
:100C4000AF03F091B00309958DB79EB708968DBF9D
:100C5000DF91CF910895CFEFD0E1DEBFCDBF8824E3
:100C60009924C1E07C2E14B815B88AE08AB98FE5C2
:100C70008BB9B7EEEB2EB3E0FB2E2EEC3FEFE20E7E
:100C8000F31EF7FEFACF189B06C0199B02C08DE039
:100C900005C08BE003C0199B04C084E1809303016D
:100CA00007C08AE0809303018EE38AB987E48BB999
:100CB00081E887B93E9A8FEF88B98BE184B981E0EA
:100CC00085B9469A84B7877F84BF80916000886128
:100CD000809360001092600084EC99E09093E701AB
:100CE0008093E60110929702109296021092E0070C
:100CF0001092DF07109299021092980210929B02B4
:100D000010929A0220910301243128F084EC94E09F
:100D1000A0E0B0E004C08BE095E0A0E0B0E08093FC
:100D2000400190934101A0934201B0934301289860
:100D3000293111F4299A01C029980E94CA150E94EC
:100D40009B150E9494110E943F2E0E94861981E0FB
:100D50000E9420290E9415610E94D66A86E00E94A6
:100D6000997180910301893111F4299A01C0299860
:100D700078940E944128809103018431E8F488E14D
:100D800090E02CE00FB6F894A895809360000FBE19
:100D90002093600080E491E09F938F938CE891E131
:100DA0009F938F93E091AF03F091B00309950F905B
:100DB0000F900F900F90EECF80913502826080935C
:100DC0003502109238020E948D3B84EF91E00E9420
:100DD00061157C018091350280FD05C0C7010E942C
:100DE0006A158823B9F382E791E09F938F93ACE86B
:100DF000AA2EA1E1BA2EBF92AF92E091AF03F0917B
:100E0000B003099580EA9FE00E9461157C01C0E073
:100E1000D0E00F900F900F900F9001E717E0F9EEE0
:100E2000CF2EF6E0DF2E0E948D3B8091350280FDB3
:100E300005C0C7010E946A158823B9F3F6018081B5
:100E40001816ACF40BC00E948D3B8091350280FDDA
:100E500005C0C7010E946A158823B9F3C7010E9423
:100E60006A15882321F4F8018081882364F7F8014A
:100E7000808187FF19C02196DF93CF93219784E863
:100E800091E09F938F93BF92AF92E091AF03F09167
:100E9000B00309958091B0018F5F8093B0012DB7A9
:100EA0003EB72A5F3F4F2DBF219684E090E0C80EE9
:100EB000D91E075F1F4FCC30D10508F4B4CFC0E076
:100EC000D0E00EE617E0E9EEEE2EE6E0FE2EF801A9
:100ED000838187FD1DC0F70180811816CCF421960F
:100EE000DF93CF93219787E891E09F938F938CE8CE
:100EF00091E19F938F93E091AF03F091B003099537
:100F000082E08093E4012DB73EB72A5F3F4F2DBFAB
:100F1000F801838180788383219624E030E0E20E1B
:100F2000F31E075F1F4FCC30D10588F20E94F804F2
:100F3000909152068091B001981728F48091C903CE
:100F400080618093C903993020F088E080933B0151
:100F500002C090933B0185EA91E09F938F93CCE888
:100F6000D1E1DF93CF93E091AF03F091B003099506
:100F700088EE93E00E9461157C010E94C4190F90D5
:100F80000F900F900F90C7010E946A158823D9F324
:100F900085EC91E09F938F93DF93CF93E091AF0324
:100FA000F091B003099580E00E940531289880ED0A
:100FB00097E09093E7018093E60185E58093E50350
:100FC0008EE090E00E9465269927182F00278FE079
:100FD00090E00E946526080F111D1093B601009342
:100FE000B5018AE090E00E9465269927182F002716
:100FF0008BE090E00E946526080F111D1093B4014C
:101000000093B3010F900F900F900F900F5F1F4F41
:1010100039F08091B5019091B6018F5F9F4F41F4F7
:101020001092B6011092B5011092B4011092B30162
:101030008091B3019091B4019F938F938091B501FA
:101040009091B6019F938F938AEC91E09F938F9339
:10105000DF93CF93E091AF03F091B00309950E9425
:10106000481E88E893E190933A0180933901C1E0EA
:10107000C093E4038C2F0E94380580917A060E9469
:10108000EC700E94F80480ED97E00E9461157C01ED
:101090008AEF90E00E94611583E08093AC05109286
:1010A000AF018091CD062DB73EB7285F3F4F2DBFD2
:1010B00084FF02C0C093B90112BC11BC8091BB0176
:1010C000882311F04798FECF8091EA01882309F424
:1010D00060C280911501882309F45BC2F894809165
:1010E000EA0181508093EA0178948091E303882398
:1010F00019F00E940A0502C00E943A3F0E948D3BEF
:10110000289880918A02882331F080918A02815048
:1011100080938A020EC080916F00806280936F007E
:101120001092DC071092DB078091C90388608093DE
:10113000C9038091390190913A01019790933A0146
:10114000809339018091390190913A01892B21F0E6
:10115000809136028823C9F18091390190913A013A
:10116000892BD9F40E944B2985E090E090933A01B5
:10117000809339018091E6059091E705019690935F
:10118000E7058093E6058091C90381608093C903D8
:101190008091AD0582608093AD0580910B019091A7
:1011A0000C018F5F9F4F91F480918902882371F029
:1011B00088EA91E69093E7018093E60180E890E069
:1011C00090930C0180930B0101C028980E946872D3
:1011D0008091EA01882309F0DAC18091E501882332
:1011E00011F40E94366180911101882311F00E9450
:1011F00024160E94DE110E94650DC7010E946A1527
:10120000882309F4C0C184E190E0E80EF91E0E9431
:10121000E21580913602882329F4809160098E318D
:1012200050F405C08091C90382608093C903809106
:10123000AD0582600FC08091E6019091E701892B96
:1012400059F48091390190913A01079728F08091E3
:10125000AD058D7F8093AD058091B901882361F044
:1012600080918A02873940F01092B90188E893E1B1
:101270009093E7018093E60180910601882321F095
:101280008150809306012EC08093EF0310925D027F
:1012900010925C0210925B0210925A021092590254
:1012A0001092580280918A028823E1F480910B0108
:1012B00090910C018F5F9F4FA9F42091B9012230CA
:1012C00089F088E99AE39093E7018093E60180E052
:1012D0009CE090930C0180930B01222319F082E093
:1012E0008093B90180919F01893C70F08150809377
:1012F0009F018091C9038B7F8093C9038091CC03A8
:1013000081608093CC0351C08091E2088823F9F07A
:101310008091C90384608093C90389E080936A0344
:1013200080910B0190910C018F5F9F4F81F4809110
:101330008902882361F088E99AE39093E70180931A
:10134000E60180E098EA90930C0180930B011092E3
:101350005D0310925C0310925B0310925A0310928B
:1013600059031092D5088FEF80934A0910921409FF
:101370001092130910921609109215098FEF9FEF22
:1013800090931209809311091092790210927A02B7
:1013900010927B0210927C0210927D028091CC030D
:1013A0008E7F8093CC0310929F0160910201262FC3
:1013B0003327809123019091240128173907F4F0F5
:1013C0008091510280628093510280910B01909133
:1013D0000C018F5F9F4F91F4809123019091240124
:1013E0000B9764F080E797E19093E7018093E60123
:1013F00080E093E090930C0180930B018091BA01FF
:101400008F5F8093BA01813309F074C01092BA01E2
:101410008091510281FF0AC08091B1019091B20187
:1014200001969093B2018093B10104C05AEA852ECF
:1014300055E0952E80915202909153028050944035
:1014400008F049C02091F5053091F6054091F70567
:101450005091F80580911B0190911C01A0911D01F4
:10146000B0911E01281739074A075B0764F4809181
:10147000F5059091F605A091F705B091F805059650
:10148000A11DB11D20C02091F5053091F6054091B8
:10149000F7055091F80580911B0190911C01A091D6
:1014A0001D01B0911E0182179307A407B5079CF494
:1014B0008091F5059091F605A091F705B091F8059A
:1014C0000597A109B1098093F5059093F605A093BE
:1014D000F705B093F805862F9927019620912301EF
:1014E00030912401821793072CF4809151028F7D53
:1014F000809351020894811C911C82E788168BE02E
:10150000980609F040C0882499242091B5013091B3
:10151000B6012F5F3F4F3093B6012093B501809104
:10152000B3019091B40101969093B4018093B301FB
:10153000832F9927682F8EE090E00E946D2680917E
:10154000B5019091B6019070682F8FE090E00E94F5
:101550006D268091B3019091B401892F9927682F4E
:101560008AE090E00E946D268091B3019091B401D1
:101570009070682F8BE090E00E946D2684E190E0EF
:101580000E9461157C010E945B660E94106B7110C5
:101590007A94772039F40E941F66882319F08CE032
:1015A000782E8ACD8091E501882309F085CD0E94AF
:1015B000366182CD1F920F920FB60F9211248F9336
:1015C0009F93EF93FF93809108018823E1F480912A
:1015D000D5019091D60101969093D6018093D501C3
:1015E000FC01E053FB4FE081ED3019F08C3D91059B
:1015F00039F41092D6011092D50181E08093080150
:10160000E093C60004C01092D6011092D501FF915C
:10161000EF919F918F910F900FBE0F901F90189593
:101620001F920F920FB60F9211242F933F934F9357
:101630005F936F937F938F939F93AF93BF93CF935A
:10164000EF93FF9390E08091BB01813029F480916A
:10165000C6008093CE00D1C08091BB01823029F4B6
:101660008091C6008093F203C8C08091C600809329
:10167000CD015091DB015C3D10F09093DC01809135
:10168000CD018D3009F06AC08091DC01823009F013
:1016900065C09093DC01852F99278E509C4FFC01EB
:1016A000329740812091D7013091D801241B310914
:1016B000DC0111978C91281B3109C9019F7090930F
:1016C000D8018093D70146E0969587954A95E1F732
:1016D000982F935C9093D9012F733070235C2093E3
:1016E000DA018081981729F48C91281711F491E080
:1016F00006C090E08091CA018F5F8093CA018091FB
:10170000CC01882309F079C0992309F476C081E0DF
:101710008093CC01580F5093C9015150E52FFF27FA
:10172000EE50FC4F8DE080838091F403823509F008
:1017300064C0C0918902CC2309F05FC00E94481E9A
:1017400088E190E02CE00FB6F894A89580936000B3
:101750000FBE20936000C093E4014FC02091DC01D4
:10176000822F992781309105F9F0823091051CF480
:10177000892B21F040C0029711F13DC08091CD012D
:10178000833239F48091CC01882319F481E080936D
:10179000DC018091CD018093F20381E08093DB0135
:1017A0008091CD01992722C02F5F2093DC01E52F86
:1017B000FF27EE50FC4F8091CD01808309C0E52FBB
:1017C000FF27EE50FC4F8091CD0180835C3D20F4DB
:1017D0005F5F5093DB0102C01092DC012091CD01CC
:1017E0008091D7019091D801820F911D9093D801DB
:1017F0008093D70102C01092DC01FF91EF91CF914D
:10180000BF91AF919F918F917F916F915F914F9118
:101810003F912F910F900FBE0F901F901895AC0124
:10182000A0E0B0E09D01A817B90748F4E0EDF4E0AE
:101830008191280F311D1196A417B507C8F33F7089
:10184000FD01E053FB4FC90156E0969587955A95E7
:10185000E1F7835C80831196FD01E053FB4F2F730A
:101860003070822F835C8083AF52BB4F8DE08C93AE
:10187000109208018091D0048093C6000895A0E0E2
:10188000B0E0E5E4FCE00C9488752C859D850E8520
:10189000BB2483E28093D0049F599093D10420937A
:1018A000D20433E0E32EF12C002309F49EC0CF8450
:1018B000D888BE016D5E7F4FA989BA890150109703
:1018C00009F493C01097B9F0F601EB0DF11DB39434
:1018D0009081119791F4002349F1FB016E5F7F4FD6
:1018E000DB01C080D1806E5F7F4F0D90BC91A02D39
:1018F000BB24015002C090E019C01097B9F0F60166
:10190000EB0DF11DB3944081119791F4002341F147
:10191000FB016E5F7F4FDB01C080D1806E5F7F4F28
:101920000D90BC91A02DBB24015002C040E018C016
:101930001097B1F0F601EB0DF11DB39410811197E2
:1019400081F4002371F0FB013296DB01CD90DC9035
:10195000BF016E5F7F4FA081B181BB24015001C0E8
:1019600010E0F701E053FB4F892F86958695835C45
:1019700080830894E11CF11CF701E053FB4F892F91
:1019800099278370907024E0880F991F2A95E1F7BA
:1019900055279A0194E0369527959A95E1F7822B81
:1019A000835C80830894E11CF11CF701E053FB4F3A
:1019B0004F705070440F551F440F551F812F9927AA
:1019C00026E0969587952A95E1F7842B835C8083A2
:1019D0000894E11CF11CF701E053FB4F1F73135CEB
:1019E00010830894E11CF11C6ACFC7010E940F0C00
:1019F000E9E00C94A475A3E07A2F4091C901465008
:101A0000442309F458C0E72FFF27EE50FC4F808194
:101A10008D537F5FE72FFF27EE50FC4F20812D5322
:101A20007F5FE72FFF27EE50FC4F30813D537F5FF4
:101A3000E72FFF27EE50FC4F60816D537F5F9927A2
:101A4000880F991F880F991F522F52955F70582B3E
:101A5000822F99278F709070F4E0880F991FFA9564
:101A6000E1F7232F26952695282B832F992783701E
:101A70009070E6E0880F991FEA95E1F7682B4150D6
:101A80004F3FC9F0EA2FFF27EE50FC4F5083AF5F66
:101A900041504F3F81F0EA2FFF27EE50FC4F20834B
:101AA000AF5F41504F3F39F0EA2FFF27EE50FC4F18
:101AB0006083AF5FA5CF85EF93E09093C8018093DB
:101AC000C701A350A093C6010895A2E0B0E0EBE6E1
:101AD000FDE00C948E758091CC01882309F418C424
:101AE0000E94FB0C8091F303823609F0E4C28091DE
:101AF000F40399278037910509F4AFC08137910528
:101B0000C4F48A36910509F441C28B36910544F438
:101B10008B34910571F18636910509F46AC1CBC207
:101B20008D36910509F469C08E36910509F44DC0D2
:101B3000C2C28437910541F1853791054CF4813754
:101B4000910509F491C08337910509F4EAC0B3C245
:101B50008737910509F4DCC1883791052CF4853766
:101B6000910509F498C1A7C28937910509F47DC18F
:101B7000A2C2E091C701F091C80180819181909348
:101B80008F0180938E0197C28091C901A091C701F6
:101B9000B091C801853140F080E1EDECF3E00D90AB
:101BA00001928A95E1F70DC08D919D910D90BC91A8
:101BB000A02D8093CD039093CE03A093CF03B09339
:101BC000D00380EF8093C4014BC08091080188232B
:101BD000E1F38DE490E09F938F938CED96E09F93DB
:101BE0008F9381E08F938F938EE48F930E943F0CAD
:101BF0008DB79EB707968DBF5EC2A091C701B09109
:101C0000C8011C91113081F48DE4ECEDF6E00D90EB
:101C100001928A95E1F70E947C2719838091C9037C
:101C20008F7E8093C90301C01982809108018823A7
:101C3000E1F381E090E09F938F93CE0101969F9313
:101C40008F9381E08F938F938DE48F930E943F0C4D
:101C5000ADB7BEB71796ADBF2EC281E08093CF015E
:101C60008FEF8093060127C2809189028823E1F5D6
:101C7000E091C701F091C801E0818E2F8A508A302F
:101C800058F48983882311F481E003C0863010F072
:101C900085E0898361E00EC08E2F84518A3070F414
:101CA0008983882311F481E003C0863010F085E039
:101CB000898360E089810E94FE2712C0E983EF3F9B
:101CC00019F40E94DF2789838981882311F481E038
:101CD00003C0863010F085E0898389810E948326C5
:101CE00080E00E94380503C00E94DF27898380912D
:101CF00008018823E1F388E890E09F938F9383E5C0
:101D000096E09F938F9381E090E09F938F93CE0115
:101D100001969F938F9382E08F9381E08F9381E56B
:101D20002DC12091C7013091C801D9018C918150FA
:101D3000853008F045C0F9018181863609F040C040
:101D4000809189028823E1F52F5F3F4F88E8E3E522
:101D5000F6E0D9010D9001928A95E1F7F90182919F
:101D60000E94EE26809194069927AA27BB27BC01E2
:101D7000CD0124EC39E040E050E00E94F074DC0139
:101D8000CB018093860190938701A0938801B09343
:101D90008901809195069927AA27BB27BC01CD010F
:101DA0000E94F074DC01CB01809382019093830147
:101DB000A0938401B09385010E94DF27898301C02D
:101DC0001982809108018823E1F381E090E09F93DC
:101DD0008F93CE0101969F938F9381E08F938F9382
:101DE00083E58F930E943F0C8DB79EB707968DBFFA
:101DF0002BC080918902882309F05DC1E091C70161
:101E0000F091C801E0818E2F8150853018F48E2F1B
:101E10000E9483260E94DF278983809108018823FE
:101E2000E1F381E090E09F938F93CE0101969F9321
:101E30008F9381E08F938F9386E48F930E943F0C62
:101E4000ADB7BEB71796ADBF10918902112341F40B
:101E50006EE670E089810E945030812F0E94380523
:101E600080917A060E94EC7026C119822981A09186
:101E7000C701B091C801EBEDF7E08D91992787FD7F
:101E8000909593A382A3822F8F5F8983282F329608
:101E90008C3098F310C1E091C701F091C8018081A6
:101EA0000E94932D8A83882319F481E0898301C0DD
:101EB0001982809108018823E1F388E090E09F93E4
:101EC0008F9386E697E09F938F9321E030E03F93D6
:101ED0002F938091C7019091C8019F938F933F9357
:101EE0002F93CE0102969F938F933F932F93CE0112
:101EF000820F931F9F938F9384E08F9381E08F9342
:101F000085E58F930E943F0CEDB7FEB773963CC0FA
:101F10008091C601893008F4CEC02091C70130916C
:101F2000C8012F5F3F4F88E0A6E6B7E0F9010190B6
:101F30000D928A95E1F7D9018E910E94E32C8A8354
:101F4000882319F481E0898301C0198280910801F6
:101F50008823E1F321E030E03F932F93CE010296F6
:101F60009F938F933F932F93CE01820F931F9F9345
:101F70008F9382E08F9381E08F9387E58F930E9408
:101F80003F0CEDB7FEB73B96EDBF95C0809189023F
:101F9000882309F090C00E94A3708983823019F0D1
:101FA000843009F088C020E430E0F8948091C100CA
:101FB0008F738093C1008091C9008F738093C90093
:101FC0008091C100877E8093C1008091C900877E87
:101FD0008093C9008091C80087FF03C08091CE0024
:101FE000F9CF8091C00087FF03C08091C600F9CF70
:101FF000E091C701F091C801E081E13021F482E075
:102000008093BB012EC0E43611F421E830E081E07A
:102010008093BB01832F99278093CD002093CC0020
:102020008091CD008093C5008091CC008093C40046
:102030008091CA008F7D8093CA008091CA008F7EF4
:102040008093CA008091C9008B7F8093C9008091E2
:10205000CA0084608093CA008091CA008260809325
:10206000CA008091CA00877F8093CA008091C20015
:10207000877F8093C2008091C9008E7F8093C900C2
:102080008091C10088618093C1008091C9008861FE
:102090008093C9008091C10080688093C1008091C5
:1020A000C90080688093C90010926E0010926F0082
:1020B0001092700078948091F403992784369105EA
:1020C00009F4BBC085369105ACF48136910509F45D
:1020D0006FC0823691052CF48B34910509F45DC0F4
:1020E0000FC18236910509F470C08336910509F459
:1020F0007FC006C18C36910509F4EDC08D3691057F
:102100004CF48736910509F4F8C08836910509F436
:10211000B2C0F6C08437910529F08637910509F4DD
:10212000E8C0EEC08091C901A091C701B091C8017B
:10213000803140F080E1EDECF3E00D9001928A9562
:10214000E1F70DC08D919D910D90BC91A02D8093D4
:10215000CD039093CE03A093CF03B093D00380918F
:1021600008018823E1F31F92809105018F9384E594
:102170008F930E943F0C8AEF8093C4018FEF80936E
:10218000060180EA9FE00E9461159093BD01809353
:10219000BC010F900F900F90B3C0E091C701F09178
:1021A000C8018081918190938F0180938E01A8C096
:1021B000E091C701F091C8018081809307018032CE
:1021C00098F08FE1809307010FC0A091C701B091F3
:1021D000C8018BE0E5EEF3E00D9001928A95E1F7FE
:1021E0008091EE038093EE058FEF8093060188C007
:1021F0008091C0019091C101892B89F4E091C701C0
:10220000F091C801E081EE2351F08AE0E89FC0011F
:1022100011240E9461159093C0038093BF03E09145
:10222000C701F091C80190818AE0989FC0011124F4
:102230009093C1018093C00115C08FEF8093060178
:10224000E091C701F091C80190818AE0989FC00198
:1022500011249093C3018093C201892B19F081E06E
:102260008093D10180EA9FE00E9461159093BD01A7
:102270008093BC0145C08FEF80930601E091C701B8
:10228000F091C801908197FD08C082E08093CE0153
:102290001092BF011092BE011AC0909580912E023B
:1022A000892B80932E0291818AE0989FC00111248E
:1022B0009093BF018093BE0184E08093CE0180EAB9
:1022C0009FE00E9461159093BD018093BC0181E065
:1022D0008093D20115C08FEF80930601E091C70172
:1022E000F091C801808180932F0281E08093D30117
:1022F00007C081E08093D00103C081E08093D401C6
:102300001092CC011092C8011092C7011092C60120
:10231000E3E0CE5F0C94AA75982F8091C00085FFF2
:10232000FCCF9093C60008950F931F9388E180938C
:10233000C1008091C00082608093C0008091C10084
:1023400080688093C1008091C10080648093C10047
:1023500000E010E00093C5008AE290E08093C400A2
:102360008091C2019091C3010E9461159093C203B4
:102370008093C1038CED90E00E9461159093F1036E
:102380008093F00382E08093C30386E08093C403CC
:102390001092C7038BE08093C5031092C60310927E
:1023A000CB03809103018093CA031093C80100936B
:1023B000C7011092C6011F910F910895A0E1B0E0EE
:1023C000E4EEF1E10C948D7580910801882309F405
:1023D0008CC28091BC019091BD010E946A15882336
:1023E00061F01092BF011092BE011092C3011092D1
:1023F000C2011092C1011092C0018091BE01909162
:10240000BF01892B41F08091CE049091CF040E94AE
:102410006A15882329F48091D201882309F460C0C9
:1024200080910801882309F45BC08091CE0102E00D
:1024300016E08430A8F00E945E1E80E590E09F9335
:102440008F931F930F9381E08F938F9388E48F93E3
:102450000E943F0C2DB73EB7295F3F4F2DBF34C0C0
:10246000109230028CEE93E09F938F9381E59EE172
:102470009F938F93E091AF03F091B003099584E1AE
:1024800090E09F938F931F930F9381E090E09F9331
:102490008F938EEC91E09F938F9382E08F9381E0F6
:1024A0008F9388E48F930E943F0C8091CE01982FE8
:1024B0008F5F8093CE012DB73EB7215F3F4F2DBF79
:1024C000943010F01092CE018091BE019091BF0126
:1024D0000E9461159093CF048093CE041092D20194
:1024E0008091D301882351F180910801882331F133
:1024F0000E945E1E80E590E09F938F9382E096E0BD
:102500009F938F9321E030E03F932F9385E291E0FA
:102510009F938F933F932F938FE292E09F938F939C
:1025200083E08F9381E08F938CE48F930E943F0C24
:102530001092D3018DB79EB70F968DBF8091D001B9
:102540008823D1F0809108018823B1F08AE090E0DF
:102550009F938F9383EC93E09F938F9381E08F936E
:102560008F9386E58F930E943F0C1092D0012DB778
:102570003EB7295F3F4F2DBF8091D4018823D9F00A
:10258000809108018823B9F08BE090E09F938F93AE
:1025900085EE93E09F938F9381E08F938091050167
:1025A0008F9387E48F930E943F0C1092D4018DB7D4
:1025B0009EB707968DBF8091C2019091C301892B70
:1025C00041F08091C1039091C2030E946A15882353
:1025D00021F48091D101882341F180910801882361
:1025E00021F10E94622F82E490E09F938F938CEA06
:1025F00095E09F938F9381E08F938F9384E48F93E3
:102600000E943F0C1092D1012DB73EB7295F3F4F7A
:102610002DBF8091C2019091C301009731F00E94BB
:1026200061159093C2038093C1038091C001909182
:10263000C101892B09F497C08091BF039091C00319
:102640000E946A15882309F48EC0809108018823AE
:1026500009F489C08091E8089091E9089093B20349
:102660008093B1038091EA089091EB089093B403B2
:102670008093B3032091CA083091CB084091CC08D5
:102680005091CD08DA01C90163E0880F991FAA1F94
:10269000BB1F6A95D1F7820F931FA41FB51F820F2E
:1026A000931FA41FB51F209140013091410140911B
:1026B000420150914301BC01CD010E9464753093E9
:1026C000B6032093B5038091AC029091AD02A09126
:1026D000AE02B091AF0249E0B595A7959795879561
:1026E0004A95D1F78093B7038091A8029091A902EF
:1026F000A091AA02B091AB0239E0B595A795979544
:1027000087953A95D1F78093B8038091B402909160
:10271000B502A091B602B091B70229E0B595A79590
:10272000979587952A95D1F78093B9038EE090E02D
:102730009F938F9381EB93E09F938F9381E08F938F
:102740008F9383E48F930E943F0C8091C0019091FE
:10275000C1010E9461159093C0038093BF038DB7A0
:102760009EB707968DBF809107018F3F79F199271A
:1027700004E0880F991F0A95E1F784519E4F40E1CC
:1027800050E0BC01CE0101960E94437380E190E0CD
:102790009F938F93CE0101969F938F9381E090E05A
:1027A0009F938F9387E091E09F938F9382E08F9325
:1027B00081E08F9381E48F930E943F0C8FEF809391
:1027C00007012DB73EB7255F3F4F2DBF8091EE0526
:1027D0008823C9F0809108018823A9F081E090E066
:1027E0009F938F938EEE95E09F938F9381E08F93CD
:1027F0008F9382E48F930E943F0C1092EE058DB769
:102800009EB707968DBF8091CF018823D1F080912C
:1028100008018823B1F086E490E09F938F938BEDBD
:1028200097E09F938F9381E08F938F9380E58F93B1
:102830000E943F0C1092CF012DB73EB7295F3F4F4A
:102840002DBF8091F0039091F1030E946A158823B7
:1028500009F44BC080910801882309F446C0809197
:102860009F01882361F58091E8089091E908909391
:10287000DE038093DD038091EA089091EB0890934A
:10288000E0038093DF03809166028093E1038091EF
:1028900065028093E20388E090E09F938F938DED33
:1028A00093E09F938F9381E08F9383E08F938BE6E8
:1028B0008F930E943F0C8DB79EB707968DBF809176
:1028C000E303853018F086E08093E3038091E30111
:1028D000882319F083E690E002C087EE93E00E941F
:1028E00061159093F1038093F003E4E0C05F0C94D2
:1028F000A9751F920F920FB60F9211242F933F9339
:102900005F936F937F938F939F93AF93BF93EF9357
:10291000FF938091E501882329F08091E5018150A2
:102920008093E50180917F03882319F08150809383
:102930007F038091ED0181508093ED018F3F09F07D
:1029400051C089E08093ED018091EB019091EC0101
:1029500001969093EC018093EB01809112018F5FBF
:10296000817080931201882349F48091EA018430B8
:1029700028F48091EA018F5F8093EA01349903C0C3
:1029800081E08093E3018091E6019091E701892B3A
:1029900011F18091E6019091E7010B9750F0809141
:1029A000E6019091E7010A979093E7018093E60191
:1029B00004C01092E7011092E6018091E601909127
:1029C000E70120910B0130910C0182239323892B85
:1029D00041F0479A07C08FEF9FEF90930C018093CF
:1029E0000B0147988091E301882309F45AC0209194
:1029F0009F01222309F055C08091B80883FF51C080
:102A000086B19927FC01E071F07084FF13C08091BA
:102A1000E8019091E90101969093E9018093E80122
:102A20008091E8019091E901895E9340D0F1209373
:102A3000E30137C08091E8019091E901892B69F1A8
:102A40008091E8019091E9018A56914030F580919A
:102A5000E8019091E90169E270E00E941B758091A4
:102A6000E8019091E901860F971F9093E901809307
:102A7000E8018091E8019091E9010B9750F0809175
:102A8000E8019091E9010A9790938F0180938E015C
:102A900004C0F0938F01E0938E011092E90110922F
:102AA000E801FF91EF91BF91AF919F918F917F913D
:102AB0006F915F913F912F910F900FBE0F901F90DC
:102AC00018952091EB013091EC01280F391FC901B5
:102AD000019608952091EB013091EC01821B930B3C
:102AE000892F99278695807490700895CF93DF93EE
:102AF0000E946115EC01CE010E946A158823D9F36A
:102B0000DF91CF910895CF93DF930E946115EC017F
:102B100009C080911501882329F0909315018FEC4D
:102B200080937A00CE010E946A15982F882389F33A
:102B3000DF91CF9108959FB7F8945F983E9A469A97
:102B40008091B0008F708093B0008091B00083605E
:102B50008093B0008091B1008B738093B10080911D
:102B6000B1008B608093B1001092B2008FEF809320
:102B7000B3008091B00080688093B00080917000B5
:102B80008A7F8093700080917000826080937000D3
:102B90009FBF08958AE090E00E9461159093F00530
:102BA0008093EF0582E085BD83EB84BD8FEF88BD08
:102BB00084EB87BD86E086BD80916E008160809346
:102BC0006E0008958091CC0620916D0182FF30C087
:102BD000909183068CE3989FB00111249091820616
:102BE00080E5989FA0011124922F905897FD9D5F3A
:102BF0009595959586E09802C001112420910901D0
:102C000030910A01281B390B30930A0120930901E6
:102C1000421753072CF050930A014093090108957D
:102C20002617370784F070930A016093090108950D
:102C3000822F992736E0880F991F3A95E1F79093F4
:102C40000A01809309010895EF92FF920F931F9359
:102C5000CF93DF9380918A06E82FFF27EA5BFE4F30
:102C60009681C08180911101813009F021C180914C
:102C7000CE0687FF05C0C0E0D0E0E0E0F0E046C04F
:102C8000892F992787FD9095A92FB92F2091E402CC
:102C90003091E5024091E6025091E702BC01CD017E
:102CA0000E94F07497FF04C061587F4F8F4F9F4F71
:102CB0007B018C0187E015950795F794E7948A9539
:102CC000D1F78C2F992787FD9095A92FB92F2091A7
:102CD000DC023091DD024091DE025091DF02BC0146
:102CE000CD010E94F07497FF04C061587F4F8F4F51
:102CF0009F4FB7E09595879577956795BA95D1F7EA
:102D0000F801E701C61BD70BE80BF90B2091640310
:102D100030916503C901A3E0880F991FAA95E1F7D7
:102D2000821B930BAA2797FDA095BA2FC81BD90B1E
:102D3000EA0BFB0B80916B019927AA27BB27BC01EB
:102D4000CD019E01AF010E94F07497FF04C0615055
:102D50007E4F8F4F9F4FFC01EB0179E0F595E79592
:102D6000D795C7957A95D1F71091CC066091090156
:102D700070910A0112FF05C07093100160930F015A
:102D800018C040910F015091100180918906282FA1
:102D90003327CB01841B950BB9010E942F758091BD
:102DA0000F0190911001860F971F9093100180934F
:102DB0000F0110FF14C080910F019091100197FD39
:102DC0000F9664E0959587956A95E1F7AA2797FD98
:102DD000A095BA2FC80FD91FEA1FFB1F15C08091FD
:102DE0000F019091100197FD0F9654E095958795EE
:102DF0005A95E1F7AA2797FDA095BA2F8C1B9D0B3A
:102E0000AE0BBF0BFD01EC012091BE06222321F188
:102E100033278091DF019091E001829FA001839F81
:102E2000500D929F500D1124CA01AA2797FDA0951D
:102E3000BA2F8C0F9D1FAE1FBF1F2F5F3F4F442720
:102E400037FD4095542FBC01CD010E94647530932D
:102E5000E0012093DF0104C0D093E001C093DF01C3
:102E600080918206282F3327220F331F220F331F12
:102E70008091DF019091E001821793077CF08091AF
:102E80008306282F3327220F331F220F331F8091F1
:102E9000DF019091E0012817390724F43093E00115
:102EA0002093DF01809111018F5F80931101F9C0A0
:102EB000892F992787FD9095A92FB92F2091DC02A2
:102EC0003091DD024091DE025091DF02BC01CD0164
:102ED0000E94F07497FF04C061587F4F8F4F9F4F3F
:102EE0007B018C0187E015950795F794E7948A9507
:102EF000D1F78C2F992787FD9095A92FB92F209175
:102F0000E4023091E5024091E6025091E702BC01F3
:102F1000CD010E94F0749B01AC0197FF04C02158C1
:102F20003F4F4F4F5F4FC7E05595479537952795D2
:102F3000CA95D1F72E0D3F1D401F511F80916A0188
:102F40009927AA27BB27BC01CD010E94F07497FFE7
:102F500004C061507E4F8F4F9F4FFC01EB01B9E0E1
:102F6000F595E795D795C795BA95D1F780916C01FE
:102F70009927A6E0880F991FAA95E1F740910D01C6
:102F800050910E01209189063327841B950BB901BE
:102F90000E942F7580910D0190910E01860F971F51
:102FA00090930E0180930D018091CC0681FF14C097
:102FB00080910D0190910E0197FD0F9674E095950B
:102FC00087957A95E1F7AA2797FDA095BA2FC80FA4
:102FD000D91FEA1FFB1F15C080910D0190910E01B2
:102FE00097FD0F9664E0959587956A95E1F7AA2776
:102FF00097FDA095BA2F8C1B9D0BAE0BBF0BFD014F
:10300000EC012091BF06222321F133278091DD01BD
:103010009091DE01829FA001839F500D929F500DE1
:103020001124CA01AA2797FDA095BA2F8C0F9D1FC6
:10303000AE1FBF1F2F5F3F4F442737FD4095542FD2
:10304000BC01CD010E9464753093DE012093DD0147
:1030500004C0D093DE01C093DD0180918606282F45
:103060003327220F331F220F331F8091DD019091F0
:10307000DE01821793077CF080918706282F332783
:10308000220F331F220F331F8091DD019091DE014B
:103090002817390724F43093DE012093DD011092C4
:1030A0001101E6E0CDB7DEB70C94A7751F920F9221
:1030B0000FB60F9211242F933F934F935F938F93EB
:1030C0009F93EF93FF938091EE01882309F0DDC079
:1030D0008091B00086FF9FC08091B0008F7B80936D
:1030E000B000E091F10120918806EE23D9F4332756
:1030F0008DED96E0289FA001299F500D389F500D1F
:103100001124CA012091EF013091F001821B930B31
:103110009093E2018093E1011092F0011092EF018F
:10312000469AB0C02E1738F48AE090E09093E201FE
:103130008093E101A7C089EA93E09093E201809334
:10314000E1018E2F992783309105D9F084309105C4
:1031500034F48130910549F0029761F020C0843049
:10316000910591F0059799F01AC08091DF01909137
:10317000E00104C08091DD019091DE0187559E4FF2
:103180001DC08091940805C080916D0802C0809197
:103190009D089927880F991F880F991FEFCFFF2748
:1031A000EE0FFF1FE552F84F20813181220F331FB0
:1031B0008091E1019091E201820F931F9093E201CF
:1031C0008093E1018091E1019091E20155E08D3D14
:1031D000950718F08CED95E005C08757914030F4C5
:1031E00087E791E09093E2018093E1012091E10172
:1031F0003091E2012C5B30403093E2012093E101F9
:103200008091EF019091F001820F931F9093F00154
:103210008093EF0137C08091B00080648093B0004C
:103220008CEB90E09093E2018093E1018091EF01BB
:103230009091F00184549F4F9093F0018093EF019F
:103240008091E401882321F080918A02882321F46F
:103250008091E401823011F4469801C0469A809131
:10326000F1018F5F8093F101282F33278091880629
:1032700099270196821793072CF481E0809311011E
:103280001092F10181E08093EE012091E1013091F3
:10329000E20141E02F37340730F08FEF8093B30025
:1032A0002F5F30400FC02F3F3105C9F0C0F0A9019A
:1032B0004F5F50404F37510550F480E88093B30082
:1032C000205830403093E2012093E10112C08FEF8B
:1032D0008093B3005093E2014093E1010AC08091D2
:1032E000E1018093B3001092E2011092E10110928B
:1032F000EE01FF91EF919F918F915F914F913F91DF
:103300002F910F900FBE0F901F90189510927C0078
:103310008FEC80937A0008958091490260911301A7
:10332000709114012091FE01882379F0CB01AA2726
:10333000BB27332727FD3095432F532FBC01CD01E9
:103340000E94F074DC01CB0116C084E0660F771F89
:103350008A95E1F7CB01AA27BB27332727FD3095B4
:10336000432F532FBC01CD010E94F074DC01CB012F
:103370000497A109B1098093F6019093F701A093F6
:10338000F801B093F9010895CF93DF931092FE01F5
:103390000E948C1983E090E00E946526C82FDD27EB
:1033A000C03FD10508F42A96C7BD8C2F809588BDF3
:1033B00086E990E00E9483158091190190911A018D
:1033C0008152934010F0C0EFD0E0C630D10510F12B
:1033D000C7BD8C2F809588BD84E690E00E94831540
:1033E00081E094E09F938F938CE891E19F938F937A
:1033F000E091AF03F091B00309958091190190918C
:103400001A010F900F900F900F908152934010F47B
:103410002197DBCFC093FF056C2F83E090E00E94E3
:103420006D268091600680FF0AC08091FF058A505A
:103430008C3D28F08091C80380648093C8038CE29F
:1034400091E00E948315DF91CF9108951F920F9212
:103450000FB60F9211242F933F934F935F936F9367
:103460007F938F939F93AF93BF93CF93DF93EF930C
:10347000FF9380911602282F3327442755278F5F0B
:1034800080931602F9012231310508F0DEC3E25CB7
:10349000FF4F0C94B675809178009091790046C0EA
:1034A00080917800909179007BC180917800909113
:1034B000790090931A02809319028BC18091EE02D9
:1034C0009091EF022091780030917900821B930B4C
:1034D0009093F2058093F1058091F1059091F205AA
:1034E000909324028093230292C18091780090915E
:1034F00079002091F0023091F102821B930B90939E
:10350000FE058093FD058091FD059091FE05909349
:103510002602809325029BC380911D0290911E027A
:103520002091780030917900820F931F90931E02B2
:1035300080931D0281E08CC380911B0290911C023C
:103540002091780030917900820F931F90931C0294
:1035500080931B0284E07CC380912C0290912D0209
:10356000892B91F42091780030917900C901E3E032
:10357000880F991FEA95E1F7820F931F820F931F1F
:1035800090932D0280932C02209178003091790045
:10359000C90173E0880F991F7A95E1F7820F931F95
:1035A000820F931F20912C0230912D0282179307D6
:1035B00018F02E5F3F4F02C02250304030932D0252
:1035C00020932C0280912C0290912D026FE170E0EB
:1035D0000E941B75709324016093230185E038C31A
:1035E00080917800909179009093F4058093F30591
:1035F0008091F3059091F4054091EA025091EB021D
:10360000841B950B2091E902332727FD3095821BFF
:10361000930B9093040280930302809149028823C4
:1036200009F06DC0809103029091040202977CF131
:1036300022E04E3E52070CF062C0209117023091FA
:1036400018022B5F3F4F309318022093170225502A
:1036500030408091520290915302845F914030F447
:10366000215F3F4F30931802209317028091170279
:1036700090911802853691050CF441C04F5F5F4F61
:103680005093EB024093EA028456904034C08091FC
:103690000302909104028F5F9F4F8CF562E04732E6
:1036A00056076CF1209117023091180225503040D6
:1036B00030931802209317022B5F3F4F80915202E4
:1036C00090915302845F914030F42F5030403093FA
:1036D00018022093170280911702909118022FEF81
:1036E0008C39920764F4415050405093EB02409360
:1036F000EA028C599F4F9093180280931702809191
:103700000302909104029C01442737FD4095542FF9
:103710008091A4029091A502A091A602B091A70267
:10372000820F931FA41FB51F8093A4029093A5023C
:10373000A093A602B093A7022091A4023091A50203
:103740004091A6025091A70257FF04C021503C4F60
:103750004F4F5F4F6AE055954795379527956A9586
:10376000D1F78091A4029091A502A091A602B091F8
:10377000A702821B930BA40BB50B8093A40290931A
:10378000A502A093A602B093A702F5C080911B02E8
:1037900090911C022091780030917900820F931F44
:1037A00090931C0280931B021092150253C2209129
:1037B0007800309179008091190290911A02280FB7
:1037C000391F8FEF97E0821B930B90930A0280932F
:1037D000090286E03DC28091EE029091EF022091B5
:1037E000780030917900821B930B9093F2058093BF
:1037F000F1058091F1059091F2052091230230911D
:103800002402820F931F909308028093070287E09F
:103810001FC280917800909179002091F002309140
:10382000F102821B930B9093FE058093FD0580911E
:10383000FD059091FE052091250230912602820F10
:10384000931F909306028093050201C220911D02EE
:1038500030911E028091780090917900280F391FD5
:10386000220F331F220F331F30931E0220931D029D
:10387000C90137FD079643E0959587954A95E1F78D
:1038800090930E0280930D0280911F02909120026E
:10389000820F931F97FD019695958795909320022F
:1038A00080931F022091FA023091FB02821B930B3E
:1038B00090932201809321012091130230911402F0
:1038C0008091210190912201280F391F37FF02C0FA
:1038D0002F5F3F4F359527953093140220931302A5
:1038E00029CE20911B0230911C028091780090918A
:1038F0007900280F391F220F331F220F331F3093F7
:103900001C0220931B02C90137FD0796F3E0959531
:103910008795FA95E1F790930C0280930B028091C2
:10392000210290912202820F931F97FD0196959597
:10393000879590932202809321022091F802309182
:10394000F902821B930B9093200180931F01209119
:1039500011023091120280911F0190912001280FD5
:10396000391F37FF02C02F5F3F4F359527953093A2
:1039700012022093110283E06BC180918402909126
:103980008502A0918602B09187028093F201909304
:10399000F301A093F401B093F5011092160281E0B7
:1039A000809315018091FA019091FB01019690930B
:1039B000FB018093FA0180917800909179009093B7
:1039C0001A01809319018091190190911A01AA2777
:1039D000BB27C0912702D0912802E0912902F091E3
:1039E0002A02C80FD91FEA1FFB1FC0932702D093DA
:1039F0002802E0932902F0932A0280912B028F5F24
:103A000080932B02803108F422C180911B01909198
:103A10001C01A0911D01B0911E019C01AD0163E04C
:103A2000220F331F441F551F6A95D1F7281B390BEE
:103A30004A0B5B0B2C0F3D1F4E1F5F1F8091F60141
:103A40009091F701A091F801B091F901281B390B71
:103A50004A0B5B0B57FF04C0295F3F4F4F4F5F4F2F
:103A600093E055954795379527959A95D1F72093EB
:103A70001B0130931C0140931D0150931E01C09106
:103A8000F505D091F605E091F705F091F8058091E4
:103A90001B0190911C01A0911D01B0911E01C81B3A
:103AA000D90BEA0BFB0BC0938402D0938502E09301
:103AB0008602F09387022091FF013091000240912D
:103AC00001025091020257FF04C0215F3F4F4F4F48
:103AD0005F4F84E055954795379527958A95D1F79F
:103AE0008091FF0190910002A0910102B091020229
:103AF000821B930BA40BB50B8093FF0190930002E4
:103B0000A0930102B09302028091FF019091000204
:103B1000A0910102B09102028C0F9D1FAE1FBF1F2A
:103B20008093FF0190930002A0930102B0930202E0
:103B30008091FF0190910002A0910102B0910202D8
:103B4000B7FF03C00F96A11DB11DC4E0B595A795A1
:103B500097958795CA95D1F7209184023091850277
:103B6000281B390B64E0213036071CF020E034E0DC
:103B700006C08CEF2030380714F420E03CEF809131
:103B8000FC019091FD018091FC019091FD0197FF56
:103B900003C0909581959F4FA901F3E0440F551FF5
:103BA000FA95E1F78D5B9240C4F08091FC01909111
:103BB000FD019C01E4E0220F331FEA95E1F7281B89
:103BC000390B240F351F37FF02C0215F3F4F74E0D0
:103BD000359527957A95E1F717C08091FC01909172
:103BE000FD019C0165E0220F331F6A95E1F7281B58
:103BF000390B240F351F37FF02C0215E3F4F45E0D0
:103C0000359527954A95E1F73093FD012093FC0106
:103C10008091270290912802A0912902B0912A0256
:103C2000B7FF03C00196A11DB11DB595A795979546
:103C300087958093270290932802A0932902B0933E
:103C40002A0288E080932B0202C01092160282E0C2
:103C5000809315028091150280937C00809116025A
:103C6000882319F08FEC80937A00FF91EF91DF9118
:103C7000CF91BF91AF919F918F917F916F915F9104
:103C80004F913F912F910F900FBE0F901F9018955D
:103C900090E2E2E0F6E08FE49193815087FFFCCF61
:103CA000089590913002903540F4E92FFF27EE5FA0
:103CB000F94F80839F5F909330020895A0E0B0E0B9
:103CC000E4E6FEE10C94897520912E0220FF0AC0E3
:103CD00080912F02882311F0815002C0809125012C
:103CE00080932F0221FF0CC090912F02809125011B
:103CF000981719F410922F0203C09F5F90932F0220
:103D0000822F992780FF04C081FF02C010922F02EA
:103D10000E94481E80912F02282F332701E51EE1C3
:103D2000C091AF03D091B0038A3098F481E18093C1
:103D300030023F932F9383E094E09F938F931F93E0
:103D40000F93FE0109952DB73EB72A5F3F4F2DBF58
:103D500011C080E1809330023F932F9388E094E07C
:103D60009F938F931F930F93FE0109958DB79EB775
:103D700006968DBF20912F02822F9927AA27BB2755
:103D8000FC010D9708F096C5E05BFF4F01E51EE1D1
:103D9000C091AF03D091B0030C94B675109230026D
:103DA0008DE094E09F938F9351E5E52E5EE1F52E33
:103DB0001F930F93FE01099584E1809330020F90C9
:103DC0000F900F900F9081E690E09F938F9386E085
:103DD00090E09F938F9382E090E09F938F938091E8
:103DE00003016AE00E940F75892F99279F938F9393
:103DF000809103010E940F7599279F938F938DE106
:103E000094E09F938F931F930F93E091AF03F091F2
:103E1000B003099588E280933002EDB7FEB73E9675
:103E2000EDBF8DED96E09F938F93809101019927CF
:103E30009F938F9385E394E09F938F931F930F93AA
:103E4000E091AF03F091B00309958091C9032DB7BC
:103E50003EB7285F3F4F2DBF84FF0AC08CE380939D
:103E6000300283E494E09F938F931F930F933DC0A0
:103E70009091C803992351F08CE380933002892FED
:103E800099279F938F9380E594E047C090913602E5
:103E9000992351F08CE380933002892F99279F93C7
:103EA0008F9387E694E02EC190916A03992371F075
:103EB0008CE380933002892F99279F938F938DE70E
:103EC00094E09F938F93FF92EF9288C38091390182
:103ED00090913A01069798F48CE3809330028EE833
:103EE00094E09F938F93FF92EF92E091AF03F09154
:103EF000B00309950F900F900F900F90E4C490912C
:103F000060099E3108F0DFC48CE380933002892F72
:103F100099279F938F938BE994E09F938F93FF92C0
:103F2000EF92E091AF03F091B00309958DB79EB782
:103F300006968DBFC8C41092300280918402909181
:103F40008502A0918602B0918702BC01CD0125E0D7
:103F500030E040E050E00E9464753F932F938FEA79
:103F600094E09F938F931F930F93FE01099584E133
:103F700080933002EDB7FEB73696EDBF8091800298
:103F800090918102A0918202B0918302BC01CD0187
:103F900025E030E040E050E00E9464753F932F93AD
:103FA0008CEB94E09F938F931F930F93E091AF035B
:103FB000F091B003099588E2809330022DB73EB7A7
:103FC0002A5F3F4F2DBF8091190190911A019F9355
:103FD0008F9389EC94E09F938F931F930F93E091BD
:103FE000AF03F091B00309958CE3809330028DB755
:103FF0009EB706968DBF87B599279F938F9386EDC1
:1040000094E09F938F931F930F93E091AF03F091F0
:10401000B0030995EDB7FEB7369690C31092300203
:1040200083EE94E09F938F9341E5E42E4EE1F42ECE
:104030001F930F93FE01099584E1809330020F9046
:104040000F900F900F908091E4029091E502A09163
:10405000E602B091E702B7FF04C081509C4FAF4F1A
:10406000BF4F3AE0B595A795979587953A95D1F7C3
:10407000BF93AF939F938F9380EF94E09F938F9321
:10408000FF92EF92E091AF03F091B003099588E2BF
:10409000809330022DB73EB7285F3F4F2DBF8091F0
:1040A000DC029091DD02A091DE02B091DF02B7FF49
:1040B00004C081509C4FAF4FBF4F2AE0B595A795E4
:1040C000979587952A95D1F7BF93AF939F938F9339
:1040D0008FEF94E09F938F93FF92EF92E091AF0365
:1040E000F091B00309958CE3809330028DB79EB7B1
:1040F00008968DBF8091C1089091C2089F938F93BD
:104100008EE095E09F938F93FF92EF927ECF91E0A8
:10411000F92EC1E0D0E00DED17E09F2D969584E1DA
:10412000989FC001112480933002F801828193810D
:104130009F938F932196DF93CF93219780819181D5
:104140009F938F93DF93CF938DE195E09F938F9310
:1041500081E59EE19F938F93E091AF03F091B003CF
:1041600009952DB73EB7245F3F4F2DBF32E0F30EC8
:1041700022960C5F1F4F88E08F1578F6A4C310922B
:10418000300280915506E82FFF27EE0FFF1FE55202
:10419000F84F808191819F938F9380915406E82FEF
:1041A000FF27EE0FFF1FE552F84F808191819F930B
:1041B0008F938FE295E09F938F931F930F93FE0150
:1041C000099584E180933002EDB7FEB73896EDBFD4
:1041D00080915706E82FFF27EE0FFF1FE552F84F9B
:1041E000808191819F938F9380915606E82FFF27BE
:1041F000EE0FFF1FE552F84F8081918181589F4F4C
:104200009F938F938FE395E09F938F931F930F93CB
:10421000E091AF03F091B003099588E280933002FA
:104220002DB73EB7285F3F4F2DBF80915906E82F2D
:10423000FF27EE0FFF1FE552F84F808191818158D3
:104240009F4F9F938F9380915806E82FFF27EE0F83
:10425000FF1FE552F84F8081918181589F4F9F93B6
:104260008F938FE495E09F938F931F930F93E0912B
:10427000AF03F091B00309958CE3809330028DB7C2
:104280009EB708968DBF80915B06E82FFF27EE0F43
:10429000FF1FE552F84F8081918181589F4F9F9376
:1042A0008F9380915A06E82FFF27EE0FFF1FE552EC
:1042B000F84F8081918181589F4F9F938F938FE515
:1042C00095E030C2109230028FE695E09F938F9375
:1042D00081E5E82E8EE1F82E1F930F93FE010995DC
:1042E00084E1809330020F900F900F900F90809197
:1042F000FA029091FB029C0197FF02C0215F3F4FA1
:10430000207F821B930B97FD0196959587959F9330
:104310008F938091FA029091FB0297FD0F96B4E083
:1043200095958795BA95E1F79F938F932091FA021F
:104330003091FB0237FF02C0295F3F4FA3E0359564
:104340002795AA95E1F780910D0290910E02821BAC
:10435000930B9F938F938DE795E09F938F93FF929D
:10436000EF92E091AF03F091B003099588E280935A
:1043700030022DB73EB7265F3F4F2DBF8091F80228
:104380009091F9029C0197FF02C0215F3F4F207F6F
:10439000821B930B97FD0196959587959F938F931D
:1043A0008091F8029091F90297FD0F96E4E09595BF
:1043B0008795EA95E1F79F938F932091F8023091CA
:1043C000F90237FF02C0295F3F4F73E0359527950B
:1043D0007A95E1F780910B0290910C02821B930B6E
:1043E0009F938F938FE895E09F938F93FF92EF9227
:1043F000E091AF03F091B00309958CE38093300214
:104400008DB79EB70A968DBF8091F6029091F70204
:1044100097FD0196959587959F938F938091F602CE
:104420009091F7022091090230910A02821B930BAE
:104430009F938F9381EA95E09F938F93FF92EF92E2
:1044400075C11092300280EB95E09F938F931F937C
:104450000F93FE01099584E1809330020F900F9035
:104460000F900F908091F0029091F1029F938F93A3
:1044700080910502909106029F938F938DEB95E0BA
:104480009F938F931F930F93E091AF03F091B0032D
:10449000099588E2809330022DB73EB7285F3F4FE1
:1044A0002DBF8091EE029091EF029F938F938091A8
:1044B0000702909108029F938F938CEC95E09F9355
:1044C0008F931F930F93E091AF03F091B003099581
:1044D0008CE3809330028DB79EB708968DBF809194
:1044E000EA029091EB029F938F9380910302909147
:1044F00004029F938F938BED95E014C110923002CC
:1045000080912301909124016AE070E00E942F7550
:104510009F938F9380912301909124016AE070E032
:104520000E942F757F936F938AEE95E09F938F93F0
:104530001F930F93FE01099584E1809330022DB7FC
:104540003EB7285F3F4F2DBF80915A0990915B097C
:104550006AE070E00E941B759F938F9380915A09C7
:1045600090915B096AE070E00E941B757F936F93E6
:104570008EEF95E09F938F931F930F93E091AF037E
:10458000F091B003099588E2809330028DB79EB711
:1045900008968DBF80915C0990915D099F938F93E0
:1045A00082E196E09F938F931F930F93E091AF0367
:1045B000F091B00309958CE380933002EDB7FEB71C
:1045C0003696EDBF80915E0990915F099F938F931E
:1045D00082E296E09F938F931F930F93E091AF0336
:1045E000F091B00309952DB73EB72A5F3F4F2DBF1D
:1045F0006AC11092300284E396E09F938F931F93D9
:104600000F93FE01099588E2809330020F900F907E
:104610000F900F9080918A0299279F938F938DE33B
:1046200096E09F938F931F930F93E091AF03F091C8
:10463000B00309958CE3809330028DB79EB7069640
:104640008DBF8091DA07992701979F938F938DE40F
:1046500096E0D7CC109230028DE596E09F938F9331
:104660001F930F93FE01099584E1809330020F9010
:104670000F900F900F90809102016AE00E940F75D9
:10468000892F99279F938F93809102010E940F7524
:1046900099279F938F938DE696E09F938F931F9317
:1046A0000F93E091AF03F091B003099588E28093F6
:1046B00030022DB73EB7285F3F4F2DBF8091B70125
:1046C0006AE00E940F75892F99279F938F9380919D
:1046D000B7010E940F7599279F938F938BE796E000
:1046E0009F938F931F930F93E091AF03F091B003CB
:1046F00009958CE3809330028DB79EB708968DBFE5
:104700008091B8016AE00E940F75892F99279F93C5
:104710008F938091B8010E940F7599279F938F9373
:1047200089E896E09F938F931F930F93E091AF03D7
:10473000F091B0030995EDB7FEB73896EDBFC3C051
:104740005BE8C52E52E0D52E20E030E0E90143E0E1
:10475000F42EC0933002F60181916F0199279F9347
:104760008F9389010F5F1F4F1F930F9387E996E087
:104770009F938F9381E59EE19F938F93E091AF0389
:10478000F091B00309952DB73EB7285F3F4F2DBF7D
:10479000FA9464969801F7FEDCCF95C09FE8C92E85
:1047A00092E0D92EC0E0D0E08E0183E0F82E009395
:1047B0003002F60181916F0199279F938F9325967F
:1047C000DF93CF9384EA96E09F938F9381E59EE1F8
:1047D0009F938F93E091AF03F091B00309952DB7AC
:1047E0003EB7285F3F4F2DBFFA940C5E1F4F2497B2
:1047F000F7FEDDCF68C01092300281EB96E09F9308
:104800008F931F930F93FE01099584E180933002EB
:104810000F900F900F900F908091B3019091B40181
:104820009F938F938FEB96E09F938F931F930F939C
:10483000E091AF03F091B003099588E280933002D4
:104840008DB79EB706968DBF8091B5019091B60148
:104850009F938F938CEC96E09F938F931F930F936E
:10486000E091AF03F091B003099589E480933002A1
:10487000EDB7FEB73696EDBF89ED96E09F938F9327
:104880001F930F93E091AF03F091B00309958091CE
:104890002E020F900F900F900F9083FF14C0109274
:1048A000B6011092B50160E070E08EE090E00E94E9
:1048B0007E2609C080912501281719F421502093E4
:1048C000250110922F0210922E02E8E0CDB7DEB73C
:1048D0000C94A575F999FECF92BD81BDF89A80B56B
:1048E00099270895F999FECF1FBA92BD81BD60BD89
:1048F0000FB6F894FA9AF99A0FBE08954AEA20E0A2
:1049000030E02617370740F4FC018191480F2F5FF4
:104910003F4F26173707C8F3842F99270895EAEAEF
:1049200040E050E04617570778F49C01F999FECF14
:1049300032BD21BDF89A80B5E80F4F5F5F4F2F5F02
:104940003F4F4617570790F38E2F9927089581E020
:104950008093560682E08093550683E08093540648
:1049600084E08093570685E08093580686E0809324
:10497000590687E080935A0688E080935B0689E0B9
:1049800080935C068AE080935D068BE080935E06F0
:104990008CE080935F06089586E6809353063CE0A2
:1049A000EFECF6E0832F11928A95E9F78AE0809385
:1049B0007306109297068BE180936F068EE48093C6
:1049C000940680939506B0E2B09396061092CB06BB
:1049D0008AE68093600682E78093CD0680E5809327
:1049E000CE0684E080937A061092B8061092B5063F
:1049F00078E070936D0626EE20936E0680E4809337
:104A0000700685E080936306FEE1F09361069FE007
:104A100090936406F09362061092660670936706A0
:104A200084E180936806109269061092BB06909309
:104A300065061092C4063093C50610927C0610924B
:104A40007D0610927E0610927F06109299061092B3
:104A50009A0610929B0610929C0690E8909380060E
:104A600042E340938106A2E0A093CC0688E18093C4
:104A700082062093830683E0809388065DE7509347
:104A80008B0650938C0650938D0690938406E5E533
:104A9000E093850666E4609386068CED8093870636
:104AA0008CE38093890610928A069AEA90939D0679
:104AB0008CEC80939F061092A1069093A20698E238
:104AC00090939E069093A0061092A3061092C9069A
:104AD0004093CA0640938E062AE520938F064093A2
:104AE000900636E03093A40684E68093A506809372
:104AF000A6062093A70688E78093A8069093AC06A5
:104B00008BE48093A906E093AA068093AB063093CA
:104B1000AD067093AE064093AF068AE28093B0066E
:104B20001092B1061092B4069CE89093B206A0933E
:104B3000B3061092B6061092B70681E48093780609
:104B4000209379061092B9061092BA0686E98093EE
:104B5000BC065093910684E3809392061092BD06A2
:104B60001092BE061092BF069093C0066093C106D5
:104B70009093C2066093C3061092C606B093770660
:104B80008FE18093C806F093C70608950E94CC2455
:104B90008AE080936A0680E180936B0626E020938A
:104BA0006C069AE59093710688E78093720690935D
:104BB0007406809375062093760680E280937B06C8
:104BC0008CE3809393068BE48093980686E491E6C9
:104BD000A3E7B4E78093CF069093D006A093D106C5
:104BE000B093D20668E870E083E596E00E947E24E8
:104BF0008093DB060895CF93DF930E94CC2488E056
:104C000080936A0630E130936B0626E020936C06B1
:104C100094E69093710688E78093720690937406E9
:104C2000809375062093760630937B0686E4809306
:104C3000930680939806AFECB6E085E0E6E2F1E0FB
:104C4000ED01019009928A95E1F768E870E0CD01E5
:104C50008C5790400E947E248093DB06DF91CF9199
:104C600008950E94CC2426E020936A068AE080936F
:104C70006B0684E080936C0694E69093710688E757
:104C8000809372069093740680937506209376063F
:104C900080E180937B0686E4809393068093980658
:104CA00085E491E6A3E7B9E78093CF069093D00619
:104CB000A093D106B093D20668E870E083E596E051
:104CC0000E947E248093DB060895F999FECF92BD61
:104CD00081BDF89A80B599270895F999FECF1FBA3A
:104CE00092BD81BD60BD0FB6F894FA9AF99A0FBED5
:104CF00008956AE674E20E947E73089542E754E2E2
:104D00000E94B8730895EF92FF920F931F93CF9371
:104D1000C82F8150853008F0C3E089E8C89F800122
:104D200011248BEDE82E8FEFF82EE00EF11E68E8CF
:104D300070E0C7010E948F24682F98012D593F4FC2
:104D40008FB39927AC014270507081FDF9CF32BD0D
:104D500021BDF89A80B5861711F0CA0121C08FB322
:104D600099279C012270307081FDF9CFF2BCE1BC23
:104D7000F89A80B5863611F0C90112C089E8C89F3B
:104D8000C001112485972AE634E249E850E0BC01CD
:104D900083E596E00E9459730E944C6681E090E0A2
:104DA000CF911F910F91FF90EF900895282F86309B
:104DB00010F025E003C0882309F421E020930101CD
:104DC000F999FECF1FBA82E090E092BD81BD20BD6F
:104DD0000FB6F894FA9AF99A0FBE0895CF93C82F98
:104DE00080915306863609F04FC0C63010F0C5E0FA
:104DF00003C0CC2309F448C00E9452728091CE06B1
:104E000082FF07C080917806843618F080E5809391
:104E1000780668E870E083E596E00E947E2480933F
:104E2000DB0689E8C89FC001112422E734E249E883
:104E300050E063E576E085970E94967322E734E2BE
:104E40004CE050E064E576E080E590E00E949673E7
:104E50006CE070E084E596E00E947E24282FF999AA
:104E6000FECF1FBA8CE590E092BD81BD20BD0FB68C
:104E7000F894FA9AF99A0FBE8C2F0E94D6260E94B7
:104E80004C6681E090E002C080E090E0CF91089510
:104E90006DE470E088EE93E00E948F24482F8FB37A
:104EA00099279C012270307081FDF9CF85E394E051
:104EB00092BD81BDF89A80B5841779F48FB3992794
:104EC0009C012270307081FDF9CF88EE93E092BD95
:104ED00081BDF89A80B5813011F0C90108952AE6A4
:104EE00034E24EE450E068EE73E08CED96E00E9410
:104EF000597381E090E008958091DC068130A9F437
:104F00006DE470E08CED96E00E947E24809329078A
:104F100022E734E24EE450E06CED76E088EE93E078
:104F20000E94967381E090E0089580E090E00895FB
:104F3000CF93DF9381E08093DC06ECEDF6E08FE029
:104F4000158616861786108A8150349687FFF8CF0B
:104F500080E48093E9068093EA061092EB06809342
:104F6000EC068093ED0690EC9093EE061092EF061F
:104F70008093F0068093F1061092F2069093F30668
:104F80009093F4068093F5061092F6068093F70648
:104F90009093F806ADEDB6E08CE0ECE2F1E0ED01C7
:104FA000019009928A95E1F76DE470E0CD010197D7
:104FB0000E947E2480932907DF91CF910895F9996B
:104FC000FECF82E090E092BD81BDF89A80B5282F97
:104FD000863078F023E0322FF999FECF1FBA82E0B5
:104FE00090E092BD81BD30BD0FB6F894FA9AF99A5F
:104FF0000FBE20930101822F992708951F93CF930D
:10500000C82F162F863010F0C5E003C0882309F49E
:10501000C1E08C2F99278230910541F083309105B2
:1050200044F4019731F40E94C62505C00E94FB2577
:1050300002C00E9431261123E1F06CE070E080E5AF
:1050400090E00E948F24282FF999FECF8CE590E004
:1050500092BD81BDF89A80B5821759F42AE634E2F0
:105060004CE050E060E570E084E596E00E94597302
:1050700002C00E94A7248C2F0E94EE26CF911F9180
:105080000895DF92EF92FF920F931F93CF93FF2427
:10509000DF2CEF2C81E090E00E946526863611F02F
:1050A00031E0E32E6CE070E080E590E00E948F2418
:1050B000C82FF999FECF8CE590E092BD81BDF89A9A
:1050C00080B58C1711F421E0D22EC1E001E010E090
:1050D000EE2029F48C2F0E9483268823B9F591E0D5
:1050E000F92E1F930F9381EE96E09F938F938CE898
:1050F00091E19F938F93E091AF03F091B0030995F5
:105100002DB73EB72A5F3F4F2DBF0130110521F06B
:105110000230110521F006C00E94C62505C00E947C
:10512000FB2502C00E943126DD2059F02AE634E238
:105130004CE050E060E570E084E596E00E94597331
:1051400002C00E94A7248C2F0E94EE26CF5F0F5F23
:105150001F4FC63008F4BCCFFF2019F083E00E9437
:10516000D6260E94DF27C82F0E9483268C2F9927DE
:105170009F938F9387E097E09F938F930CE811E1C3
:105180001F930F93E091AF03F091B003099581E075
:1051900090E00E9465262DB73EB72A5F3F4F2DBF96
:1051A0008F3F21F00E944827882399F480E297E0FE
:1051B0009F938F931F930F93E091AF03F091B003F0
:1051C00009950E9498270E947C270F900F900F90BE
:1051D0000F90EE2029F066E681E090E00E946D26B7
:1051E0001092520690E0E9EEF6E0CFE0808134962E
:1051F00018160CF49F5FC150C7FFF8CF909352066A
:10520000892F99279F938F938DED96E09F938F938E
:1052100081E497E09F938F931F930F93E091AF03E7
:10522000F091B00309950E94F8048DB79EB70896D7
:105230008DBFCF911F910F91FF90EF90DF90089558
:10524000982F2FB7F8943998389A88B1836088B925
:105250008091B9008C7F8093B9008AE28093B80076
:1052600010923B021092390210923802992381F079
:10527000EEE6F7E08BE01082118212821382148234
:1052800015821682178210868150399687FFF3CFD8
:1052900078942FBF089510923B0284E98093BC005C
:1052A00080E88093BC001092BD001092BA0010926A
:1052B000BB001092B9001092B8001092370280E043
:1052C0000E9420291092BB0085E88093BC00809149
:1052D000350282608093350208951F920F920FB6B7
:1052E0000F9211242F933F936F937F938F939F93EC
:1052F000EF93FF9380913B02282F33278F5F80939A
:105300003B022330310509F41CC1243031055CF423
:105310002130310509F454C0223031050CF099C018
:10532000232B71F02DC32530310509F470C12530D0
:1053300031050CF41EC12630310509F433C220C3F7
:1053400081E08093370209C0809139028C3090F45B
:10535000809139028F5F8093390280913902E82F62
:10536000FF27EE0FFF1FEE0FFF1FE452F94F858559
:10537000181654F7809139026CE00E940F759093D3
:105380003902809141028F5F8093410290913B01ED
:10539000981770F410924102109234021092330266
:1053A00085E080933B0280913802880F8D5A04C0BB
:1053B00080913902880F8E5A8093BB0085E824C102
:1053C000809139029927FC0123E0EE0FFF1F2A95F7
:1053D000E1F7E80FF91FE259F84F81818093BB0094
:1053E00085E88093BC00809139029927FC01EE0F7B
:1053F000FF1FEE0FFF1FEE0FFF1FE80FF91FE2590F
:10540000F84F808180FF9BC0809139029927FC0171
:10541000EE0FFF1FEE0FFF1FEE0FFF1FE80FF91F2C
:10542000E259F84F8281882329F080915206873013
:1054300008F4BCC28091330290913402892B09F0A8
:10544000B5C28091310290913202892B09F0AEC22F
:1054500076C08091390221E030E002C0220F331F74
:105460008A95E2F780913102909132022823392304
:10547000232B81F0809139029927FC0173E0EE0F14
:10548000FF1F7A95E1F7E80FF91FE259F84F80E125
:1054900084830EC0809139029927FC0163E0EE0FEE
:1054A000FF1F6A95E1F7E80FF91FE259F84F1482E0
:1054B000809139029927FC01EE0FFF1FEE0FFF1FAD
:1054C000EE0FFF1FE80FF91FE259F84F8481282FD4
:1054D0003327220F331F220F331F220F331F8091D8
:1054E00039029927FC0133E0EE0FFF1F3A95E1F7EF
:1054F000E80FF91FE259F84F82818770822B809361
:10550000BB0085E88093BC002091390281E090E0E7
:1055100002C0880F991F2A95E2F72091330230913B
:10552000340282239323892B51F086E697E09093EF
:105530003F0280933E0288E08093400237C284E0BD
:105540001CC2E0913E02F0913F0281918093BB002A
:1055500085E88093BC00F0933F02E0933E02809187
:105560004002815080934002882309F41FC283E0E7
:1055700004C28091B900803379F580913C02882380
:1055800029F4809139028F5F80933C028091390227
:105590009927FC01EE0FFF1FEE0FFF1FEE0FFF1FFD
:1055A000E80FF91FE259F84F838199278F779070A0
:1055B0008F3791058CF4809139029927FC01EE0F09
:1055C000FF1FEE0FFF1FEE0FFF1FE80FF91FE2593D
:1055D000F84F83818F5F838310923B0284E980932D
:1055E000BC008AE090E090933A0180933901809169
:1055F00039028F5F8093390210923B02809135020D
:105600008E7F8093350285EA8093BC00CFC1809164
:10561000B9008034D1F1809138029927FC0173E000
:10562000EE0FFF1F7A95E1F7E80FF91FE259F84FE7
:1056300083818F778383809138028F5F80933802D4
:10564000809138028C30A0F0109238021092320211
:105650001092310280913D028F5F80933D028C3029
:1056600038F010923D02809135028D7F8093350293
:105670008091350281608093350210923B0284E96B
:105680008093BC001092370286C08091380299271F
:10569000FC0163E0EE0FFF1F6A95E1F7E80FF91FC9
:1056A000E259F84F8381806883838091380299277B
:1056B000FC01EE0FFF1FEE0FFF1FEE0FFF1FE80FA5
:1056C000F91FE259F84F808180FF41C08091380274
:1056D0009927FC01EE0FFF1FEE0FFF1FEE0FFF1FBC
:1056E000E80FF91FE259F84F848199270097D9F004
:1056F000409709F047C086E697E090933F02809379
:105700003E0288E080934002809138029927FC0194
:1057100033E0EE0FFF1F3A95E1F7E80FF91FE2596A
:10572000F84F14822FC09091380289E0989FC001F1
:1057300011248D58984F90933F0280933E02909190
:10574000380280913D029817D1F483E019C09091FE
:10575000380289E0989FC00111248D58984F90938A
:105760003F0280933E028091350281FD06C09091F8
:10577000380280913D02981711F482E001C081E067
:105780008093400280914002813011F485E801C08D
:1057900085EC8093BC0080913C028093360210928D
:1057A0003C0204C1E0913E02F0913F028091BB00B7
:1057B000808380913E0290913F02019690933F0238
:1057C00080933E028091400281508093400282305B
:1057D00010F085ECCFC0813011F485E8CBC080910A
:1057E000350281FF7BC08091510280FD77C080919E
:1057F00038029927FC0123E0EE0FFF1F2A95E1F7FD
:10580000E80FF91FE259F84F868199278C7F907035
:10581000883F910591F4809138029927FC01EE0FA1
:10582000FF1FEE0FFF1FEE0FFF1FE80FF91FE259DA
:10583000F84F8081816080830FC080913802992762
:10584000FC01EE0FFF1FEE0FFF1FEE0FFF1FE80F13
:10585000F91FE259F84F1082809138029927FC0114
:1058600073E0EE0FFF1F7A95E1F7E80FF91FE25999
:10587000F84F8681883F81F4809138029927FC0196
:1058800063E0EE0FFF1F6A95E1F7E80FF91FE25999
:10589000F84F8081866021C0809138029927FC01F1
:1058A000EE0FFF1FEE0FFF1FEE0FFF1FE80FF91F98
:1058B000E259F84F8681893F89F48091380299270F
:1058C000FC01EE0FFF1FEE0FFF1FEE0FFF1FE80F93
:1058D000F91FE259F84F80818460808380915102E2
:1058E00081FF20C0809138029927FC0133E0EE0F40
:1058F000FF1F3A95E1F7E80FF91FE259F84F86814B
:105900008E3F80F4809138029927FC0123E0EE0F4E
:10591000FF1F2A95E1F7E80FF91FE259F84F80853C
:105920008F5F8087809138028F5F809338028091EB
:1059300038028C30A0F0109238021092320210928D
:10594000310280913D028F5F80933D028C3038F0B0
:1059500010923D02809135028D7F80933502109226
:105960003B0284E98093BC00809135028160809382
:1059700035021AC08093BC0086E080933B0216C0BB
:1059800010923B0284E98093BC00809135028160D3
:10599000809335028AE090E090933A018093390138
:1059A000109239021092380210923702FF91EF9153
:1059B0009F918F917F916F913F912F910F900FBE8B
:1059C0000F901F9018951F93CF93DF93182F8091FE
:1059D0008902882321F48091C401882319F081E091
:1059E00090E09DC01D3008F098C01123C9F0812FB0
:1059F0009927FC0143E0EE0FFF1F4A95E1F7E80FFE
:105A0000F91FE259F84F36978081369688230CF0BB
:105A100084C03997808180FD03C083E090E07FC01F
:105A20008091660799278B709070029719F084E037
:105A300090E075C067E070E086E697E00E947E2403
:105A400090916D07891719F085E090E068C080EDAE
:105A500097E00E946115EC018091350280FD05C040
:105A6000CE010E946A158823B9F3112319F48FEF30
:105A700090E00BC0212F33272150304081E090E08F
:105A800002C0880F991F2A95E2F790933402809301
:105A90003302A1E0B0E0EEE6F7E040E050E06BE07A
:105AA000CD01042E02C0880F991F0A94E2F72091BD
:105AB00033023091340282239323892B11F0118217
:105AC000128261504F5F5F4F399667FFE9CF1092A6
:105AD000390210923B02809135028E7F809335020D
:105AE00085EA8093BC008091350280FD05C0CE011F
:105AF0000E946A158823B9F3809133029091340291
:105B0000892B29F0CE010E946A15882311F3809118
:105B1000330290913402009711F082E090E0DF911F
:105B2000CF911F9108950F931F93CF93DF93982FD9
:105B300080918902882321F48091C401882319F07F
:105B400081E090E097C09D30B0F4992319F486E08D
:105B500090E090C0C92FDD27FE0153E0EE0FFF1F3C
:105B60005A95E1F7EC0FFD1FE259F84F3697808107
:105B7000369687FD03C082E090E07CC03997808133
:105B800080FD03C083E090E075C080ED97E00E9447
:105B900061158C018091350280FD05C0C8010E940D
:105BA0006A158823B9F3219721E030E0C90102C0CA
:105BB000880F991FCA95E2F79093320280933102C1
:105BC000D901EEE6F7E040E050E06BE0CD01042EB5
:105BD00002C0880F991F0A94E2F720913102309198
:105BE000320282239323892B11F011821282615099
:105BF0004F5F5F4F399667FFE9CF109238021092DE
:105C0000660710926D0710923B02809135028E7FDD
:105C10008093350285EA8093BC008091350280FD37
:105C200005C0C8010E946A158823B9F3809131022A
:105C300090913202892B29F0C8010E946A158823AD
:105C400011F38091660799278B709070029719F075
:105C500084E090E00FC067E070E086E697E00E9485
:105C60007E2490916D07891719F085E090E002C0BD
:105C700080E090E0DF91CF911F910F910895CF9335
:105C8000DF9380E021E83FEFC1E2D8E0EBEDF7E001
:105C9000DF01853020F411961C921E9202C03183E0
:105CA00020831982188222968F5F12963296833251
:105CB00080F38FE790E090931A088093190881E8A9
:105CC0009FEF909318088093170810921C08109269
:105CD0001B081092F7021092F6021092F90210922D
:105CE000F8021092FB021092FA02DF91CF91089510
:105CF0001F920F920FB60F9211240F931F932F93A1
:105D00003F934F935F936F937F938F939F93AF9343
:105D1000BF93CF93DF93EF93FF9340918600509111
:105D200087008091430290914402481B590B809157
:105D30008600909187009093440280934302CA01A9
:105D40008D549440A0914502B0914602835F9A41E0
:105D500058F4809145028093DA07149714F010925A
:105D60003E0181E090E095C0A131B1050CF095C0F5
:105D7000CA018B5F9040845B914008F085C08091A0
:105D80003C0190913D01481B590BE091BD06EE236B
:105D900051F0FF27EE0FFF1FE552F84F80819181F0
:105DA00084369105ECF4FD01EA0FFB1FE552F84F34
:105DB00080819181FA01E81BF90BCF01F7FF03C045
:105DC000909581959F4F06975CF480918A02883C5C
:105DD00020F480918A02865F01C088EC80938A0259
:105DE000FD01EA0FFB1FE552F84F808191819C0174
:105DF000220F331F280F391F240F351F37FF02C012
:105E00002D5F3F4FE901D595C795D595C795CA0137
:105E100001968C179D0714F4219706C041505040FD
:105E2000C417D5070CF4219680918A02833CD8F0E0
:105E30008D010A0F1B1FF801E552F84F80819181F7
:105E40009E01281B390BC90163E070E00E942F7589
:105E5000CB01880F991F860F971F0F5D174FF80111
:105E60009183808307C0AA0FBB1FAF5DB74F119608
:105E70001C921E92E0914502F0914602EE0FFF1F28
:105E8000E552F84FD183C08380914502909146023C
:105E900001969093460280934502FF91EF91DF9126
:105EA000CF91BF91AF919F918F917F916F915F91B2
:105EB0004F913F912F911F910F910F900FBE0F9017
:105EC0001F9018958091E8089091E9089093AF058C
:105ED0008093AE058091EA089091EB089093B1050C
:105EE0008093B0058091BC089091BD0897FD039602
:105EF00095958795959587959093B3058093B20571
:105F00008091CE089091CF0897FD0396959587953F
:105F1000959587959093B5058093B4058091F60289
:105F20009091F7022091090230910A02821B930B93
:105F30009093B7058093B605809184029091850275
:105F4000A0918602B0918702BC01CD012AE030E029
:105F500040E050E00E9464753093B9052093B80585
:105F60008091F3059091F4059093BB058093BA0559
:105F700080918E0190918F019093BF058093BE0513
:105F800080912301909124019093C1058093C005D5
:105F900080918A0299279093C3058093C2058091CE
:105FA0007508909176089093C5058093C4058091FB
:105FB0006F0799279093C7058093C605809178074E
:105FC00099279093C9058093C805809181079927E7
:105FD0009093CB058093CA0580918A079927909367
:105FE000CD058093CC058091DF019091E0019093E5
:105FF000D7058093D60580916E0290916F029093A1
:10600000D9058093D80580915A0990915B099093A6
:10601000DB058093DA0580915E0990915F0990938A
:10602000DD058093DC058091800290918102A09132
:106030008202B0918302BC01CD012AE030E040E051
:1060400050E00E9464753093DF052093DE05809157
:10605000600999279093E9058093E80580915C0396
:1060600090915D039093EB058093EA0580915A032C
:1060700090915B039093ED058093EC058091C803AC
:10608000882321F48091C903882321F08091AD05F4
:10609000816003C08091AD058E7F8093AD0508952A
:1060A000EF92FF921F93CF93DF93182F7B01809184
:1060B0008902882371F580910301893111F42998AF
:1060C00001C0299A11501F3FE9F0F092E701E092D8
:1060D000E601E7018091E6019091E701892B11F437
:1060E000209781F38091EA018823A1F31092EA01BD
:1060F0008091E6019091E701892B09F421970E9494
:106100006872E8CF80910301893111F4299A01C0A6
:106110002998DF91CF911F91FF90EF900895EF9212
:10612000FF920F931F9310927A0080910D0290912D
:106130000E029093800880937F0880910B029091CB
:106140000C029093710880937008809109029091DD
:106150000A029093C4088093C308209105023091ED
:106160000602C901880F991F880F991F820F931F7C
:10617000820F931F9093BD088093BC082091070263
:1061800030910802C901880F991F880F991F820F4B
:10619000931F820F931F9093CF088093CE088FECAC
:1061A00080937A00809194069927AA27BB2744EC14
:1061B000E42E49E0F42E012D112DBC01CD01A801E2
:1061C00097010E94F074DC01CB01809386019093CB
:1061D0008701A0938801B093890180919506992742
:1061E000AA27BB27BC01CD010E94F074DC01CB01C2
:1061F0008093820190938301A0938401B0938501E1
:106200001F910F91FF90EF900895A0E0B0E0EBE0B8
:10621000F1E30C948375682E91E0792EEE24FF242F
:1062200057014701E7011092C803F092F102E09292
:10623000F002F092EF02E092EE02F092EB02E092B6
:10624000EA021092E902F092FB02E092FA02F09266
:10625000F902E092F802F092F702E092F602109250
:106260006801109267011092FE010E948F3084E64F
:1062700090E00E9483150E948F30F092CF05E0924B
:10628000CE05F092D105E092D0058091600680FFA6
:1062900014C08091190190911A01875B934058F4C2
:1062A0008091190190911A018E5E924020F08091A8
:1062B000FE01882311F00E94C41900911901109168
:1062C0001A0187B5865F87BD87B5809588BD8FE148
:1062D000C82E8AE090E00E94831580910902909177
:1062E0000A02E80EF91E80910D0290910E02A80E8E
:1062F000B91E80910B0290910C02880E991E80911C
:10630000F3059091F405C80FD91FCA94C7FEE1CFD9
:106310008091190190911A01825F934080F48091DD
:10632000190190911A01459750F0809119019091AF
:106330001A01081B190B109314010093130187B560
:106340008A5087BD87B5809588BD9501205F3F4FF6
:1063500036952795369527953093FB022093FA02C0
:10636000C401409696958795969587959093F902E6
:106370008093F80240E150E0E40EF51EA5E0F694AB
:10638000E794AA95E1F7F092F702E092F602C40FC3
:10639000D51FF5E0D695C795FA95E1F7D093EB02B6
:1063A000C093EA029093F5028093F4023093F302D3
:1063B0002093F20252E06516C9F58091BC089091D5
:1063C000BD0897FF03C0909581959F4F6CE070E0EA
:1063D0000E942F759B017093F1026093F0028091EF
:1063E000CE089091CF0897FF03C0909581959F4F5D
:1063F0006CE070E00E942F757093EF026093EE02E4
:10640000B90184E090E00E947E266091EE027091D6
:10641000EF0286E090E00E947E266091EA02709191
:10642000EB0288E090E00E947E264FC084E090E07E
:106430000E9479269093F1028093F00286E090E02A
:106440000E9479269C019093EF028093EE02809146
:10645000F0029091F1028150984018F42150384098
:10646000A0F182E697E09F938F938CE891E19F9350
:106470008F93E091AF03F091B00309958091BC0830
:106480009091BD0897FF03C0909581959F4F6CE058
:1064900070E00E942F757093F1026093F00280917A
:1064A000CE089091CF0897FF03C0909581959F4F9C
:1064B0006CE070E00E942F757093EF026093EE0223
:1064C00077240F900F900F900F9012BC11BC109278
:1064D000800810927F081092710810927008109234
:1064E000C4081092C30888EC90E00E948315809144
:1064F0000502909106029C01220F331F220F331FC9
:10650000280F391F280F391F3093BD082093BC086E
:1065100080910702909108028C01000F111F000F5B
:10652000111F080F191F080F191F1093CF08009390
:10653000CE0880916F06C82EDD24EE24FF24442768
:1065400037FD4095542FC701B6010E94F0744B01EE
:106550005C016093E4027093E5028093E6029093FD
:10656000E7029801442737FD4095542FC701B60133
:106570000E94F074DC01CB018093DC029093DD0279
:10658000A093DE02B093DF028092C4029092C50213
:10659000A092C602B092C7028093BC029093BD0243
:1065A000A093BE02B093BF021092B4021092B50243
:1065B0001092B6021092B70200918E0110918F01D5
:1065C0001093A3020093A20284E690E090938B01C3
:1065D00080938A0182E390E09093E7018093E60143
:1065E000809194069927AA27BB27BC01CD0124ECF2
:1065F00039E040E050E00E94F074DC01CB018856A5
:10660000954CAF4FBF4F8093860190938701A09325
:106610008801B0938901809195069927AA27BB2705
:10662000BC01CD010E94F074DC01CB018856954C71
:10663000AF4FBF4F8093820190938301A093840159
:10664000B09385011092450110924401C801AA2718
:1066500097FDA095BA2F20914001309141014091C2
:10666000420150914301BC01CD010E94F074DC0154
:10667000CB018093CA089093CB08A093CC08B09329
:10668000CD0810929F0210929E020E944C666620D6
:1066900029F0809151028460809351028FEF8093A2
:1066A0004A0910924B0980E280934C0984E680935A
:1066B0008A028091E401882311F0579A17C08091D3
:1066C000CC06992780FF05C082FF03C080EE9EE2C2
:1066D00002C080E091E190930A018093090181E07A
:1066E000809311010E9424160E94241688E090E0F5
:1066F0000E9479269093EB028093EA0212BC11BCAF
:106700008091FA029091FB0280569940815C9B42F5
:1067100028F08091C80381608093C8038091F802BB
:106720009091F90280569940815C9B4228F08091BB
:10673000C80382608093C8038091F6029091F702AB
:106740008C5291408957954028F08091C80384600D
:106750008093C8038091F0029091F1028C52914095
:10676000835C914028F08091C80388608093C803BF
:106770008091EE029091EF028C529140835C9140A7
:1067800028F08091C80380618093C8038091EA0259
:106790009091EB02805092408355914028F0809177
:1067A000C80380628093C8038091C8038111772455
:1067B00086E480937D0180911B0190911C01A09142
:1067C0001D01B0911E018093F5059093F605A093ED
:1067D000F705B093F8051092FD011092FC0110929C
:1067E000FF01109200021092010210920202109218
:1067F000A4021092A5021092A6021092A702109273
:10680000E7051092E6050E948C19872D9927EEE086
:10681000CDB7DEB70C949F75A3E1B0E0E2E1F4E3FD
:106820000C947F758091F6029091F70220910902F5
:1068300030910A02821B930B9093C4088093C30883
:10684000809113029091140297FD07969C0153E0EA
:10685000359527955A95E1F73093800820937F0866
:10686000809111029091120297FD079643E0959551
:1068700087954A95E1F7909371088093700830935B
:106880008C0820938B0890938308809382088091D2
:10689000BC089091BD08AC01440F551F480F591F0B
:1068A0002091050230910602C901880F991F880FB7
:1068B000991F820F931F820F931F480F591F57FF75
:1068C00002C04D5F5F4F559547955595479550933D
:1068D000BD084093BC088091CE089091CF08AC01D0
:1068E000440F551F480F591F20910702309108028D
:1068F000C901880F991F880F991F820F931F820F5C
:10690000931F480F591F57FF02C04D5F5F4F5595AA
:106910004795559547955093CF084093CE082091C1
:10692000050230910602C901880F991F880F991F2F
:10693000820F931F820F931F9C01442737FD4095C0
:10694000542F8091D4029091D502A091D602B0919B
:10695000D702820F931FA41FB51F8093D402909378
:10696000D502A093D602B093D702209107023091AE
:106970000802C901880F991F880F991F820F931F62
:10698000820F931F9C01442737FD4095542F80911F
:10699000D0029091D102A091D202B091D302820F85
:1069A000931FA41FB51F8093D0029093D102A09390
:1069B000D202B093D30280919508909196082091CD
:1069C000050230910602820F931F909396088093E0
:1069D00095088091C6089091C708209107023091D0
:1069E0000802820F931F9093C7088093C608809176
:1069F000EC029091ED0201969093ED028093EC02EF
:106A00008091F3059091F4052091EA023091EB0218
:106A1000821B930B9C01442737FD4095542F809196
:106A2000CC029091CD02A091CE02B091CF02820F04
:106A3000931FA41FB51F8093CC029093CD02A09307
:106A4000CE02B093CF028FEC80937A0010921501A2
:106A50002091BC023091BD024091BE025091BF0214
:106A600029873A874B875C8729543B4641405040F1
:106A70002CF028E43BE641E050E00DC089859A8582
:106A8000AB85BC85885B9449AE4FBF4F4CF428EB77
:106A900034E94EEF5FEF2D833E834F83588708C064
:106AA00089859A85AB85BC858D839E83AF83B887A6
:106AB0002091C4023091C5024091C6025091C70294
:106AC0002D873E874F87588B29543B464140504085
:106AD0002CF028E43BE641E050E00DC08D859E851A
:106AE000AF85B889885B9449AE4FBF4F4CF428EB13
:106AF00034E94EEF5FEF29833A834B835C8308C010
:106B00008D859E85AF85B88989839A83AB83BC8345
:106B1000A091C308B091C408BB8BAA8BFD01CF0123
:106B2000AA2797FDA095BA2FA090B402B090B50205
:106B3000C090B602D090B702A80EB91ECA1EDB1EC6
:106B4000A092B402B092B502C092B602D092B7023F
:106B5000E090CA08F090CB080091CC081091CD08C5
:106B6000E80EF91E0A1F1B1FE092CA08F092CB081C
:106B70000093CC081093CD08F0916D02F98BFF23A0
:106B800009F098C180916C02882309F093C180912B
:106B9000B80886FF8FC18091700890917108AA276C
:106BA00097FDA095BA2FBC01CD0129813A814B8177
:106BB0005C810E94F0749B01AC0197FF04C02150DE
:106BC000384F4F4F5F4F6BE0559547953795279559
:106BD0006A95D1F780916701682E772488249924DB
:106BE000CA01B901A40193010E94F074DC01CB0138
:106BF0008093060390930703A0930803B0930903BF
:106C0000B7FF04C08150904FAF4FBF4F1C012D0103
:106C10003CE055944794379427943A95D1F72092C5
:106C200006033092070340920803509209038091B3
:106C30007F0890918008AA2797FDA095BA2FBC01E4
:106C4000CD012D813E814F8158850E94F07497FFC0
:106C500004C06150784F8F4F9F4F2BE095958795DB
:106C6000779567952A95D1F7A40193010E94F07456
:106C7000DC01CB0180930A0390930B03A0930C03D8
:106C8000B0930D03B7FF04C08150904FAF4FBF4F7B
:106C90009C01AD018CE055954795379527958A95D0
:106CA000D1F720930A0330930B0340930C035093C6
:106CB0000D038091060390910703909368088093D9
:106CC000670880910A0390910B0390936C0880935E
:106CD0006B08221933094409550920930A0330939C
:106CE0000B0340930C0350930D03E20EF31E041F9D
:106CF000151FE092CA08F092CB080093CC081093BD
:106D0000CD08809166018823B1F457FF04C02F5F3E
:106D10003F4F4F4F5F4F5595479537952795A21A8F
:106D2000B30AC40AD50AA092B402B092B502C092C6
:106D3000B602D092B7022A893B8979010027F7FC75
:106D40000095102F80910A0390910B03A0910C03E2
:106D5000B0910D03E80EF91E0A1F1B1FC801B701F1
:106D600029813A814B815C810E94F0749B01AC01C6
:106D700097FF04C02150384F4F4F5F4FBBE05595F0
:106D8000479537952795BA95D1F780916801A82E38
:106D9000BB24CC24DD24CA01B901A60195010E94BF
:106DA000F074DC01CB018093FE029093FF02A0936C
:106DB0000003B0930103B7FF04C08150904FAF4F61
:106DC000BF4F3C014D01ACE0959487947794679454
:106DD000AA95D1F76092FE027092FF0280920003A2
:106DE00090920103C801B7012D813E814F815885E2
:106DF0000E94F07497FF04C06150784F8F4F9F4FEF
:106E0000FBE09595879577956795FA95D1F7A6015B
:106E100095010E94F074DC01CB01809302039093F2
:106E20000303A0930403B0930503B7FF04C081508C
:106E3000904FAF4FBF4FAC01BD01ECE0759567952A
:106E400057954795EA95D1F7409302035093030372
:106E500060930403709305032A893B8937FF03C0BD
:106E6000309521953F4F21343105E4F1D401C30120
:106E700097FE07C0B095A095909581959F4FAF4F15
:106E8000BF4F81389105A105B10584F4DB01CA012A
:106E900077FF07C0B095A095909581959F4FAF4F14
:106EA000BF4F81389105A105B105E4F081E08093E1
:106EB000A00218C010926C0810926B08109268081B
:106EC00010926708109202031092030310920403B9
:106ED000109205031092FE021092FF02109200031E
:106EE000109201038091020390910303A091040387
:106EF000B0910503BC01CD0124E630E040E050E054
:106F00000E946475E090FE02F090FF02E21AF30A1C
:106F1000F0927E08E0927D088091FE029091FF023F
:106F2000A0910003B0910103BC01CD0124E630E043
:106F300040E050E00E946475DA01C901209102032B
:106F4000309103038C01021B130B10937308009301
:106F500072088091400190914101A0914201B0914D
:106F60004301BC01CD0128E631E040E050E00E9441
:106F7000F0742091CA083091CB084091CC08509110
:106F8000CD08261737074807590764F0261B370B2B
:106F9000480B590B2093CA083093CB084093CC0878
:106FA0005093CD082091CA083091CB084091CC086D
:106FB0005091CD0857FF0CC0260F371F481F591F8F
:106FC0002093CA083093CB084093CC085093CD0847
:106FD00060917008709171086E0D7F1D9B014427B0
:106FE00037FD4095542F8091B8029091B902A0913D
:106FF000BA02B091BB02820F931FA41FB51F8093EA
:10700000B8029093B902A093BA02B093BB028091E8
:10701000720290917302681B790BCB01AA2797FD2E
:10702000A095BA2F29853A854B855C85820F931FE1
:10703000A41FB51F8093BC029093BD02A093BE0213
:10704000B093BF02C0908201D0908301E090840190
:10705000F0908501C816D906EA06FB06C4F488EA52
:1070600091E6A0E0B0E08C199D09AE09BF098093BC
:10707000BC029093BD02A093BE02B093BF02809366
:10708000B8029093B902A093BA02B093BB02222730
:107090003327A9012C193D094E095F098091BC02D3
:1070A0009091BD02A091BE02B091BF0282179307DA
:1070B000A407B507B4F4D701C601885A9146A04089
:1070C000B0408093BC029093BD02A093BE02B093E7
:1070D000BF028093B8029093B902A093BA02B09312
:1070E000BB0260917F0870918008600F711F9B0147
:1070F000442737FD4095542F8091C0029091C102E2
:10710000A091C202B091C302820F931FA41FB51FAA
:107110008093C0029093C102A093C202B093C302B5
:107120008091700290917102681B790BCB01AA27A4
:1071300097FDA095BA2F2D853E854F855889820FE2
:10714000931FA41FB51F8093C4029093C502A09300
:10715000C602B093C702E0908601F09087010091CB
:10716000880110918901E816F9060A071B07C4F483
:1071700088EA91E6A0E0B0E08E199F09A00BB10B60
:107180008093C4029093C502A093C602B093C70235
:107190008093C0029093C102A093C202B093C30235
:1071A00022273327A9012E193F09400B510B80914B
:1071B000C4029091C502A091C602B091C702821785
:1071C0009307A407B507B4F4D801C701885A9146BC
:1071D000A040B0408093C4029093C502A093C60221
:1071E000B093C7028093C0029093C102A093C202E1
:1071F000B093C3028091B4029091B502A091B602FF
:10720000B091B7028093C8029093C902A093CA02BA
:10721000B093CB028091C4029091C502A091C602A6
:10722000B091C7028093E4029093E502A093E60236
:10723000B093E7028091BC029091BD02A091BE0282
:10724000B091BF028093DC029093DD02A093DE0236
:10725000B093DF028091C0029091C102A091C2025E
:10726000B091C3028093E0029093E102A093E20206
:10727000B093E3028091B8029091B902A091BA0252
:10728000B091BB028093D8029093D902A093DA0206
:10729000B093DB02809121019091220197FD079626
:1072A00033E0959587953A95E1F790938008809320
:1072B0007F0880911F019091200197FD079623E0A0
:1072C000959587952A95E1F79093710880937008BA
:1072D00080910D0290910E020F9734F488E19CEF9B
:1072E0009093800880937F0880910D0290910E0208
:1072F000079734F480E398EF9093800880937F0899
:1073000080910D0290910E02815D974034F088EEDD
:1073100093E09093800880937F0880910D02909174
:107320000E02805E974034F080ED97E090938008E5
:1073300080937F0880910B0290910C020F9734F498
:1073400088E19CEF909371088093700880910B0204
:1073500090910C02079734F480E398EF90937108B2
:107360008093700880910B0290910C02815D974090
:1073700034F088EE93E090937108809370088091C8
:107380000B0290910C02805E974034F080ED97E004
:10739000909371088093700860917501662309F4D9
:1073A000AEC0409121015091220180910E03909135
:1073B0000F03481B590B509315034093140320915E
:1073C000210130912201280F391F37FF02C02F5FA2
:1073D0003F4F3595279530930F0320930E03413887
:1073E00051051CF080E890E005C040585F4F34F430
:1073F00080E89FEF909315038093140340911F0141
:10740000509120018091100390911103481B590B5A
:10741000509313034093120320911F0130912001D8
:10742000280F391F37FF02C02F5F3F4F3595279533
:107430003093110320931003413851051CF080E86C
:1074400090E005C040585F4F34F480E89FEF909380
:10745000130380931203462F5527809114039091B4
:107460001503849FB001859F700D949F700D1124AA
:107470009B0177FF02C0215F3F4FB4E03595279510
:10748000BA95E1F780917F0890918008820F931F51
:107490009093800880937F0880911203909113034A
:1074A000849F9001859F300D949F300D1124A90178
:1074B00037FF02C0215F3F4FA4E035952795AA957D
:1074C000E1F78091700890917108820F931F90935B
:1074D0007108809370088091210190912201860F9C
:1074E000971F909322018093210180911F01909119
:1074F0002001840F951F9093200180931F0100911C
:10750000820810918308809167089091680810168E
:1075100011065CF59C0197FF04C022273327281B26
:10752000390BC901AA2797FDA095BA2F20916601B2
:10753000332744275527BC01CD010E94F0749B01DD
:10754000AC0197FF04C0215C3F4F4F4F5F4FF6E007
:107550005595479537952795FA95D1F780917D08F0
:1075600090917E08820F931F27C097FF03C09095CC
:1075700081959F4FAA2797FDA095BA2F209166016C
:10758000332744275527BC01CD010E94F0749B018D
:10759000AC0197FF04C0215C3F4F4F4F5F4FE6E0C7
:1075A0005595479537952795EA95D1F780917D08B0
:1075B00090917E08821B930B90937E0880937D08A8
:1075C000E0908B08F0908C0880916B0890916C088B
:1075D0001E141F045CF59C0197FF04C0222733276B
:1075E000281B390BC901AA2797FDA095BA2F209116
:1075F0006601332744275527BC01CD010E94F07452
:107600009B01AC0197FF04C0215C3F4F4F4F5F4F80
:1076100076E055954795379527957A95D1F78091DE
:10762000720890917308820F931F27C097FF03C0C1
:10763000909581959F4FAA2797FDA095BA2F2091ED
:107640006601332744275527BC01CD010E94F07401
:107650009B01AC0197FF04C0215C3F4F4F4F5F4F30
:1076600066E055954795379527956A95D1F78091AE
:10767000720890917308821B930B90937308809308
:1076800072088091B80887FF44C03989332309F014
:1076900040C080916C028823E1F541E0E41641E0AE
:1076A000F4064CF080917F08909180088E0D9F1D0C
:1076B000805091400DC050E0E5165FEFF50664F490
:1076C00080917F08909180088E0D9F1D80509F4F64
:1076D0009093800880937F0881E0013018074CF078
:1076E0008091700890917108800F911F8050914097
:1076F0000CC09FEF0030190764F4809170089091DE
:107700007108800F911F80509F4F90937108809354
:107710007008E2E1CD5E0C949B758091890288230C
:1077200029F5809151028C7F809351028091500203
:107730008F7D80935002ADECB3E0EEE6F7E09BE086
:107740008091C401882309F48C938D9181831282E6
:107750009150399697FFF4CF8091C401882359F056
:107760008091C40181508093C40105C08091510271
:1077700081608093510280913702882319F0109222
:107780003702089580933B02809135028E7F80936B
:10779000350285EA8093BC000895882319F480E0BF
:1077A00090E00895E82FFF27EE0FFF1FE552F84FF6
:1077B0008081918181589F4F8F3F910521F01CF06E
:1077C0008FEF90E004C097FF02C080E090E099271F
:1077D0000895CF93DF93ABE8B2E0C8E5D6E057E079
:1077E0008991E82FFF27EE0FFF1FE552F84F019018
:1077F000F081E02DE158FF4FEF3FF10521F01CF043
:10780000EFEFF0E004C0F7FF02C0E0E0F0E0893104
:1078100011F4EC931BC04C91242F3327E217F3078C
:10782000A9F0CF01821B930B97FD03969595879541
:1078300095958795242F280F2C93822F9927E81749
:10784000F90714F4215001C02F5F2C935150119669
:1078500057FFC6CF80916206883F38F0EFEFF0E027
:10786000E81BF109E557FD4F808180937A018091F3
:107870007A01882329F0843618F084E680937A010F
:1078800080916406883F38F0EFEFF0E0E81BF109E3
:10789000E557FD4F8081809379018091790188239C
:1078A00029F0843618F084E680937901809171067E
:1078B000883F38F0EFEFF0E0E81BF109E557FD4FA6
:1078C000808180937401809174018B3010F48AE080
:1078D00002C08F3F11F48093740180919E06883F0F
:1078E00038F0EFEFF0E0E81BF109E557FD4F80813C
:1078F0008093970880919708863010F485E002C045
:107900008F3F11F4809397088091A006883F38F04C
:10791000EFEFF0E0E81BF109E557FD4F8081809320
:10792000BF088091BF08863010F485E002C08F3F09
:1079300011F48093BF0880918B06873F19F4429918
:1079400005C007C0863F41F4439B03C08091C00639
:1079500016C08091C10613C0883F38F0EFEFF0E009
:10796000E81BF109E557FD4F8081809394088091D1
:107970009408893110F488E102C08F3F11F480939C
:10798000940880918C06873F19F4429905C007C07E
:10799000863F41F4439B03C08091C20616C080918C
:1079A000C30613C0883F38F0EFEFF0E0E81BF109A1
:1079B000E557FD4F808180936D0880916D08893176
:1079C00010F488E102C08F3F11F480936D0880911C
:1079D0008D06883F38F0EFEFF0E0E81BF109E5573E
:1079E000FD4F808180939D0880919D08893110F41E
:1079F00088E102C08F3F11F480939D088091630657
:107A00000E94CD3B8093670280916606883F38F0E4
:107A1000EFEFF0E0E81BF109E557FD4F808180931F
:107A2000780180916806883F38F0EFEFF0E0E81BBE
:107A3000F109E557FD4F80818093760180917006B2
:107A4000883F38F0EFEFF0E0E81BF109E557FD4F14
:107A500080818093770180917206883F38F0EFEF44
:107A6000F0E0E81BF109E557FD4F80818093730139
:107A700080917306883F38F0EFEFF0E0E81BF109E2
:107A8000E557FD4F80818093750180917406883F92
:107A900038F0EFEFF0E0E81BF109E557FD4F80818A
:107AA0008093720180917506883F38F0EFEFF0E027
:107AB000E81BF109E557FD4F8081809371018091AA
:107AC0007B06883F38F0EFEFF0E0E81BF109E5575F
:107AD000FD4F808180936F0180917C06883F38F054
:107AE000EFEFF0E0E81BF109E557FD4F808180934F
:107AF000660280917D06883F38F0EFEFF0E0E81BEA
:107B0000F109E557FD4F80818093650280917E06E3
:107B1000883F38F0EFEFF0E0E81BF109E557FD4F43
:107B200080818093640280917F06883F38F0EFEF78
:107B3000F0E0E81BF109E557FD4F80818093630277
:107B400080919906883F38F0EFEFF0E0E81BF109EB
:107B5000E557FD4F80818093620280919A06883FAD
:107B600038F0EFEFF0E0E81BF109E557FD4F8081B9
:107B70008093610280919B06883F38F0EFEFF0E040
:107B8000E81BF109E557FD4F8081809360028091E9
:107B90009C06883F38F0EFEFF0E0E81BF109E5576D
:107BA000FD4F808180935F0280918006883F38F08E
:107BB000EFEFF0E0E81BF109E557FD4F808180937E
:107BC0006D0180918406883F38F0EFEFF0E0E81B0C
:107BD000F109E557FD4F808180936C01809181060A
:107BE000883F38F0EFEFF0E0E81BF109E557FD4F73
:107BF000808180936B0180918506883F38F0EFEF9C
:107C0000F0E0E81BF109E557FD4F808180936A01A0
:107C100080918E06883F38F0EFEFF0E0E81BF10925
:107C2000E557FD4F80818093690180919106883FDF
:107C300038F0EFEFF0E0E81BF109E557FD4F8081E8
:107C40008093680180919206883F38F0EFEFF0E072
:107C5000E81BF109E557FD4F808180936701809112
:107C60009306883F38F0EFEFF0E0E81BF109E557A5
:107C7000FD4F8081809366018091BC06883F38F07B
:107C8000EFEFF0E0E81BF109E557FD4F80818093AD
:107C90007C08809160068093B8088091CD0680931F
:107CA0009C0880919806883F38F0EFEFF0E0E81BE1
:107CB000F109E557FD4F8081809365018091B506FC
:107CC000883F38F0EFEFF0E0E81BF109E557FD4F92
:107CD00080818093D10880916F01282F33272F5FF7
:107CE0003F4F8CE398E2B9010E942F7570937C019D
:107CF00060937B0180916E068093C00880916D0631
:107D000080938408E091B706EE23D9F181E0809357
:107D10005E02FF27EE0FFF1FE552F84F8081918131
:107D2000805C9F4F14F410925E0280917D0120913F
:107D30005E028217B1F0833088F4222319F08CEDB3
:107D400095E002C088EC90E09093E7018093E60113
:107D500085E08093740220937D0103C0815080935D
:107D60007D01809111099091120997FF0FC08091B8
:107D70005E02882359F08091C80380688093C8030D
:107D800005C0E0935E028AE080937D018091110935
:107D90009091120997FF1DC0809189028823C9F034
:107DA00080915E028823A9F080910B0190910C01D3
:107DB0008F5F9F4F71F488E99AE39093E701809376
:107DC000E60180E094EA90930C0180930B011092FD
:107DD0005E0280915E02882321F0809150028160D2
:107DE00003C0809150028E7F80935002DF91CF912B
:107DF000089580916906882301F560916E02709163
:107E00006F0277FF02C06D5F7F4F7595679575951F
:107E10006795409123015091240180910201282F00
:107E20003327649FC001659F900D749F900D1124AE
:107E3000B9010E941B75CB0101C099279093810164
:107E40008093800180918001909181018734910518
:107E500038F486E490E09093810180938001089546
:107E60008F3A910530F08FEA90E0909381018093F2
:107E700080010895A8E1B0E0E0E4FFE30C947F7591
:107E80000E940C3480915102992784719070892B43
:107E900091F58091CE0682FF27C080916E0290916D
:107EA0006F020097F1F002E088359007D4F49C014E
:107EB00097FF02C02D5F3F4F359527953595279544
:107EC000809178069927289FA001299F500D389FFF
:107ED000500D1124CA0164E670E00E942F75CB0199
:107EE00006C08DE290E003C08091780699279093B8
:107EF0004F0280934E0220914C0230914D0255E783
:107F00002033350759F41092950210929402809113
:107F10008408992790934F0280934E0260919402B7
:107F2000709195027A8369838091840899270A96D3
:107F30006817790714F49A83898380918A028436BA
:107F400008F062C08091500282FD5EC080912A03D9
:107F500090912B03009731F0019790932B0380931E
:107F60002A030BC01092890290935302809352020D
:107F7000809151028D7E80935102289A8091520205
:107F800090915302895E9340E0F1809160098536BB
:107F9000C0F180914E0290914F029A838983809123
:107FA000510280618093510280915406A82FBB2713
:107FB000AA0FBB1FFD01EF5DF74F11821082809168
:107FC0005506282F3327220F331FC9018F5D974F86
:107FD000FC0111821082A552B84F11961C921E927C
:107FE0002552384FD90111961C921E928091570646
:107FF000E82FFF27EE0FFF1FE552F84F1182108286
:1080000051C4109289024EC480918A028D3808F4BE
:108010001FC4809151028F7E809351029091790606
:1080200082E3989FC001112490932B0380932A032D
:10803000E981FA81B9978CF080918902882369F0EF
:108040008091520290915302FFEF8F3F9F0729F0DA
:1080500001969093530280935202209152023091E4
:1080600053022F3F310509F030F51092AC02109207
:10807000AD021092AE021092AF021092A8021092BE
:10808000A9021092AA021092AB021092160310924B
:10809000170310921803109219031092B402109251
:1080A000B5021092B6021092B7028091500280621F
:1080B000809350024DC080915102826080935102A2
:1080C0008091500285FF44C08091F2019091F301AC
:1080D000A091F401B091F50187399105A105B10591
:1080E0008CF48091840290918502A0918602B091D7
:1080F0008702825A9E4FAF4FBF4F24F08091B8083D
:1081000080FD05C0809150028F71809350021092C3
:10811000AC021092AD021092AE021092AF02109219
:10812000A8021092A9021092AA021092AB02109219
:10813000B4021092B5021092B6021092B702295EF4
:10814000334030F088EE93E09093530280935202D4
:1081500080915606E82FFF27EE0FFF1FE552F84FDC
:1081600080819181813591050CF434C1209189027F
:10817000222309F02FC180915706E82FFF27EE0F29
:10818000FF1FE552F84F808191818C3491050CF4EA
:10819000FFC080912C038F5F80932C03893C08F4EF
:1081A00019C120932C031092530210925202309165
:1081B0005406E32FFF27EE0FFF1FE552F84F808193
:1081C000918187349105B4F480915506E82FFF27FB
:1081D000EE0FFF1FE552F84F808191810190F081F1
:1081E000E02DF7FF03C0F095E195FF4FE734F1056F
:1081F0000CF478C041E020915506A22FBB27AA0FAE
:10820000BB1FA552B84F8D919C9111978734910552
:1082100044F0E32FFF27EE0FFF1FE552F84F808158
:1082200091818D919C918734910574F080915406D1
:10823000E82FFF27EE0FFF1FE552F84F8081918155
:10824000873491050CF042E0E22FFF27EE0FFF1F6D
:10825000E552F84F808191818634910574F48091C4
:108260005406E82FFF27EE0FFF1FE552F84F8081DD
:108270009181873491050CF043E0E22FFF27EE0F48
:10828000FF1FE552F84F808191818A5B9F4F74F404
:1082900080915406E82FFF27EE0FFF1FE552F84F9D
:1082A00080819181873491050CF044E0E22FFF2713
:1082B000EE0FFF1FE552F84F808191818A5B9F4F3F
:1082C00074F480915406E82FFF27EE0FFF1FE5524C
:1082D000F84F80819181863491050CF445E0842F1C
:1082E0000E94D62680915506E82FFF27EE0FFF1F2C
:1082F000E552F84F808191810190F081E02DF7FFE8
:1083000003C0F095E195FF4F7E97CCF48091540621
:10831000E82FFF27EE0FFF1FE552F84F8081918174
:108320008A5B9F4F64F481E08093E30310927502AF
:1083300088EE93E09093E7018093E6014BC0809133
:1083400001010E94832680E00E94380580917A0610
:108350000E94EC708091B80880FF10C080911901D4
:1083600090911A01875B934038F4809119019091A4
:108370001A018E5E924010F40E94C41981E00E949E
:1083800005318093750281E08093E401579A19C00A
:1083900080819181855B9F4FDCF480912C038F5FFE
:1083A00080932C03893CB0F02093890220932C0306
:1083B000109253021092520282E00E940531809383
:1083C000750268E770E0809101010E94503002C0A0
:1083D00020932C0380915606E82FFF27EE0FFF1FF6
:1083E000E552F84F808191818C599F4F0CF029C242
:1083F0002091B806E22FFF27EF77F070EE0FFF1FF6
:10840000EF5DF74F80819181069714F084E606C0F6
:10841000808191818B5F9F4F1CF48CE980932F03A7
:1084200080918902E0915706882309F058C1FF27FF
:10843000EE0FFF1FE552F84F808191818C599F4FBD
:108440009CF48091CE0683FD0BC0E22FFF27EE0F38
:10845000FF1FE552F84F80819181855B9F4FDCF0D3
:108460008091B8068823B9F08091CE0683FF34C18D
:108470008091B806E82FFF27EE0FFF1FE552F84F57
:1084800080819181875F9F4F0CF426C180912F03DB
:10849000843609F021C180917502882329F08091EA
:1084A000510288608093510280911B0190911C01C0
:1084B000A0911D01B0911E018093F5059093F605E2
:1084C000A093F705B093F8051092F2011092F30112
:1084D0001092F4011092F50110928402109285021C
:1084E00010928602109287021092FF0110920002F1
:1084F000109201021092020280915406E82FFF2789
:10850000EE0FFF1FE552F84F808191818D599F4FEB
:10851000ACF480915506E82FFF27EE0FFF1FE552C0
:10852000F84F808191810190F081E02DF7FF03C029
:10853000F095E195FF4FE436F10534F48091B806EB
:10854000882311F480932D0380912D038F5F8093F6
:108550002D038E3F08F458C18091C3089091C40840
:1085600097FF03C0909581959F4F8197B4F48091B8
:108570007F089091800897FF03C0909581959F4F49
:1085800045975CF4809170089091710897FF03C043
:10859000909581959F4F459714F010927502109217
:1085A0002D038091C803882309F093C08091750240
:1085B000882309F48EC080916A03882309F089C05A
:1085C00081E090E0909353028093520281E0809387
:1085D000890210921603109217031092180310923A
:1085E00019031092B4021092B5021092B6021092C2
:1085F000B7021092B0021092B1021092B202109221
:10860000B30280916F06E82EFF2400271127809186
:10861000BC089091BD089C01442737FD4095542F1C
:10862000C801B7010E94F074DC01CB018093C40241
:108630009093C502A093C602B093C7028091CE0862
:108640009091CF089C01442737FD4095542FC801D5
:10865000B7010E94F074DC01CB018093BC029093BF
:10866000BD02A093BE02B093BF028091E40290913C
:10867000E502A091E602B091E7028093C0029093D8
:10868000C102A093C202B093C3028091DC02909118
:10869000DD02A091DE02B091DF028093B8029093D8
:1086A000B902A093BA02B093BB021092AC0210922E
:1086B000AD021092AE021092AF021092A802109278
:1086C000A9021092AA021092AB0284E6809374026F
:1086D0009BC08CED95E091C010922D0395C0FF27B3
:1086E000EE0FFF1FE552F84F80819181853691058D
:1086F0009CF08091CE0683FD0BC0E22FFF27EE0F8A
:10870000FF1FE552F84F80819181855B9F4FDCF020
:108710008091B8068823B9F08091CE0683FF72C09D
:108720008091B806E82FFF27EE0FFF1FE552F84FA4
:10873000808191818E5C9F4F0CF064C080912F03EB
:108740008C3909F05FC080915406E82FFF27EE0FA7
:10875000FF1FE552F84F808191818D599F4FACF4F6
:1087600080915506E82FFF27EE0FFF1FE552F84FC7
:10877000808191810190F081E02DF7FF03C0F09599
:10878000E195FF4FE436F1053CF48091B80688236B
:1087900019F480932E0318C01092AC021092AD020F
:1087A0001092AE021092AF021092A8021092A9028B
:1087B0001092AA021092AB0210929B0210929A029F
:1087C000109299021092980280912E038F5F8093ED
:1087D0002E038B3F70F01092890210922E0310929C
:1087E000530210925202809150028F718093500276
:1087F0000BC0843649F48CEA9DE09093E7018093A6
:10880000E60102C010922E0320914C0230914D02DD
:1088100073E0283E370708F045C08091FC01909135
:10882000FD018B569F4F1CF02F5F3F4F05C0211558
:108830003105C1F12150304030934D0220934C025C
:1088400031C010922F0310924D0210924C022AC098
:108850002E5E324038F18091D9089091DA08805923
:10886000914000F58091840290918502A09186024A
:10887000B09187028C5D9540A040B0409CF480E3AD
:1088800095E790934D0280934C0280915202909113
:1088900053028A5E934030F089EE93E09093530246
:1088A0008093520280913E01815080933E018091DD
:1088B0003E018F3F21F08091510284FFDFC30E946F
:1088C000E93BB0906A0680913803909139039C018E
:1088D000220F331F280F391FC0905406AC2DBB2721
:1088E000AA0FBB1FFD01E552F84F4B2D5527808184
:1088F0009181849FB001859F700D949F700D11240C
:10890000260F371F37FF02C02D5F3F4FB901759506
:10891000679575956795AF5DB74F80916B06082F8A
:1089200011278D919C91809FD001819FB00D909FC8
:10893000B00D11246A0F7B1F7093390360933803C5
:1089400080913A0390913B039C01220F331F280F23
:10895000391FD0905506AD2DBB27AA0FBB1FFD01B7
:10896000E552F84F80819181849FF001859FF00D41
:10897000949FF00D11242E0F3F1F37FF02C02D5F73
:108980003F4FA9015595479555954795AF5DB74F11
:108990008D919C91809F7001819FF00C909FF00CB5
:1089A00011244E0D5F1D50933B0340933A03809179
:1089B0005E02882309F448C0CB0177FD0396DC01F1
:1089C000B595A795B595A795CA0157FD0396FC01E6
:1089D000F595E795F595E7958091A001682F7727A4
:1089E00067FD70956A9F90016B9F300D7A9F300DE7
:1089F000112480916C03482F552747FD50954E9FB9
:108A0000C0014F9F900D5E9F900D1124280F391FBC
:108A100037FF02C0295F3F4F03E0359527950A9540
:108A2000E1F730939B0220939A026E9F90016F9F13
:108A3000300D7E9F300D11244A9FC0014B9F900D39
:108A40005A9F900D11243FC08091B606E82FFF2752
:108A5000EA5BFE4F86818093A001908190936C0326
:108A6000A82FBB27A7FDB095A69F9001A79F300D0B
:108A7000B69F300D1124E92FFF27E7FDF095E49F05
:108A8000C001E59F900DF49F900D1124280F391F10
:108A900037FF02C0295F3F4F13E0359527951A95A0
:108AA000E1F730939B0220939A02A49F9001A59F27
:108AB000300DB49F300D1124E69FC001E79F900D4B
:108AC000F69F900D1124281B390B37FF02C0295F38
:108AD0003F4F43E0359527954A95E1F7309399024A
:108AE0002093980280915706E82FFF27EE0FFF1F73
:108AF000E552F84F80819181909581959F4F909399
:108B00009702809396028530910514F0049705C072
:108B10000FEF8C3F900734F4049690939702809364
:108B2000960204C0109297021092960280914C0215
:108B300090914D028150924078F180919A029091EB
:108B40009B0297FD079623E0959587952A95E1F777
:108B500090939B0280939A0280919802909199023F
:108B600097FD079603E0959587950A95E1F7909311
:108B70009902809398021092AC021092AD0210926A
:108B8000AE021092AF021092A8021092A9021092A7
:108B9000AA021092AB0243C080915903882309F4C2
:108BA0003EC0282F332780919A0290919B0297FD17
:108BB000079613E0959587951A95E1F7289FA001F0
:108BC000299F500D389F500D1124CA0157FD0F9653
:108BD000B4E095958795BA95E1F790939B028093C1
:108BE0009A02809198029091990297FD0796A3E0CE
:108BF00095958795AA95E1F7289FB001299F700D5B
:108C0000389F700D1124CB0177FD0F96F4E09595F8
:108C10008795FA95E1F79093990280939802809056
:108C20009A0290909B0280915C0390915D03881A58
:108C3000990A90929B0280929A0200919802109158
:108C4000990280915A0390915B03081B190B1093B2
:108C500099020093980280915606E82FFF27EE0FA5
:108C6000FF1FE552F84FE080F1808FE790E0E80EBB
:108C7000F91EF0929502E092940280917401992776
:108C8000AA2797FDA095BA2FBC01CD010E9464745C
:108C9000DC01CB0120E030E040E251E4BC01CD0139
:108CA0000E94D273DC01CB01BC01CD010E9436745D
:108CB000DC01CB018093C8088091730180939E08EA
:108CC000809172019927AA2797FDA095BA2FBC0120
:108CD000CD010E946474DC01CB0120E030E040E271
:108CE00051E4BC01CD010E94D273DC01CB01BC0177
:108CF000CD010E943674DC01CB018093770880910E
:108D0000710180938D088091EF0380FF59C080919D
:108D1000D108813808F454C08091E803992787FD71
:108D200090952B2D3327829FD001839FB00D929F6A
:108D3000B00D11248A0E9B1E90929B0280929A0283
:108D40008091E903992787FD9095829FF001839F89
:108D5000F00D929FF00D11240E0F1F1F109399021A
:108D6000009398028091EA03282F332727FD30953E
:108D70008091960290919702820F931F9093970291
:108D8000809396028091EC03282F332727FD30959E
:108D9000809165069927289F8001299F100D389F93
:108DA000100D112410934501009344018091EB03B1
:108DB00099278E159F0524F4909395028093940231
:108DC000809194029091950297FF04C010929502B1
:108DD000109294028091B80882FF02C010929E08FF
:108DE00040919A0250919B02CA0157FD03969C0143
:108DF000359527953595279537FF03C030952195F3
:108E00003F4F809156029091570282179307B4F416
:108E1000CA0157FF03C0909581959F4F97FD039618
:108E200095958795959587959093570280935602CF
:108E30008536910544F084E690E001C00197909357
:108E40005702809356024091980250919902CA01AC
:108E500057FD03969C01359527953595279537FF46
:108E600003C0309521953F4F809154029091550257
:108E700082179307B4F4CA0157FF03C090958195F8
:108E80009F4F97FD03969595879595958795909318
:108E90005502809354028536910544F084E690E0B3
:108EA00001C0019790935502809354028091510222
:108EB00084FF08C010925702109256021092550279
:108EC00010925402ED2DFF27EE0FFF1FE552F84FD1
:108ED00040918F06242F33278081918128173907ED
:108EE00044F48091CB0682FF04C081E080936B0242
:108EF00013C0ED2DFF27EE0FFF1FE552F84F842F13
:108F0000992720919006821B910920813181281791
:108F1000390714F410926B0240915506E42FFF2795
:108F2000EE0FFF1FE552F84F50918F06852F9927BE
:108F300022273327281B390B8081918182179307C1
:108F400044F48091CB0683FF04C081E080936A02E1
:108F500016C080916A02882391F0E42FFF27EE0F5C
:108F6000FF1FE552F84F809190069927851B9109C4
:108F7000208131818217930714F410926A02EC2D3C
:108F8000FF27EE0FFF1FE552F84F40918F06242F69
:108F90003327808191812817390744F48091CB06CB
:108FA00080FF04C081E08093680217C0809168024E
:108FB000882399F0EC2DFF27EE0FFF1FE552F84FA5
:108FC000842F992720919006821B9109208131815D
:108FD0002817390714F41092680240915406E42FC0
:108FE000FF27EE0FFF1FE552F84F50918F06852F98
:108FF000992722273327281B390B808191818217DB
:10900000930744F48091CB0681FF04C081E08093F4
:10901000690216C080916902882391F0E42FFF272E
:10902000EE0FFF1FE552F84F809190069927851BA0
:109030009109208131818217930714F410926902FB
:1090400080916B02882319F480916A02811181E07A
:1090500080936C0280916802882321F480916902D8
:10906000882351F081E080936D0210926C0210927F
:109070006B0210926A0202C080936D0280916C02B2
:10908000882321F480916D02882369F080918E06F7
:10909000992729813A818217930714F49A83898347
:1090A00081E08093A0028091500299279C01247056
:1090B000307082FF31C080915C0390915D03909588
:1090C00081959F4F90939B0280939A0280915A03BF
:1090D00090915B03909581959F4F90939902809317
:1090E00098028091800190918101909395028093E4
:1090F000940210929702109296028091B8088B7792
:109100008B668093B80880919C088C7B80939C0828
:1091100088EC809367021EC08091510284FF1AC0C0
:10912000309397022093960230939B0220939A02E9
:1091300030939902209398029AE59093C80888E7A3
:1091400080939E089093770880938D0810926C020C
:1091500010926D028091900890919108A0919208D0
:10916000B09193082091E4023091E5024091E6022B
:109170005091E702820F931FA41FB51F80939008A0
:1091800090939108A0939208B093930880919808C7
:1091900090919908A0919A08B0919B08E090DC0208
:1091A000F090DD020091DE021091DF02EB82FC8282
:1091B0000D831E838E0D9F1DA01FB11F80939808E5
:1091C00090939908A0939A08B0939B088091850882
:1091D00090918608A0918708B0918808E090E002FD
:1091E000F090E1020091E2021091E302EF82F88632
:1091F00009871A878E0D9F1DA01FB11F80938508B8
:1092000090938608A0938708B09388088091780887
:1092100090917908A0917A08B0917B08E090D802EB
:10922000F090D9020091DA021091DB02EB86FC8605
:109230000D871E878E0D9F1DA01FB11F809378087C
:1092400090937908A0937A08B0937B08F0906D0210
:10925000FF86FF2029F480916C02882309F460C006
:109260001092D4021092D5021092D6021092D70218
:109270001092D0021092D1021092D2021092D30218
:1092800010929008109291081092920810929308F0
:10929000109298081092990810929A0810929B08C0
:1092A00010928508109286081092870810928808FC
:1092B000109278081092790810927A0810927B0820
:1092C0008091C4029091C502A091C602B091C702DC
:1092D0008093C0029093C102A093C202B093C302D4
:1092E0008091BC029091BD02A091BE02B091BF02DC
:1092F0008093B8029093B902A093BA02B093BB02D4
:109300001092FB011092FA011092710210927002F9
:1093100010927302109272020F85002309F0D0C1DF
:1093200080916C02882309F0CBC18091F305909164
:10933000F405815092402CF480918902882309F42D
:10934000BFC190904A09A0906F062090BC08309051
:10935000BD084090CE085090CF0819140CF0BBC047
:10936000BB24CC24DD24CA01B901A60195010E94C9
:10937000647579018A018091130990911409281A62
:10938000390AC101AA2797FDA095BA2FE81AF90A50
:109390000A0B1B0B6B817C818D819E81A60195013F
:1093A0000E94647559016A0180911509909116090E
:1093B000481A590AC201AA2797FDA095BA2FA81AE0
:1093C000B90ACA0ADB0A292C332427FC3094432C1F
:1093D000532CC801B701A20191010E94F07497FFBC
:1093E00004C061507E4F8F4F9F4F3B014C0109E0FD
:1093F00095948794779467940A95D1F7C601B5013F
:10940000A20191010E94F07497FF04C061507E4F49
:109410008F4F9F4F5B016C0119E0D594C794B794AF
:10942000A7941A95D1F780915602909157028134F2
:1094300091053CF48091540290915502813491053C
:10944000D4F0D401C30197FE03C00196A11DB11D44
:109450003C014D019594879477946794D601C5019A
:10946000D7FE03C00196A11DB11D5C016D01D5940D
:10947000C794B794A79480914C09282F332727FDD0
:109480003095432F532F261537054805590514F4F9
:1094900039014A01992787FD9095909581959F4FB5
:1094A000AA2797FDA095BA2F681679068A069B060B
:1094B00014F43C014D012A153B054C055D0514F4DF
:1094C00059016A01A816B906CA06DB060CF0D0C01D
:1094D0005C016D01CDC0EA2CFF2400271127CA01D1
:1094E000B901A80197010E94647539014A01C101BF
:1094F000AA2797FDA095BA2F681A790A8A0A9B0AAB
:109500006B817C818D819E81A80197010E94647589
:1095100059016A01C201AA2797FDA095BA2FA81A7E
:10952000B90ACA0ADB0AD401C30197FE03C00F9629
:10953000A11DB11D3C014D01F4E0959487947794F1
:109540006794FA95D1F7D601C501D7FE03C00F96EF
:10955000A11DB11D5C016D01E4E0D594C794B794E1
:10956000A794EA95D1F780915602909157028134E1
:1095700091053CF4809154029091550281349105FB
:10958000A4F0C401B30123E030E040E050E00E94C9
:10959000647539014A01C601B50123E030E040E0BD
:1095A00050E00E94647559016A0180915706E82FC6
:1095B000FF27EE0FFF1FE552F84F80819181019048
:1095C000F081E02DF7FF03C0F095E195FF4F7A970A
:1095D000A4F0C401B30123E030E040E050E00E9479
:1095E000647539014A01C601B50123E030E040E06D
:1095F00050E00E94647559016A0189E180938C01F1
:1096000021E262167104810491042CF070E2672E4D
:10961000712C812C912C30EE63163FEF73063FEFD7
:1096200083063FEF930644F460EE662E6FEF762ECE
:109630006FEF862E6FEF962E41E2A416B104C1049F
:10964000D1042CF050E2A52EB12CC12CD12C50EE1F
:10965000A5165FEFB5065FEFC5065FEFD50644F4CC
:1096600040EEA42E4FEFB42E4FEFC42E4FEFD42E6A
:109670008091C4029091C502A091C602B091C70228
:1096800086199709A809B9098093C4029093C50265
:10969000A093C602B093C7028091BC029091BD0214
:1096A000A091BE02B091BF028A199B09AC09BD0905
:1096B0008093BC029093BD02A093BE02B093BF0200
:1096C0008091FA019091FB018F3F910509F008F418
:1096D000C4C56F85662309F04EC580916C0288234E
:1096E00009F049C58091A002882309F044C5709112
:1096F0009706788B772309F43EC580919008909166
:109700009108A0919208B0919308B7FF04C08150CE
:109710009F4FAF4FBF4FE92EFA2E0B2F112707FD9A
:109720001A95E0929008F092910800939208109395
:1097300093088091980890919908A0919A08B09107
:109740009B08B7FF04C081509F4FAF4FBF4F892F79
:109750009A2FAB2FBB27A7FDBA95898B9A8BAB8B22
:10976000BC8B8093980890939908A0939A08B09323
:109770009B0880916F06A82EBB24CC24DD24209169
:10978000D4023091D5024091D6025091D702C60141
:10979000B5010E94F07497FF04C061507F4F8F4F56
:1097A0009F4F672E782E892E992487FC9A94609279
:1097B000D4027092D5028092D6029092D702209164
:1097C000D0023091D1024091D2025091D302C60111
:1097D000B5010E94F07497FF04C061507F4F8F4F16
:1097E0009F4F272E382E492E552447FC5A942092FD
:1097F000D0023092D1024092D2025092D302809194
:10980000CC029091CD02A091CE02B091CF02B7FFD1
:1098100004C081509F4FAF4FBF4F892F9A2FAB2F5E
:10982000BB27A7FDBA958093CC029093CD02A0935D
:10983000CE02B093CF02D801C70186199709A809B3
:10984000B9098093220390932303A0932403B09338
:10985000250320919606E22EFF2400271127BC0144
:10986000CD01A80197010E94647559016A012093F6
:10987000300330933103409332035093330389898B
:109880009A89AB89BC8982199309A409B509809387
:10989000260390932703A0932803B0932903BC01C8
:1098A000CD01A80197010E94647520933403309381
:1098B00035034093360350933703D601C501D7FED5
:1098C00004C081509F4FAF4FBF4F892F9A2FAB2FAE
:1098D000BB27A7FDBA95909371028093700257FF42
:1098E00004C021503F4F4F4F5F4FBB2757FDBA95E4
:1098F000A52F942F832F90937302809372028091EF
:1099000056029091570281349105DCF48091540203
:109910009091550281349105A4F480915706E82F67
:10992000FF27EE0FFF1FE552F84F808191810190D4
:10993000F081E02DF7FF03C0F095E195FF4F7A9796
:10994000E4F080914A098F3FC1F4809170029091B8
:10995000710297FD0196959587959093710280937A
:109960007002809172029091730297FD0196959515
:1099700087959093730280937202809185089091ED
:109980008608A0918708B0918808B7FF04C081506D
:109990009F4FAF4FBF4F892F9A2FAB2FBB27A7FDEC
:1099A000BA958093850890938608A0938708B09312
:1099B00088088091780890917908A0917A08B091F0
:1099C0007B08B7FF04C081509F4FAF4FBF4F892F17
:1099D0009A2FAB2FBB27A7FDBA9580937808909359
:1099E0007908A0937A08B0937B088091E402909163
:1099F000E502A091E602B091E7022F813885498502
:109A00005A85281B390B4A0B5B0B20931A033093A2
:109A10001B0340931C0350931D038091DC02909123
:109A2000DD02A091DE02B091DF02EB84FC840D85A3
:109A30001E85E81AF90A0A0B1B0BE0921E03F0922E
:109A40001F030093200310932103209322033093DC
:109A500023034093240350932503E0922603F092BE
:109A6000270300932803109329038091C00290914B
:109A7000C102A091C202B091C302821B930BA40B3E
:109A8000B50B8093C0029093C102A093C202B09321
:109A9000C3028091B8029091B902A091BA02B0912C
:109AA000BB028E199F09A00BB10B8093B802909353
:109AB000B902A093BA02B093BB0288898823E1F06F
:109AC00020919E0230919F02213831054CF0809107
:109AD000F6029091F70201969093F7028093F602B6
:109AE00020583F4F4CF48091F6029091F702019775
:109AF0009093F7028093F60210929F0210929E02BA
:109B000081E090E090933D0380933C03E09022033A
:109B1000F09023030091240310912503D801C7017D
:109B200017FF07C088279927DC018E199F09A00B12
:109B3000B10B81509240A040B04034F084E090E0FE
:109B400090933D0380933C038091420390914303A3
:109B5000A0914403B0914503209190083091910861
:109B60004091920850919308821B930BA40BB50B64
:109B7000815E914BAF4FBF4F8F539C49A040B04087
:109B800028F080914B0989310CF4FFC021E0E216E6
:109B900020E1F20620E0020720E012070CF473C077
:109BA00080913E03882309F46AC0D801C70117FFDA
:109BB00007C088279927DC018E199F09A00BB10BDC
:109BC0009C01AD01B7FF04C021503E4F4F4F5F4F86
:109BD000F9E05595479537952795FA95D1F78091F6
:109BE0003C0390913D03820F931F90933D0380931C
:109BF0003C03D801C70117FF03C00796A11DB11D83
:109C0000E3E0B595A79597958795EA95D1F7809369
:109C1000300390933103A0933203B09333038958F8
:109C20009341A040B04064F088E893E1A0E0B0E048
:109C30008093300390933103A0933203B0933303A6
:109C4000209130033091310340913203509133031E
:109C500057FF04C021503F4F4F4F5F4F232F342FEA
:109C6000452F552747FD5A958091700290917102BA
:109C7000820F931F909371028093700206C081E05F
:109C800080933E0302C010923E0340E0E41640EF92
:109C9000F4064FEF04074FEF14070CF073C08091E8
:109CA0003F03882309F46AC0D801C70117FF07C022
:109CB00088279927DC018E199F09A00BB10B9C0105
:109CC000AD01B7FF04C021503E4F4F4F5F4F69E0D9
:109CD00055954795379527956A95D1F780913C031F
:109CE00090913D03820F931F90933D0380933C031B
:109CF000D801C70117FF03C00796A11DB11D23E0BE
:109D0000B595A795979587952A95D1F780933003B8
:109D100090933103A0933203B093330388579C4E42
:109D2000AF4FBF4F64F488E79CEEAFEFBFEF809377
:109D3000300390933103A0933203B0933303209107
:109D4000300330913103409132035091330357FF78
:109D500004C021503F4F4F4F5F4F232F342F452FCB
:109D6000552747FD5A958091700290917102820F9C
:109D7000931F909371028093700211C081E08093D1
:109D80003F030DC010923F030AC010923D03109292
:109D90003C0384E690E090938B0180938A0168896C
:109DA000262F332780913C0390913D0328173907D4
:109DB00024F430933D0320933C0310914B0911236D
:109DC00079F0212F332727FD309580913C03909126
:109DD0003D032817390724F430933D0320933C03B7
:109DE0004091220350912303609124037091250335
:109DF000413851056105710574F08091FA02909126
:109E0000FB0220913C0330913D03820F931F9093FE
:109E1000FB028093FA0240585F4F6F4F7F4F74F4FC
:109E20008091FA029091FB0220913C0330913D0316
:109E3000821B930B9093FB028093FA0281E090E0E7
:109E400090933D0380933C03C0902603D09027035A
:109E5000E0902803F0902903D701C601F7FE07C060
:109E600088279927DC018C199D09AE09BF0981500B
:109E70009240A040B04034F084E090E090933D03E5
:109E800080933C038091460390914703A09148033F
:109E9000B0914903209198083091990840919A080F
:109EA00050919B08821B930BA40BB50B815E914BC9
:109EB000AF4FBF4F8F539C49A040B04018F01931AD
:109EC0000CF4FFC001E0C01600E1D00600E0E0069F
:109ED00000E0F0060CF473C080914003882309F47D
:109EE0006AC0D701C601F7FE07C088279927DC01A1
:109EF0008C199D09AE09BF099C01AD01B7FF04C0D3
:109F000021503E4F4F4F5F4F09E05595479537958C
:109F100027950A95D1F780913C0390913D03820FDC
:109F2000931F90933D0380933C03D701C601F7FE36
:109F300003C00796A11DB11D13E0B595A795979590
:109F400087951A95D1F78093340390933503A093A6
:109F50003603B093370389589341A040B04064F072
:109F600088E893E1A0E0B0E0809334039093350358
:109F7000A0933603B0933703209134033091350317
:109F8000409136035091370357FF04C021503F4F93
:109F90004F4F5F4F232F342F452F552747FD5A959D
:109FA0008091720290917302820F931F90937302BB
:109FB0008093720206C081E08093400302C0109239
:109FC000400320E0C21620EFD2062FEFE2062FEF6B
:109FD000F2060CF073C080914103882309F46AC033
:109FE000D701C601F7FE07C088279927DC018C1925
:109FF0009D09AE09BF099C01AD01B7FF04C0215006
:10A000003E4F4F4F5F4FE9E0559547953795279560
:10A01000EA95D1F780913C0390913D03820F931F05
:10A0200090933D0380933C03D701C601F7FE03C024
:10A030000796A11DB11D73E0B595A79597958795D6
:10A040007A95D1F78093340390933503A093360328
:10A05000B093370388579C4EAF4FBF4F64F488E7E7
:10A060009CEEAFEFBFEF8093340390933503A09342
:10A070003603B09337032091340330913503409178
:10A0800036035091370357FF04C021503F4F4F4FC5
:10A090005F4F232F342F452F552747FD5A95809129
:10A0A000720290917302820F931F909373028093B8
:10A0B000720211C081E0809341030DC010924103F0
:10A0C0000AC010923D0310923C0384E690E0909306
:10A0D0008B0180938A014889242F332780913C0388
:10A0E00090913D032817390724F430933D032093C2
:10A0F0003C0380914B09882379F0282F332727FDD3
:10A10000309580913C0390913D032817390724F442
:10A1100030933D0320933C03409126035091270345
:10A12000609128037091290341385105610571053B
:10A1300074F08091F8029091F90220913C033091E3
:10A140003D03820F931F9093F9028093F8024058C9
:10A150005F4F6F4F7F4FCCF48091F8029091F902DE
:10A1600020913C0330913D03821B930B9093F902A5
:10A170008093F8020AC01092730210927202109239
:10A180007102109270021092A00280919E088823A2
:10A1900041F41092730210927202109271021092A6
:10A1A00070028091900890919108A0919208B091CE
:10A1B00093088093420390934303A0934403B09386
:10A1C00045038091980890919908A0919A08B091C0
:10A1D0009B088093460390934703A0934803B09352
:10A1E00049031092D4021092D5021092D602109216
:10A1F000D7021092D0021092D1021092D202109285
:10A20000D3021092CC021092CD021092CE02109284
:10A21000CF0210929008109291081092920810921A
:10A220009308109298081092990810929A08109228
:10A230009B08109285081092860810928708109249
:10A240008808109278081092790810927A08109273
:10A250007B081092FB011092FA01E0909602F090B8
:10A260009702C701F7FE04C0882799278E199F0916
:10A2700004973CF08091B80884FD03C082E380938A
:10A28000740210916C06A12EBB24CC24DD24B701EE
:10A29000882777FD8095982F9701F7FE04C0222725
:10A2A00033272E193F09442737FD4095542F0E942C
:10A2B000F0749B01AC01C601B5010E94F07497FFD8
:10A2C00004C061507E4F8F4F9F4F59E09595879501
:10A2D000779567955A95D1F79B01812F99278E9D88
:10A2E000D0018F9DB00D9E9DB00D1124CD01B7FD05
:10A2F00003969595879595958795280F391F809199
:10A300004C0290914D028150924010F020E030E0DC
:10A310008091760290917702280F391F442737FDEC
:10A320004095542F2093160330931703409318033E
:10A33000509319038091B4029091B502A091B60296
:10A34000B091B702821B930BA40BB50B8093B402A0
:10A350009093B502A093B602B093B7028155934C87
:10A36000A040B04064F080E593ECA0E0B0E08093C2
:10A37000B4029093B502A093B602B093B702809155
:10A38000B4029091B502A091B602B091B702805B81
:10A390009C43AF4FBF4F64F480EB9CE3AFEFBFEF44
:10A3A0008093B4029093B502A093B602B093B70223
:10A3B00080908E0190908F0197FCFBC08091B8082F
:10A3C00083FFF7C080918D01815080938D01882398
:10A3D00009F0F3C08DE080938D018091E4029091AB
:10A3E000E502A091E602B091E702B7FF04C08150F8
:10A3F0009E4FAF4FBF4F39E0B595A795979587957D
:10A400003A95D1F78C0197FF03C0109501951F4F26
:10A410008091DC029091DD02A091DE02B091DF021A
:10A42000B7FF04C081509E4FAF4FBF4F29E0B59595
:10A43000A795979587952A95D1F79C0197FF03C01B
:10A44000309521953F4F021713070CF48901B8018D
:10A4500017FF02C0695F7F4F3B01B3E075946794BB
:10A46000BA95E1F7A2E0EA2EF12C6E0C7F1CA090C9
:10A47000CA08B090CB08C090CC08D090CD082091ED
:10A480004001309141014091420150914301C60188
:10A49000B5010E94647519012A0130937608209352
:10A4A0007508821A930AC401845E9D4F68E671E0C4
:10A4B0000E942F75AC01445B50402091740222230E
:10A4C00021F03092A3022092A20280918A01909101
:10A4D0008B01009731F0019790938B0180938A0153
:10A4E00012C0093111057CF480919E0290919F0267
:10A4F000840F951F90939F0280939E02222319F050
:10A5000021502093740280918A0190918B01892BB4
:10A51000F9F480918C019927489F8001499F100D83
:10A52000589F100D1124C801B3010E942F75CB0153
:10A53000AA2797FDA095BA2FA80EB91ECA1EDB1E2A
:10A54000A092CA08B092CB08C092CC08D092CD0895
:10A5500080917402882369F58091A2029091A302F0
:10A560002091750830917608821B930B845E9D4F75
:10A5700068E671E00E942F759C01245B3040809159
:10A58000770186959927289FA001299F500D389F14
:10A59000500D11249A0157FF02C0215F3F4FF4E094
:10A5A00035952795FA95E1F7309377022093760257
:10A5B00004C010927702109276028091A002882344
:10A5C00081F01092A8021092A9021092AA02109291
:10A5D000AB021092AC021092AD021092AE02109239
:10A5E000AF0280916D028823F1F480919E08282F9C
:10A5F0003327442755278091E4029091E502A091EA
:10A60000E602B091E702BC01CD010E94F074DC01CA
:10A61000CB01BC01CD0128EF3AE240E050E00E94BE
:10A620006475390102C06624772480916C02882306
:10A63000F1F480919E08282F3327442755278091D5
:10A64000DC029091DD02A091DE02B091DF02BC013C
:10A65000CD010E94F074DC01CB01BC01CD0128EFDB
:10A660003AE240E050E00E946475290102C04424AF
:10A6700055248091720890917308893C91051CF0D3
:10A6800088EC90E005C088539F4F34F488E39FEF37
:10A69000909373088093720880917D0890917E0852
:10A6A000893C91051CF088EC90E005C088539F4FD1
:10A6B00034F488E39FEF90937E0880937D08809127
:10A6C0007F0890918008AA2797FDA095BA2F209126
:10A6D000C808A22EBB24CC24DD24BC01CD01A601D8
:10A6E00095010E94F0749B01AC01809172089091D9
:10A6F0007308AA2797FDA095BA2FE7E0880F991F46
:10A70000AA1FBB1FEA95D1F7280F391F4A1F5B1FED
:10A7100057FF04C0215C3F4F4F4F5F4F76E0559588
:10A720004795379527957A95D1F78301020F131F27
:10A730001093800800937F088091700890917108B1
:10A74000AA2797FDA095BA2FBC01CD01A6019501BE
:10A750000E94F0749B01AC0180917D0890917E086D
:10A76000AA2797FDA095BA2F67E0880F991FAA1F07
:10A77000BB1F6A95D1F7280F391F4A1F5B1F57FF70
:10A7800004C0215C3F4F4F4F5F4FA6E05595479562
:10A7900037952795AA95D1F77201E20EF31EF09234
:10A7A0007108E09270088091C3089091C408880FE6
:10A7B000991FAA2797FDA095BA2F209177083327D4
:10A7C00044275527BC01CD010E94F0745B016C0148
:10A7D00097FF08C08FE390E0A0E0B0E0A80EB91E9C
:10A7E000CA1EDB1EF6E0D594C794B794A794FA95D9
:10A7F000D1F780918D08282F332744275527809142
:10A80000C8029091C902A091CA02B091CB02BC01CA
:10A81000CD010E94F074DC01CB01BC01CD0120EF21
:10A8200035E540E050E00E946475B501620F731F8A
:10A830007093C4086093C3080150104134F080E065
:10A8400090E19093800880937F0880917F08909199
:10A8500080088050904F34F480E090EF909380080F
:10A8600080937F08B1E0EB16B0E1FB0634F080E0A6
:10A8700090E1909371088093700880917008909196
:10A8800071088050904F34F480E090EF90937108FD
:10A89000809370086150704134F080E090E19093B3
:10A8A000C4088093C3088091C3089091C408805065
:10A8B000904F34F480E090EF9093C4088093C308E5
:10A8C0008091510285FD16C0809102019927209147
:10A8D00023013091240169817A81689FA001699FD9
:10A8E000500D789F500D1124CA01B9010E941B75AB
:10A8F0007A83698380914A03815080934A038F3F12
:10A9000009F05EC080914B0390914C03892B41F478
:10A91000809123019091240190934C0380934B03E9
:10A92000809123019091240120914B0330914C039D
:10A930002817390718F42F5F3F4F09C08091230172
:10A94000909124018217930730F4215030403093C6
:10A950004C0320934B0384E680934A038091B80113
:10A96000282F332740914B0350914C034217530734
:10A9700010F48AE00CC080910001280F311D2417CB
:10A98000350738F480914802882319F0815080936C
:10A9900048028091B701282F33274217530710F43C
:10A9A00089E10CC080910001280F311D2417350763
:10A9B00038F480914702882319F081508093470230
:10A9C000809148028823D1F080917A0290917B0295
:10A9D000A0917C02B0917D02B7FD10C08091C506A8
:10A9E0008093790280EE91EBAFEFBFEF80937A0214
:10A9F00090937B02A0937C02B0937D028091E5014D
:10AA0000882311F40E94366189819A81880F991FE9
:10AA1000880F991F9A8389838091B80880FD02C0AE
:10AA20000C94155D80916C02882311F00C94155DD7
:10AA300040916D02442311F00C94155D8091C80380
:10AA400099278F779070009711F00C94155D4C0149
:10AA50002091FC023091FD022115310509F044C01E
:10AA60008091190190911A018959934058F087B546
:10AA7000853F20F48091FE01815011C081E08093D8
:10AA8000580353C08091190190911A0184369105A1
:10AA900030F587B58B30F8F08091FE018F5F8093A1
:10AAA000FE019AE08902900111248091FF05821B2A
:10AAB00087BD87B5809588BD8CE291E09093E701D2
:10AAC0008093E6018EE591E09093FD028093FC0275
:10AAD0000E948C192AC081E08093570326C04093BE
:10AAE00057034093580321C09093FD018093FC01CC
:10AAF0008091840290918502A0918602B091870294
:10AB000074E0880F991FAA1FBB1F7A95D1F7809315
:10AB1000FF0190930002A0930102B0930202215022
:10AB200030403093FD022093FC028091B8082091C0
:10AB3000670281FF25C02233E8F4809190018150A3
:10AB4000809390018F3FE1F51092A10280918402E1
:10AB500090918502A0918602B09187028093800235
:10AB600090938102A0938202B093830281E080934C
:10AB7000900126C0273420F188EC809390011DC0FD
:10AB80008091440190914501820F911D20916506AD
:10AB90003327829FF001839FF00D929FF00D1124C7
:10ABA000CF01AA2797FDA095BA2F8093800290939A
:10ABB0008102A0938202B093830281E08093A1027C
:10ABC0008091E4029091E502A091E602B091E70243
:10ABD000E0904001F0904101009142011091430149
:10ABE000BC01CD01A80197010E94647559016A0159
:10ABF0008091DC029091DD02A091DE02B091DF0233
:10AC0000BC01CD01A80197010E946475B901C5017D
:10AC10000E944B6C90938A0880938908CC9734F0FB
:10AC20008CE390E090938A0880938908809189084A
:10AC300090918A080E94C26A90938A08809389083A
:10AC400080E280933F0110927F0210927E028091F9
:10AC5000A102882309F487C58091510299279C019C
:10AC60002071307084FD7FC5809150028260809396
:10AC7000500270919C08872F992761E0C62ED12C35
:10AC8000C822D92280FD04C08091B80881FD10C07F
:10AC9000E980FA8030934E0320934D0330937F0276
:10ACA00020937E0280915102806C80935102BBC23E
:10ACB0008091510281FF8AC200918001109181012F
:10ACC000C8010F96A0909402B09095028A159B053A
:10ACD00008F07DC080915703882309F078C08091E7
:10ACE000510287FF15C0809151028F7780935102E6
:10ACF0008091F2019091F301A091F401B091F501DE
:10AD00008093800290938102A0938202B093830289
:10AD1000E0907C08EE20F9F0809180029091810211
:10AD2000A0918202B0918302BC01CD0124E630E003
:10AD300040E050E00E9464758E2D9927AA27BB271A
:10AD400082179307A407B50734F4D0927F02C0920C
:10AD50007E028DE337C080914F0390915003459759
:10AD600084F08091F2019091F301A091F401B091EF
:10AD7000F5018093800290938102A0938202B093A8
:10AD80008302809151028064809351029501201BBF
:10AD9000310B2F50304037FF03C0309521953F4F86
:10ADA00030937F0220937E0280914802882349F0ED
:10ADB000C90163E070E00E942F7570937F02609379
:10ADC0007E028BE280933F011092780234C1C80169
:10ADD0000F97A816B906C0F5209158032223A1F5B4
:10ADE0008091510286FF15C0809151028F7B809324
:10ADF00051028091F2019091F301A091F401B09180
:10AE0000F5018093800290938102A0938202B09317
:10AE1000830280915102806880935102C501801B9A
:10AE2000910B0F9697FF03C0909581959F4F90953A
:10AE300081959F4F90937F0280937E028DE2809355
:10AE40003F0120937802F7C08DE380933F0160912A
:10AE50007902662371F120917A0230917B02409150
:10AE60007C0250917D028091800290918102A0919C
:10AE70008202B091830282179307A407B507CCF42E
:10AE800080915102806480935102862F992790937C
:10AE90007F0280937E028AE0809378028EE5809321
:10AEA0003F018091510287FFC6C0809151028F7788
:10AEB00033C0662309F443C020917A0230917B02AB
:10AEC00040917C0250917D0280918002909181029C
:10AED000A0918202B0918302281739074A075B07C5
:10AEE00074F580915102806880935102862F9927D2
:10AEF000909581959F4F90937F0280937E0286EF7D
:10AF00008093780286E780933F018091510286FF0B
:10AF100092C0809151028F7B809351028091F20107
:10AF20009091F301A091F401B091F501809380021A
:10AF300090938102A0938202B09383027CC080919F
:10AF40005102807C09F477C080917802882309F04F
:10AF50004CC08091F2019091F301A091F401B09165
:10AF6000F501885C9040A040B04020918002309173
:10AF70008102409182025091830282179307A407B5
:10AF8000B5076CF08091F2019091F301A091F4016A
:10AF9000B091F501885C9040A040B0401DC0809108
:10AFA000F2019091F301A091F401B091F501885361
:10AFB0009F4FAF4FBF4F281739074A075B07BCF0B9
:10AFC0008091F2019091F301A091F401B091F5010B
:10AFD00088539F4FAF4FBF4F809380029093810261
:10AFE000A0938202B093830202C0109278028091F3
:10AFF00051028F738093510210924E0310924D03B1
:10B0000071FF06C084EF91E09093E7018093E60121
:10B0100080918802882379F480918402909185023E
:10B02000A0918602B0918702C397A105B1051CF0DB
:10B0300081E08093880260914D0370914E0380916E
:10B040007E0290917F02680F791F70934E03609388
:10B050004D03CB0177FF04C088279927861B970BE8
:10B06000855F91400CF49BC040917802442389F1A4
:10B0700080917A0290917B0220918002309181022E
:10B08000821B930B0996439748F480917A02909122
:10B090007B02A0917C02B0917D0212C0242F332745
:10B0A00027FD3095432F532F80918002909181028C
:10B0B000A0918202B0918302820F931FA41FB51F3B
:10B0C0008093800290938102A0938202B0938302C6
:10B0D00024C08091650620918002309181024091C8
:10B0E0008202509183021616170644F463E00E9410
:10B0F0000F75280F311D411D511D07C063E00E94CF
:10B100000F75281B310941095109209380023093A2
:10B110008102409382025093830210924E03109258
:10B120004D03E0908402F090850200918602109118
:10B130008702D801C70180509440A040B0402091C0
:10B1400080023091810240918202509183028217E5
:10B150009307A407B5075CF4D801C70180509C4F42
:10B16000AF4FBF4F281739074A075B0744F080935A
:10B17000800290938102A0938202B0938302809117
:10B180009C0881FF06C084E690E09093E7018093DD
:10B19000E60180917902882311F40E94F93E8091A2
:10B1A000FC029091FD02892BD1F18091F2019091E6
:10B1B000F301A091F401B091F50180938002909386
:10B1C0008102A0938202B093830229C080918402FD
:10B1D00090918502A0918602B0918702805991409A
:10B1E000A040B0408093800290938102A09382029D
:10B1F000B093830280916906882311F0992702C0D9
:10B200008FE790E09093810180938001E980FA803C
:10B21000F0926F02E0926E028EE280933F01E09026
:10B220006E02F0906F028091F2019091F301A09173
:10B23000F401B091F501209180023091810240919A
:10B24000820250918302281739074A075B0724F0CE
:10B2500080919C0880FD99C280914902882309F061
:10B2600094C28091FC029091FD02892B49F0E090FC
:10B270006E02F0906F021092500310924F03E1C0E3
:10B280008091F2019091F301A091F401B091F50148
:10B29000821B930BA40BB50B80931A0390931B0393
:10B2A000A0931C03B0931D03823000E890070FEFBA
:10B2B000A0070FEFB0072CF481E090E8AFEFBFEFED
:10B2C00009C08F5F9F47A040B04064F08FEF9FE7B9
:10B2D000A0E0B0E080931A0390931B03A0931C039B
:10B2E000B0931D0380911A0390911B039093500318
:10B2F00080934F0380917901282F332744275527C6
:10B3000080911A0390911B03A0911C03B0911D031F
:10B31000BC01CD010E94F07497FF04C0615E7F4FB5
:10B320008F4F9F4F55E095958795779567955A95DF
:10B33000D1F760931A0370931B0380931C039093BF
:10B340001D0365302EEF72072FEF82072FEF920754
:10B350002CF484E09EEFAFEFBFEF09C06050744063
:10B360008040904064F080E094E0A0E0B0E0809302
:10B370001A0390931B03A0931C03B0931D038090AA
:10B380001A0390901B032091FC013091FD0137FFBF
:10B3900002C0295F3F4F43E0359527954A95E1F775
:10B3A0004FEF223834071CF421E83FEF05C0203866
:10B3B000310514F020E830E0C901AA2797FDA095D7
:10B3C000BA2F20917A01332744275527BC01CD019C
:10B3D0000E94F07497FF04C06D5F7F4F8F4F9F4FA7
:10B3E00022E095958795779567952A95D1F79B01EA
:10B3F0005FEF613075071CF420E03FEF06C06F3F40
:10B40000710519F014F020E031E080915102807C48
:10B4100049F0C90137FD03969C013595279535956F
:10B4200027950DC080919C0880FF09C0C90137FD98
:10B4300007969C0103E0359527950A95E1F7820E62
:10B44000931E20917801222309F454C06091A40234
:10B450007091A5028091A6029091A70297FF04C067
:10B4600061587F4F8F4F9F4F17E095958795779540
:10B4700067951A95D1F73327442755270E94F07412
:10B4800097FF04C0615E7F4F8F4F9F4FB5E095954A
:10B49000879577956795BA95D1F760931A0370935E
:10B4A0001B0380931C0390931D036138AFEF7A0751
:10B4B000AFEF8A07AFEF9A072CF480E89FEFAFEF6A
:10B4C000BFEF0AC06F3F71058105910569F064F017
:10B4D00080E091E0A0E0B0E080931A0390931B031A
:10B4E000A0931C03B0931D0380911A0390911B033A
:10B4F000880E991E80917601282F332780914E095E
:10B50000992787FD9095289FF001299FF00D389F7E
:10B51000F00D11249F01F7FF02C021583F4F220F69
:10B52000232F221F330BFFEF21383F071CF420E8A5
:10B530003FEF06C02F3F310519F014F020E031E055
:10B54000280D391DC901AA2797FDA095BA2F009192
:10B550006E0210916F029801442737FD4095542FD9
:10B56000BC01CD010E94F07497FF04C061507E4F72
:10B570008F4F9F4FF9E09595879577956795FA9549
:10B58000D1F7E61AF70A80917E0290917F02892B0B
:10B5900009F064C0101611060CF060C020914F0332
:10B5A00030915003C90137FF03C0309521953F4FBB
:10B5B0002D33310540F480919C0290919D028E15AF
:10B5C0009F0574F526C02C533040E5E0369527954D
:10B5D000EA95E1F72031310510F02FE030E040919D
:10B5E0009C0250919D0218161906E4F480E190E047
:10B5F000821B930B489F9001499F300D589F300D3F
:10B60000112474E0369527957A95E1F72E153F05BC
:10B6100020F580917E0190917F01E816F906F4F003
:10B620007C011CC0205F3F4F80917E0190917F0183
:10B63000829FB001839F700D929F700D11249B011A
:10B6400064E0369527956A95E1F74E155F0514F08D
:10B650007A0104C0E216F30608F07901C701AA27AF
:10B6600097FDA095BA2F5DE0880F991FAA1FBB1FF9
:10B670005A95D1F72091890830918A08442737FDDF
:10B680004095542FBC01CD010E94647520931E0388
:10B6900030931F034093200350932103E0901E0337
:10B6A000F0901F0380915103909152039C01220F4F
:10B6B000331F280F391F2E0D3F1D37FF02C02D5F8E
:10B6C0003F4FA9015595479555954795509352037E
:10B6D0004093510380916106282F3327220F331F97
:10B6E000220F331F241735076CF48091C008282FD0
:10B6F0003327220F331F220F331F205530404217AC
:10B70000530724F0309352032093510380919C08F7
:10B7100080FF14C08091510390915203A981BA8196
:10B720008A179B0724F0B0935203A0935103E09132
:10B730005103F0915203FA83E98327C029813A81AA
:10B74000201B310B37FF02C02D5F3F4F35952795EA
:10B7500035952795E0905103F0905203E20EF31EC9
:10B76000FA82E98212C00E94F93E09811A8110937F
:10B7700052030093510380915102806C80935102D7
:10B78000809150028D7F80935002809151029927C1
:10B790009C012270307081FF39C1809153039091D8
:10B7A0005403A0915503B09156030097A105B1052C
:10B7B00021F0809188028130B9F480916E029091DD
:10B7C0006F02AA2797FDA095BA2F1EE0880F991F38
:10B7D000AA1FBB1F1A95D1F780935303909354036C
:10B7E000A0935503B093560380918802813019F4D9
:10B7F00082E08093880229813A8179010027F7FC51
:10B800000095102F8091890890918A089C01442707
:10B8100037FD4095542FC801B7010E94F074DC0138
:10B82000CB0180931E0390931F03A0932003B0933A
:10B830002103B7FF04C08150904EAF4FBF4F7C0132
:10B840008D01FDE015950795F794E794FA95D1F7EA
:10B85000E0921E03F0921F03009320031093210334
:10B8600060915202709153023FE0603A730750F5C5
:10B870008091530390915403A0915503B0915603C6
:10B880009C01AD01EAE05695479537952795EA95D5
:10B89000D1F7821B930BA40BB50BA8019701F4E021
:10B8A000220F331F441F551FFA95D1F7820F931FA4
:10B8B000A41FB51F8093530390935403A093550383
:10B8C000B093560360547F4118F5809153039091D3
:10B8D0005403A0915503B09156039C01AD01ECE0D7
:10B8E0005695479537952795EA95D1F7821B930B87
:10B8F000A40BB50BA801970172E0220F331F441F60
:10B90000551F7A95D1F7820F931FA41FB51F41C011
:10B910008091FC019091FD018091FC019091FD01CD
:10B9200097FF03C0909581959F4F84369105CCF584
:10B930008091F2019091F301A091F401B091F50191
:10B940009C018091800290918102281B390B37FF66
:10B9500003C0309521953F4F2F3F310509F00CF57D
:10B960008091530390915403A0915503B0915603D5
:10B970009C01AD016EE056954795379527956A95E0
:10B98000D1F7821B930BA40BB50B8E0D9F1DA01F2F
:10B99000B11F8093530390935403A0935503B09326
:10B9A00056038091530390915403A0915503B09195
:10B9B00056031EE0B695A795979587951A95D1F7EA
:10B9C00090936F0280936E0240916706442399F032
:10B9D00055279C01BA010E942F75C901861B970B40
:10B9E00090939D0280939C02260F371F30937F0116
:10B9F00020937E011FC010929D0210929C028FEF37
:10BA000093E090937F0180937E0114C0109288028E
:10BA10001092530310925403109255031092560340
:10BA200030936F0220936E0205C080915102806CAA
:10BA3000809351028091660381FF37C089819A818A
:10BA400097FD0396959587959595879520914E023C
:10BA500030914F022817390760F480916E0290915F
:10BA60006F02892B31F0220F331F220F331F3A83CD
:10BA700029838091F2019091F301A091F401B0919A
:10BA8000F5018093800290938102A0938202B0938B
:10BA9000830288E99AE39093E7018093E60180E0CE
:10BAA0009EE090930C0180930B0120918408822FDB
:10BAB0009927880F991F880F991F889669817A8125
:10BAC0008617970714F09A8389838091C008992775
:10BAD000880F991F880F991F80559040A981BA81BE
:10BAE0008A179B0714F49A838983809136028823EE
:10BAF00041F4809160098E3F20F080916A03882391
:10BB0000E9F080915202909153020297C097B0F4ED
:10BB1000E981FA811E161F068CF481E090E0909373
:10BB2000530280935202E22EFF24EE0CFF1CEE0C17
:10BB3000FF1C8701085D1F4F1A8309838091E5016F
:10BB4000882311F40E94366129813A813093BD0522
:10BB50002093BC058091160390911703A0911803C0
:10BB6000B091190342E0880F991FAA1FBB1F4A9585
:10BB7000D1F70091C3081091C408081B190B213A92
:10BB800031058CF0C90137FD019695958795801791
:10BB900091070CF48C01909581959F4F0817190718
:10BBA0006CF48C010BC00135110514F000E510E0B8
:10BBB0003FEF003B130714F400EB1FEF8091C00828
:10BBC000282F3327220F331F220F331FC90149812A
:10BBD0005A81841B950B801791070CF48C016981A5
:10BBE0007A81621B730B061717070CF48B01809187
:10BBF0007F089091800860919A0270919B02861B49
:10BC0000970B90938F0880938E08D0909E08209178
:10BC1000AC023091AD024091AE025091AF02DD20F6
:10BC200041F0661A770AC301AA2797FDA095BA2F9B
:10BC300004C0AA2797FDA095BA2F280F391F4A1FC5
:10BC40005B1F2093AC023093AD024093AE02509341
:10BC5000AF028091AC029091AD02A091AE02B09182
:10BC6000AF0281509A4FA040B04064F080E09AEF5C
:10BC7000A0E0B0E08093AC029093AD02A093AE023E
:10BC8000B093AF028091AC029091AD02A091AE0250
:10BC9000B091AF0280509640AF4FBF4F64F480E048
:10BCA00096E0AFEFBFEF8093AC029093AD02A0930C
:10BCB000AE02B093AF02C090760620918E0830910C
:10BCC0008F08F8E0FC1598F08C2D9927829F700161
:10BCD000839FF00C929FF00C1124C701F7FC07968C
:10BCE0007C01B3E0F594E794BA95E1F712C08C2D8E
:10BCF00086959927829FA001839F500D929F500D9A
:10BD00001124CA0157FD03967C01F594E794F5943C
:10BD1000E794A0907B01B0907C019501442737FD0A
:10BD20004095542F8091AC029091AD02A091AE024B
:10BD3000B091AF02BC01CD010E946475E20EF31E0A
:10BD400090906501692D772788279927980117FF1B
:10BD500004C022273327201B310B37FF02C02F5F7F
:10BD60003F4F35952795A981BA812A0F3B1F44275C
:10BD700037FD4095542F0E94F07497FF04C0615C1A
:10BD80007F4F8F4F9F4FE6E0959587957795679505
:10BD9000EA95D1F79B016E157F050CF47B01309578
:10BDA00021953F4FE216F3060CF47901809170085B
:10BDB000909171086091980270919902861B970B7F
:10BDC00090936F0880936E082091A8023091A90289
:10BDD0004091AA025091AB02DD2041F0461A570A69
:10BDE000C201AA2797FDA095BA2F04C0AA2797FDE4
:10BDF000A095BA2F280F391F4A1F5B1F2093A80256
:10BE00003093A9024093AA025093AB028091A802FA
:10BE10009091A902A091AA02B091AB0281509A4FD1
:10BE2000A040B04064F080E09AEFA0E0B0E08093E2
:10BE3000A8029093A902A093AA02B093AB028091AA
:10BE4000A8029091A902A091AA02B091AB028050E1
:10BE50009640AF4FBF4F64F480E096E0AFEFBFEF86
:10BE60008093A8029093A902A093AA02B093AB0278
:10BE700020916E0830916F0848E04C1598F08C2D99
:10BE80009927829FB001839F700D929F700D11249E
:10BE9000CB0177FD07966C0163E0D594C7946A9552
:10BEA000E1F712C0C6948C2D9927829FD001839F01
:10BEB000B00D929FB00D1124CD01B7FD03966C011A
:10BEC000D594C794D594C7949501442737FD4095E0
:10BED000542F8091A8029091A902A091AA02B0913A
:10BEE000AB02BC01CD010E946475C20ED31E692D48
:10BEF000772788279927980117FF04C0222733271F
:10BF0000201B310B37FF02C02F5F3F4F3595279520
:10BF1000E981FA812E0F3F1F442737FD4095542FAA
:10BF20000E94F07497FF04C0615C7F4F8F4F9F4F5A
:10BF300036E095958795779567953A95D1F79B016A
:10BF40006C157D050CF46B01309521953F4FC216A1
:10BF5000D3060CF469018091E501882311F40E9455
:10BF6000366180918408282F33273E8B2D8B80915A
:10BF7000C008282E33245090B9062EE6A22E27E0C2
:10BF8000B22E99EE892E96E0992E8BE0482EBFE9CD
:10BF90006B2EB8E07B2ED4012C9112160CF02FC121
:10BFA000203429F4E981FA81F88FEF8B1FC0498191
:10BFB0005A81CA01AA2797FDA095BA2F332727FDDA
:10BFC0003095432F532FBC01CD010E94F07497FF91
:10BFD00004C0615C7F4F8F4F9F4FA6E0959587957A
:10BFE00077956795AA95D1F7788F6F8BF4012181AA
:10BFF000203439F42F89388D2E0D3F1D388F2F8B2B
:10C000002AC0203C39F44F89588D4E195F09588F4A
:10C010004F8B21C0C701AA2797FDA095BA2F3327C0
:10C0200027FD3095432F532FBC01CD010E94F074A2
:10C0300097FF04C0615C7F4F8F4F9F4FF6E095954F
:10C04000879577956795FA95D1F7AF89B88DA60F43
:10C05000B71FB88FAF8BF4012281203439F42F89B8
:10C06000388D2C0D3D1D388F2F8B2AC0203C39F484
:10C070004F89588D4C195D09588F4F8B21C0C601CF
:10C08000AA2797FDA095BA2F332727FD3095432F78
:10C09000532FBC01CD010E94F07497FF04C0615C76
:10C0A0007F4F8F4F9F4FE6E09595879577956795E2
:10C0B000EA95D1F7AF89B88DA60FB71FB88FAF8BB0
:10C0C000F4012381203439F42F89388D200F311F5A
:10C0D000388F2F8B2AC0203C39F44F89588D401B54
:10C0E000510B588F4F8B21C0C801AA2797FDA095EF
:10C0F000BA2F332727FD3095432F532FBC01CD0195
:10C100000E94F07497FF04C0615C7F4F8F4F9F4F78
:10C1100056E095958795779567955A95D1F7AF89AC
:10C12000B88DA60FB71FB88FAF8BF501808181FD49
:10C1300008C0D3018D919C91EF89F88D8E179F07D0
:10C1400074F4D3018D919C91EF89F88D8E0F9F1F10
:10C1500097FD019695958795988F8F8B1EC05520DA
:10C1600049F42F89388D220F331F281B390B388F44
:10C170002F8B13C031E0351580F4252D33274F89DF
:10C18000588D841B950BB9010E942F75CB016F89C7
:10C19000788D680F791F788F6F8B8D899E89880FB6
:10C1A000991F880F991FAF89B88D8A179B0754F480
:10C1B000C101880F991F880F991FEF89F88DE81723
:10C1C000F90714F0988F8F8B8F89988D97FD0396C0
:10C1D0009595879595958795F5018183880F991F8A
:10C1E000880F991F2F89388D281B390BC901880F9B
:10C1F0008283EF89F88DD301ED93FC9303C0F501A1
:10C20000118212824A9422E030E0620E731E44E0F2
:10C2100050E0840E951E69E070E0A60EB71E47FE42
:10C22000BACEE2E1C85E0C949B7584B1806A84B991
:10C230003D9A82E58CBD1DBC459A81E08093D4086F
:10C240008AEA8093E50883E88093E6088AE0809391
:10C25000E7081092E9081092E8081092EB08109293
:10C26000EA0810924D091092090908953091D408F6
:10C27000332309F070C00DB407FE6DC085E08093D4
:10C28000E501459A2EB580916D039927813091057E
:10C2900089F0823091051CF4892B21F03EC0029771
:10C2A000B9F03BC03093080920936E032138A9F5FB
:10C2B00081E008C0253549F480916E03820F809398
:10C2C0006E0382E080936D0328C030936D0325C018
:10C2D00080910809E82FFF27E65DF64F20838F5FE6
:10C2E0008093080990916E038032A0F0291769F4B9
:10C2F00080E2AAE2B9E0EAE0F9E00D9001928A95C5
:10C30000E1F781E08093090902C030930909109296
:10C310006D0303C0920F90936E032091E4082232C4
:10C32000A0F445980000000000000000E091DD0846
:10C33000F091DE08E20FF11D80818EBD809106092B
:10C340009081890F8093060903C081E08093D4080F
:10C350002F5F2093E4080895EF92FF920F931F93AD
:10C3600080916F069927880F991F880F991F7C016C
:10C370000027F7FC0095102F8091E4029091E502D0
:10C38000A091E602B091E702BC01CD01A80197019E
:10C390000E9464753093E9082093E8088091DC02DC
:10C3A0009091DD02A091DE02B091DF02BC01CD01CF
:10C3B000A80197010E9464753093EB082093EA0866
:10C3C0002091CA083091CB084091CC085091CD08FB
:10C3D000DA01C90173E0880F991FAA1FBB1F7A9564
:10C3E000D1F7820F931FA41FB51F820F931FA41FA5
:10C3F000B51F20914001309141014091420150917F
:10C400004301BC01CD010E9464753093F108209373
:10C41000F0088091F6029091F70220910902309184
:10C420000A02821B930B9093F7088093F608E09121
:10C43000EC02F091ED028091950890919608BF0171
:10C440000E942F75CB019B01220F331F220F331F38
:10C45000280F391F280F391F37FF02C02D5F3F4FAC
:10C4600035952795359527953093ED082093EC0861
:10C470008091C6089091C708BF010E942F759B014B
:10C48000220F331F220F331F260F371F260F371F90
:10C4900037FF02C02D5F3F4F35952795359527957E
:10C4A0003093EF082093EE081092ED021092EC0208
:10C4B00010929608109295081092C7081092C6081C
:10C4C0008091E7089927AA27BB27FC013A97E83013
:10C4D000F10508F03DC2E35AFF4F0C94B675809108
:10C4E00066028093FA08809165028093FB08809130
:10C4F00064028093FC08809163028093FD08809120
:10C5000062028093FE08809161028093FF0880910F
:10C5100060028093000980915F02809301098091FD
:10C5200051028093020980915102837F80935102CE
:10C53000809101018093030980912301909124014E
:10C54000809304098091500280930509429900C2AA
:10C5500080915002877F80935002FAC180915A09DE
:10C5600090915B099093FB088093FA0880916F0388
:10C570008093FC08809160098093FD088091A40657
:10C580000E94CD3B8093FE0880913F018093FF087D
:10C5900020916F03822F9927FC0113E0EE0FFF1FFC
:10C5A0001A95E1F7E80FF91FE259F84F808580935B
:10C5B000000980818093010986818093020983812B
:10C5C00080930309878180930409858180930509FD
:10C5D0002F5F20936F03E22FFF27EE0FFF1FEE0F59
:10C5E000FF1FE452F94F858518160CF4B1C12223C0
:10C5F00009F4AEC1822F992701966DE070E00E9488
:10C600002F75AC01282FE82FFF27EE0FFF1FEE0F2D
:10C61000FF1FE452F94F8585181614F0442351F793
:10C6200040936F0395C1809102018093FA08809135
:10C63000A5068093FB088091A6068093FC08809154
:10C64000A7068093FD088091A8068093FE0880913C
:10C65000AC068093FF088091AD068093000980911D
:10C66000AE06809301098091B10680930209809102
:10C67000AF06809303098091B006809304098091EE
:10C68000B2063BC18091A3068093FA081092FB0882
:10C690008091C5068093FC088091BA068093FD08BE
:10C6A000809147028093FE08809191038093FF0858
:10C6B00080918F038093000980918E0380930109FC
:10C6C0001092910310928F0310928E038091A20218
:10C6D0009091A30290930309809302098091C90667
:10C6E000809304098091CA0608C1F8948091560687
:10C6F000E82FFF27EE0FFF1FE552F84F0190F08162
:10C70000E02DE038F1051CF0EFE7F0E006C02FEF78
:10C71000E138F20714F4E1E8FFEFE093FA088091C2
:10C720005706E82FFF27EE0FFF1FE552F84F019045
:10C73000F081E02DE038F1051CF0EFE7F0E006C0F5
:10C740007FEFE138F70714F4E1E8FFEFE093FB082F
:10C7500080915506E82FFF27EE0FFF1FE552F84F97
:10C760000190F081E02DE038F1051CF0EFE7F0E0FA
:10C7700006C08FEFE138F80714F4E1E8FFEFE0932B
:10C78000FC0880915406E82FFF27EE0FFF1FE552AB
:10C79000F84F0190F081E02DE038F1051CF0EFE753
:10C7A000F0E006C02FEFE138F20714F4E1E8FFEF04
:10C7B0007894E093FD0880918B028093FE0880912D
:10C7C0008C028093FF0880918D02809300098091F4
:10C7D0008E028093010980918F02809302098091DB
:10C7E00090028093030980919102809304098091C3
:10C7F000920283C08091E303853018F01092E30326
:10C8000085E08093FA088091B3068093FB088091BD
:10C81000840290918502A0918602B0918702BC01AA
:10C82000CD0125E030E040E050E00E946475309397
:10C83000FD082093FC088091800290918102A091D4
:10C840008202B0918302BC01CD0125E030E040E0DE
:10C8500050E00E9464753093FF082093FE08809199
:10C86000A906809300098091AA068093010980910E
:10C87000AB068093020980918A028093030980911C
:10C880007003809304098091BC059091BD0597FDCC
:10C89000039695958795959587952FC082E080930F
:10C8A000FA0886E08093FB081092FC0884E48093E9
:10C8B000FD08809103018093FE088091C803809356
:10C8C000FF089091C903909300098F778093C80364
:10C8D00090719093C9038091C6068093010980915D
:10C8E000B8088093020980919C0880930309809185
:10C8F000B606809304098091CE068093050928C06E
:10C9000080915E0990915F099093FB088093FA08EB
:10C9100080916D018093FC0880916C018093FD08EB
:10C920008091E6058093FE088091AE018093FF0818
:10C930008091B4068093000980917C08809301095E
:10C940008091B3019091B4019093030980930209FF
:10C9500080910909882309F465C160910A098091D1
:10C96000A101681719F08AEF80939F016093A101DC
:10C9700081E080938D0140910B0950910C09CA010F
:10C9800081509E4F8F5F9340B0F420910D093091FC
:10C990000E09C90181509E4F8F5F934060F48091D2
:10C9A000600685FF08C050935D0340935C0330939D
:10C9B0005B0320935A03809111099091120921E0A1
:10C9C0008936920724F490938F0180938E012091F1
:10C9D0001B0930911C098091E6019091E7018217B3
:10C9E000930740F48091B901882321F43093E70143
:10C9F0002093E601862F99278836910509F468C0AF
:10CA00008936910524F48736910551F013C1893692
:10CA1000910509F492C08B36910509F4DEC00AC174
:10CA200080911D0980934A0980911E0980934C09C9
:10CA300080911F0980934B098091200980938C017C
:10CA40008091210980934E09809122098093A00151
:10CA50008091230980936C0380912409809359036A
:10CA600080915E028823F9F02091250930912609F2
:10CA700037FD19C03093A3022093A20290918A0639
:10CA8000992389F08FE0989FC0011124281B390B4E
:10CA9000C90188599E4F68E671E00E942F759093F6
:10CAA000A3028093A20220916403309165038091D8
:10CAB000270990912809280F391F37FF02C02F5FDF
:10CAC0003F4F359527953093650320936403B2C09B
:10CAD00080911D098093DF0880911E098093E008F2
:10CAE00080911F098093E108809120098093E208DA
:10CAF000809121098093E3088091AC0590912209EF
:10CB0000892B8093AC059091AD059370809123099A
:10CB10008C70982B9093AD058091240980936A03C3
:10CB200080912509809391018091260980934D0978
:10CB300080912709809366037DC080911D098093B1
:10CB4000D50880911E098093D60880911F09809393
:10CB5000D708809120098093D8088091210990916D
:10CB600022099093DA088093D90880912309909143
:10CB700024099093DC088093DB088091250999278C
:10CB800087FD90959093160880931508809126094B
:10CB90008093790280912709909128099C0144276C
:10CBA00037FD4095542FDA01C90163E0880F991FC2
:10CBB000AA1FBB1F6A95D1F7820F931FA41FB51F31
:10CBC000820F931FA41FB51F80937A0290937B025C
:10CBD000A0937C02B0937D022DC080911D098093AB
:10CBE000690380911E098093680380911F098093D7
:10CBF0006703809121098093940380912209809397
:10CC00009303809125098093920380912609809354
:10CC1000900380912709909128099093C2088093EE
:10CC2000C10808C010925D0310925C0310925B0370
:10CC300010925A031F910F91FF90EF9008958091E9
:10CC4000D408882319F480E090E00895459885EE93
:10CC500098E09093DE088093DD0890916B03E92FB4
:10CC6000FF27EE56FE4F9F5F90936B03808180936A
:10CC7000E7089D3010F010926B031092D4080E94C8
:10CC8000AC6181E08093E4088091E5088093060917
:10CC90008EBD81E090E0089587B18C6087B942989D
:10CCA00043981092720380E88093A301109271035D
:10CCB0008093A201089580911508909116088158DB
:10CCC0009F4F39F0809115089091160881588093F4
:10CCD0007C03809177038150809377038F3F09F025
:10CCE00052C180919D068093780380919F06809326
:10CCF000790389E0809377038091510299278073AB
:10CD00009070892B21F48091C90380FF1DC0809110
:10CD1000A106882351F080917A03882319F484E0D6
:10CD20008093720381E080937A038091A206882326
:10CD300079F080917B03882319F484E08093710358
:10CD400081E080937B0304C010927A0310927B03EE
:10CD500080917A03882309F082C08091CB06282F26
:10CD6000332724FF07C080918902882319F425FD09
:10CD70008FC090C090919E06983F48F08091970890
:10CD80008D3D28F08091780388236CF00AC0983F8D
:10CD900078F080919708853059F48091780387FF67
:10CDA00002C0429A01C0429881E08093A30154C01E
:10CDB000809172038150809372038F3F09F06BC0A2
:10CDC0008091CE0685FF2FC090917C03892F869598
:10CDD00080937203992361F4909370038091780398
:10CDE00087FF02C0429A01C042981092A30153C02B
:10CDF00081E0809370038091A30190917803882350
:10CE000049F480937C0380E48093A30199230CF47C
:10CE10003FC040C0982311F0429A01C042988695C5
:10CE20008093A30138C08091970886958093720300
:10CE30008091A301813021F410927C0380E401C031
:10CE400086958093A3018091A30190917803892313
:10CE500011F0429A01C04298109270031CC0809158
:10CE600072038150809372038F3FA9F489E080930D
:10CE700072038091A301813011F480E801C086958E
:10CE80008093A3018091A3019091A106892311F0C1
:10CE9000429A01C0429880917B03882309F043C0E5
:10CEA0009091CB0697FF07C080918902882319F4DF
:10CEB00096FD52C053C09091A006983F48F08091D3
:10CEC000BF088D3D28F08091790388236CF00AC05B
:10CED000983F78F08091BF08853059F480917903AC
:10CEE00087FF02C0439A01C0439881E08093A2016A
:10CEF00036C0809171038150809371038F3F79F523
:10CF00008091BF088695809371038091A201813042
:10CF100011F480E401C086958093A2018091A20162
:10CF20009091790317C080917103815080937103B0
:10CF30008F3FA9F489E0809371038091A201813031
:10CF400011F480E801C086958093A2018091A2012E
:10CF50009091A206892311F0439A01C04398429B05
:10CF600005C080915002886080935002439B06C0A8
:10CF70008091500280618093500208958091500208
:10CF80008F7E8093500208950F931F93CF93DF936A
:10CF9000482FEB0180918A02E42FFF27843BD8F0D1
:10CFA0008F010E0F1F1FF801E552F84F808191810C
:10CFB0009B01281B390BC90163E070E00E942F75AB
:10CFC000CB01880F991F860F971F0F5D174FF80130
:10CFD0009183808306C0EE0FFF1FEF5DF74F118234
:10CFE0001082E42FFF27EE0FFF1FE552F84FD18389
:10CFF000C083DF91CF911F910F9108954FB724E126
:10D0000030E0F8948091C9008F778093C9008091B7
:10D01000C9008F7B8093C9008091C9008F7D809368
:10D02000C900832F99278093CD002093CC00809155
:10D03000C80082608093C80080E18093C90080911D
:10D04000CA008F778093CA008091CA008F7B80933B
:10D05000CA008091CA008F7D8093CA008091CA0067
:10D060008F7E8093CA008091CA00877F8093CA0018
:10D070008091C9008B7F8093C9008091CA00846031
:10D080008093CA008091CA0082608093CA00809118
:10D09000C80087FF03C08091CE00F9CF8091C900FE
:10D0A00080688093C9004FBF0895EF92FF920F935D
:10D0B0001F93CF93DF93482F00E010E08091A401ED
:10D0C000813061F41092A40184E480937F03109274
:10D0D0008103109280031092820303C280917F0328
:10D0E000882319F421E030E001C098019091800379
:10D0F000992371F4232B11F081E010C084E4809314
:10D100007F03909381039093800390938203D2C115
:10D11000913069F4232B09F0C3C182E0809380032E
:10D12000809181038F5F8093810383E0C1C192303E
:10D13000D1F4232B09F0B4C183E080937F034093A3
:10D14000820390918103923039F41092830347FF58
:10D1500003C081E08093830383E0809380039F5F1B
:10D1600090938103A7C1933009F09AC1232B09F052
:10D1700097C190937F0382E0809380038091810325
:10D180008F5F8093810320918203822F9927782FCC
:10D190006627842F9927682B792B80917A06813016
:10D1A00051F47370CB018050924063E070E00E94B4
:10D1B0002F75EB0119C0823069F47770CB01805074
:10D1C000944066E070E00E942F75EB01269526954D
:10D1D00026950CC0EB01D370C856D140CE01D7FDC7
:10D1E0000196EC01D595C79526952695022F112716
:10D1F0000F7010700F5F1F4F0D30110508F049C1FF
:10D200000230110519F404E010E005C004301105E6
:10D2100011F402E010E0D801A00FB11FFD01E552AA
:10D22000F84F808191819E01281B390BC90137FF7E
:10D2300003C0909581959F4F069704F5E091BD0638
:10D24000EE2351F0FF27EE0FFF1FE552F84F8081CC
:10D2500091818436910594F480918A02883C30F45F
:10D2600080918A02865F80938A0208C088EC80934E
:10D270008A0280916F008F7D80936F00A552B84F16
:10D280008D919C91BC01660F771F680F791F6C0F01
:10D290007D1F77FF02C06D5F7F4F7B01F594E794A0
:10D2A000F594E794CE0101968E159F0524F4089419
:10D2B000E108F10808C0CE010197E816F9061CF450
:10D2C0000894E11CF11C0630110509F0CEC0C536EA
:10D2D000D1050CF4A5C090917E03E92FFF27E15BF7
:10D2E000F64FE081ED3729F480917D03809580939E
:10D2F0007D03963061F480917D03882311F0E3383B
:10D30000B9F0882309F088C0ED3791F085C09930D5
:10D3100009F082C080917D03882329F48091580907
:10D32000833831F079C0809158098D3709F074C085
:10D33000809150098D3739F480915109833899F4DF
:10D3400063E87FEF0DC0833871F480915109833811
:10D3500019F460E070E004C08D3729F46DE770E0E7
:10D3600085E00E94C46780915209992787FD9095B6
:10D37000BC0186E00E94C46780915309992787FD0C
:10D380009095BC018BE00E94C46780915409992755
:10D3900087FD9095BC018CE00E94C46780917E035C
:10D3A0008930D1F5809156098D3749F48091EB078A
:10D3B0009091EC070596BC0188E00E94C4678091BB
:10D3C00057098D3749F48091EB079091EC07059749
:10D3D000BC0188E00E94C4678091EB079091EC0744
:10D3E00083589F4F1CF483E89FEF09C08091EB079F
:10D3F0009091EC078E37910534F08DE790E0909393
:10D40000EC078093EB0780915509992787FD90954C
:10D41000BC018AE00E94C46710927E0310927D03D3
:10D42000CA30D1055CF480917E038F5F80937E03C8
:10D43000E82FFF27E15BF64F83E8808380917E032E
:10D440008A3011F410927E038FEFCC39D8076CF438
:10D4500080917E03E82FFF27E15BF64F8DE7808305
:10D4600080917D03809580937D030530110518F42C
:10D47000B701802F0BC00530110519F4BE0187E0FC
:10D4800005C007301105B1F4BE0189E00E94C467F0
:10D4900011C00231110570F081E08093A4010AC02F
:10D4A00081E08093A401109281031092830384E4AD
:10D4B00080937F0380918103803198F08091830372
:10D4C000882331F48091A401882311F480933E01D4
:10D4D00010928103109283031092800384E480935E
:10D4E0007F03E6E0CDB7DEB70C94A775CF93FC01C0
:10D4F00097FF05C0CFEFF095E195FF4F01C0C1E068
:10D5000028E631E0CF01B9010E942F75FC018B356F
:10D51000910554F08B5590408A35910538F484EB91
:10D5200090E08E1B9F0BFC0141E00DC0CF01855B9D
:10D5300090408A35910518F4E45BF04003C02E1B3F
:10D540003F0BF9014FEFEE0FFF1FE658F84F259103
:10D5500034918C2F992787FD9095289FB001299FA2
:10D56000700D389F700D1124842F992787FD909599
:10D57000689FA001699F500D789F500D1124CA012A
:10D58000CF9108952AE530E0281B390BC9010E948C
:10D59000766A089508950895089508950895089560
:10D5A00008950895089580E090E0089510925B0931
:10D5B00010925A0910925F0910925E0910925D094B
:10D5C00010925C091092600982E390E00E9461155C
:10D5D000909385038093840308959927FC0123E0A9
:10D5E000EE0FFF1F2A95E1F7E80FF91FE259F84FF8
:10D5F00095819F3F19F480E090E00895993C18F4DC
:10D60000892F99270895808182FF07C08AE0989F1B
:10D61000C0011124885097400895892F99270895B3
:10D62000A0E0B0E0E6E1FBE60C948875809184030D
:10D63000909185030E946A15882309F4CFC08091D8
:10D64000840390918503C29690938503809384030D
:10D65000C0E0D0E07E01BB247FEFC72E809160093F
:10D660008E3F21F481E08093AE0104C08F3F11F41E
:10D67000B092AE01DD240EE617E0F801838187FF4A
:10D6800017C0B3948581893C30F08D2D0E94ED6ADE
:10D69000C80FD91F02C0C80FD11DF8018181E80E43
:10D6A000F11C8681C81610F0C82E02C01092AE017F
:10D6B000D394075F1F4FFBE0FD15F8F6C092600999
:10D6C000EF2841F520918A0330918B0340918C0320
:10D6D00050918D03BB27A52F942F832F90938903FF
:10D6E00080938803AA27BB27281B390B4A0B5B0BA7
:10D6F000CE01AA27BB27280F391F4A1F5B1F209383
:10D700008A0330938B0340938C0350938D03C5E0C1
:10D71000D0E013C080918803909189038C179D07F6
:10D7200018F4C81BD90B02C0C0E0D0E08B2D99279C
:10D73000880F991FC80FD91F2596D0935B09C093F6
:10D740005A09CF3FD10578F48091230190912401AB
:10D750008C9F90018D9F300D9C9F300D1124C9012D
:10D7600064E670E013C0CE019695879596958795EF
:10D770002091230130912401289FA001299F500D61
:10D78000389F500D1124CA0169E170E00E941B7599
:10D7900070935D0960935C09809186039091870383
:10D7A0008C0F9D1F909387038093860352E0813DE9
:10D7B0009507A0F020915E0930915F092F5F3F4FE0
:10D7C000805D9240E2E0813D9E07C0F79093870321
:10D7D0008093860330935F0920935E09E9E0CDB71B
:10D7E000DEB70C94A47508950895002422273327EA
:10D7F000442751E0BB27EE27FF27A0E1660F771FE4
:10D80000881F991F001C221F331F441F660F771F9C
:10D81000881F991F001C221F331F441F2AF4050E66
:10D820002B1F3E1F4F1F04C0051A2B0B3E0B4F0B27
:10D83000550FBB1FEE1F587F556047FD5250AA95EC
:10D84000E9F6E695B7955795E695B7955795852FDF
:10D850009B2F08952227332741E0552768E0880F42
:10D86000991F221F331F880F991F221F331F1AF47D
:10D87000240F351F02C0241B350B440F551F487F52
:10D88000456037FD42506A9551F756954795569534
:10D890004795842F0895AA2797FF04C080959095F7
:10D8A0008A1F9A1F77FF04C0609570956A1F7A1FC0
:10D8B000669F9001779FA001679F300D411D5A1F01
:10D8C000300D411D5A1F889FF001999F2E0F3F1F59
:10D8D000401D511D899F300D411D5A1F300D411DA6
:10D8E0005A1FCA01B901112480CF90919803933235
:10D8F00040F4E92FFF27E559F64F80839F5F90930F
:10D9000098030895833218F48D5F809398030895E7
:10D9100090E2EEE6F9E08FE19193815087FFFCCF32
:10D920000895CF93CFB723E031E0F8948091C900F8
:10D930008F778093C9008091C9008F7B8093C90045
:10D940008091C9008F7D8093C900832F9927809390
:10D95000CD002093CC008091C80082608093C800E5
:10D9600088E18093C9008091CA008F778093CA00B4
:10D970008091CA008F7B8093CA008091CA00806228
:10D980008093CA008091CA0080618093CA00809110
:10D99000CA0088608093CA008091C9008460809327
:10D9A000C9008091CA0084608093CA008091CA0037
:10D9B00082608093CA008091C80087FF03C0809175
:10D9C000CE00F9CF8091C90080688093C900809112
:10D9D000C90080648093C9000E94886CCFBFCF913A
:10D9E0000895282F99278F709070892B31F42095F6
:10D9F00080919703822B8093970308958091AB01C8
:10DA0000882309F44BC08091510285FD04C08091A8
:10DA1000AF01882381F082E980936B0983E28093D0
:10DA20006C098091AF01882309F485E580936D0925
:10DA30001092AF0102C080936B098091AC018F30CE
:10DA400071F4809197030E94D36A882341F081E9A1
:10DA500080936B0980936C0981E380936D09109228
:10DA6000AB018091C80085FFFCCF8091C9008F7EFB
:10DA70008093C9008091C9008E7F8093C9008091F6
:10DA80006B09882311F48EEF01C08EE78093CE00DE
:10DA9000809197038093AC011092970308951F9291
:10DAA0000F920FB60F9211248F939F93EF93FF93D2
:10DAB0009091AB01992309F040C08091990388238C
:10DAC00061F480916B09882311F483E003C08139EC
:10DAD00099F481E0809399030FC0833099F4809189
:10DAE0006B09882349F090936B098091C9008E7F60
:10DAF0008093C9008EEF1EC08091C9008160809321
:10DB0000C9000EC0833261F48091C9008E7F80937A
:10DB1000C9008FEF8093CE0081E08093AB0118C0E5
:10DB200080919903E82FFF27E559F64F8F5F809387
:10DB3000990380818093CE000BC0109299031092BC
:10DB40009A0310929B038091C90080618093C90061
:10DB5000FF91EF919F918F910F900FBE0F901F90AB
:10DB60001895EF92FF920F931F93CF93DF937C0151
:10DB70008B01EA01452B39F0F80181918F01F70102
:10DB800009952197C9F7E6E0CDB7DEB70C94A775E4
:10DB9000EF92FF920F931F93CF93DF937C018B0142
:10DBA000EA01452B41F0F8010F5F1F4F8491F70107
:10DBB00009952197C1F7E6E0CDB7DEB70C94A775BC
:10DBC0000F931F93CF938C01C62F161634F480E267
:10DBD000F8010995C1501C16D4F3CF911F910F91F4
:10DBE00008950F931F93CF938C01C62F161634F40C
:10DBF00080E3F8010995C1501C16D4F3CF911F9111
:10DC00000F910895A5E3B0E0E8E0FEE60C947F757F
:10DC10002E96EEADFFAD2E97882499245401809165
:10DC20009603882321F42C961FAE1EAE2C97AEE4EB
:10DC30004A2E512C4C0E5D1E6F01B60105C01532E7
:10DC400039F00894C11CD11CF60114911123B9F7C5
:10DC5000A601461B570B31F02C968EAD9FAD2C972D
:10DC60000E94C86D112309F46AC20894C11CD11C1A
:10DC7000FF24FDA6FCA67FEFE72EF9A6F601089487
:10DC8000C11CD11C1491153721F0812F8062883777
:10DC9000B1F4F0FE0AC0F20124E030E0420E531E5F
:10DCA00080809180A280B3800AC0F20142E050E0FF
:10DCB000440E551E808191814C01AA24BB24103250
:10DCC00021F489A58823D1F61DC0133219F458E038
:10DCD000F52AD4CF1A3211F01D3291F41A3259F4C8
:10DCE000F20182E090E0480E591EE081ECA7EE239D
:10DCF0002CF6E195ECA790E1F92AAFEDFA22BECF20
:10DD00001B3211F419A7BACF1E32C1F5F6010894DF
:10DD1000C11CD11C14911A3279F4F20122E030E0D6
:10DD2000420E531E408151813FEF4F3F530714F481
:10DD30004FEF5FEFE42EA2CF40E050E0812F805301
:10DD40008A30A0F4CA0163E0880F991F6A95E1F751
:10DD5000840F951F480F591F410F511D40535040CC
:10DD6000F6010894C11CD11C1491E8CF8FEF4F3FEE
:10DD7000580714F44FEF5FEFE42E85CF103329F4EA
:10DD8000F4FC7CCF90E2F92A79CF812F815389303E
:10DD9000D8F440E050E0CA0133E0880F991F3A956B
:10DDA000E1F7840F951F480F591F410F511D405334
:10DDB0005040F6010894C11CD11C1491812F80534E
:10DDC0008A3048F34CA75FCF183619F4A4E0FA2A3A
:10DDD00055CF1C3619F4B1E0FB2A50CF133661F44D
:10DDE0003E010894611C711CF20122E030E0420EF9
:10DDF000531E808189833CC1143421F0143611F004
:10DE0000193651F5143411F431E0F32AF0FE0AC04A
:10DE1000F20144E050E0440E551E80809180A280C3
:10DE2000B3800CC0F20182E090E0480E591E808160
:10DE300091814C01AA2497FCA094BA2CB7FE0AC089
:10DE4000B094A09490948094811C911CA11CB11C4E
:10DE50008DE289A70AE06FC01F3411F01F3631F43C
:10DE60001F3411F491E0F92A08E064C0103779F406
:10DE7000F201A2E0B0E04A0E5B1E808191814C016C
:10DE8000AA24BB2400E1B0E4FB2A18E753C01337EF
:10DE9000C1F5F20122E030E0420E531E6080718035
:10DEA0006114710489F43E010894611C711C88E2BC
:10DEB00089838EE6F301818385E78B838CE68C83EF
:10DEC0008D8389E28E831F82E7FC13C08E2D9927F4
:10DED00087FD9095AC0160E070E0C3010E944C7337
:10DEE000009729F0382E3618E3140CF0C3C03E2CEE
:10DEF000C1C0F30101900020E9F731973E2E36189A
:10DF0000B9C0153511F0153731F4153511F4F1E0BC
:10DF1000FF2A0AE00FC0183519F0183709F0A0C021
:10DF200000E1F3FE07C081149104A104B10411F0D3
:10DF300020E4F22A19A6EDA6E7FC02C03FEDF32289
:10DF400029E2622E712C6C0E7D1E81149104A104B5
:10DF5000B10421F44DA5442309F47BC0802F9927F7
:10DF6000AA27BB278EA79FA7A8ABB9AB202E332427
:10DF700090E0891690E0990691E0A90690E0B90634
:10DF800048F0C501B4012EA53FA548A959A90E9492
:10DF9000427517C0AFEF8A169104A104B10449F08D
:10DFA00040F0C401B1010E941B759B014427552715
:10DFB00008C0882D602F0E940F75282F3327442713
:10DFC00055272AAB3BAB4CAB5DAB0A3059F48AA961
:10DFD000880F880F880F9AA9990F890F382D381B41
:10DFE000832F10C0003139F48AA98295807F482D93
:10DFF000481B842F07C08AA9880F880F880F582DC7
:10E00000581B852F90E02EA53FA548A959A9821637
:10E010009306A406B50608F091E08AA89BA8ACA8D0
:10E02000BDA88A3010F4805D04C0895A183509F4FF
:10E030008F7DD3018E933D01992309F099CF08304C
:10E0400041F4F3FE06C0803321F080E3FD018293AA
:10E050003F01CE010196382E3618F8E23F0E0BC074
:10E06000112309F46CC03E010894611C711C1983D2
:10E0700091E0392E19A6032D2DA4231827FC222464
:10E0800089A5882311F00F5F02C0F6FC0E5F020D18
:10E09000EF2CFF24C70180739070892B49F48CA565
:10E0A000801B682F2C968EAD9FAD2C970E94E06D43
:10E0B00089A5882331F041E050E0BE01675D7F4FC4
:10E0C0000AC0E6FE0EC080E38AA71BA742E050E02C
:10E0D000BE01665D7F4F2C968EAD9FAD2C970E9442
:10E0E000B16DC70180739070809749F48CA5801B37
:10E0F000682F2C968EAD9FAD2C970E94F16D622DEE
:10E100002C968EAD9FAD2C970E94F16D832D992793
:10E1100087FD9095AC01B3012C968EAD9FAD2C97E9
:10E120000E94B16DE4FE89CD2CA5201B2CA7622F87
:10E130002C968EAD9FAD2C970E94E06D7ECDE2E1D6
:10E14000CB5C0C949B752FB740E0F894E0E0F0E0D6
:10E1500081E2809357009491E2E0F0E080935700D1
:10E160003491E4E0F0E08093570084912FBF9E311A
:10E1700099F4363941F4893011F441E00DC08A3008
:10E1800059F442E009C0373939F4863011F443E0DC
:10E1900003C0853009F444E0842F992708959FB780
:10E1A000F8948091C900877F8093C9008091C9004D
:10E1B0008F7E8093C9008091C9008F778093C900BA
:10E1C0008091C9008F7B8093C9008091C9008F7DA9
:10E1D0008093C9009FBF08951F93CF93DF93182F9B
:10E1E00080919603882309F4A0C08091AA01181792
:10E1F00009F49BC080919503882321F40E94A370A9
:10E200008093950382ED91E090933D0180933C01D2
:10E210008FEC98E09F938F93CCE8D1E1DF93CF937D
:10E22000E091AF03F091B00309950F900F900F901C
:10E230000F90812F992784309105F1F08530910559
:10E240001CF4892B51F00CC086309105D9F0863032
:10E250009105ACF0089741F12AC08BEC98E002C020
:10E2600082EC98E09F938F93DF93CF93E091AF037D
:10E27000F091B003099527C08DEB98E0F3CF85EBC3
:10E2800098E0F0CF8DEA98E09F938F93DF93CF9340
:10E29000E091AF03F091B003099588ED91E0909380
:10E2A0003D0180933C010FC088EA98E0DBCF8CED04
:10E2B00098E09F938F93DF93CF93E091AF03F0911A
:10E2C000B003099510E00F900F900F900F90809180
:10E2D0009503843011F0823099F40E94CF70812F21
:10E2E0008150833018F40E94FE671DC0143019F469
:10E2F0000E94916C18C01830B1F40E94F36B13C0E7
:10E30000112389F082EF98E09F938F938CE891E13D
:10E310009F938F93E091AF03F091B00309950F9015
:10E320000F900F900F901093AA01DF91CF911F9142
:10E3300008950F931F93082F81E0809396034091D7
:10E34000A901E8E5F8E020E030E05FE48491992756
:10E350002F5F3F4F829FB001839F700D929F700D82
:10E36000112446275150319657FFF0CF4093A90111
:10E37000E0E3F8E020E030E057E2849199272F5F56
:10E380003F4F829FB001839F700D929F700D1124AB
:10E3900046275150319657FFF0CF4093A901809105
:10E3A0009503882321F40E94A3708093950382E053
:10E3B0009EE69093B0038093AF038091A9018334CC
:10E3C00059F088E190E029E20FB6F894A89580937F
:10E3D00060000FBE20936000063091F08DE099E060
:10E3E0009F938F938CE891E19F938F93E091AF037C
:10E3F000F091B00309950F900F900F900F90EECF12
:10E400000E94F80481E690E09F938F9386E090E06D
:10E410009F938F9382E090E09F938F93809103016D
:10E420006AE00E940F75892F99279F938F9380919F
:10E4300003010E940F7599279F938F938AE299E0B9
:10E440009F938F930CE811E11F930F93E091AF031B
:10E45000F091B003099588E598E09F938F931F93FF
:10E460000F93E091AF03F091B003099580E398E03A
:10E470009F938F931F930F93E091AF03F091B0039D
:10E4800009950E94F80483EC8093810080916F00CD
:10E49000806280936F008DB79EB746968DBF1F91A7
:10E4A0000F9108958091BB068D3338F08091D50887
:10E4B00087FD03C08CE38093BB06809169068823A7
:10E4C00031F08055853618F08FE7809369060895FE
:10E4D00080919603882309F482C08091AC03815017
:10E4E0008093AC03882309F069C089E18093AC0371
:10E4F0008091BB068E3338F08091D50887FD03C02C
:10E500008DE38093BB0680918A028238A0F58091CA
:10E51000520290915302805D974020F080916009F3
:10E52000843620F41092AE031092AD032091AD0317
:10E530003091AE0321153105B1F1C90101979093D6
:10E54000AE038093AD03419798F18091D50884FF85
:10E550002FC0809150028460809350028091E30824
:10E5600087FF26C080919403882311F13093AE0376
:10E570002093AD031DC080918A02853BC8F0909125
:10E58000BB0684E1989FC001112440962091AD0301
:10E590003091AE032817390730F42F5F3F4F309387
:10E5A000AE032093AD03809150028B7F8093500285
:10E5B0008091A901833411F0109296038091AD01EE
:10E5C000882321F081508093AD0108958BE48093DE
:10E5D000AD018091AA01843011F40E94FE6C08956F
:10E5E0001F920F920FB60F9211242F933F934F93C8
:10E5F0005F936F937F938F939F93AF93BF93EF93AB
:10E60000FF932091CE008091BB018823B1F020932D
:10E61000C6008091BB01823029F52F3F19F58FEF9D
:10E6200094E3ACE0B0E0C297A109B109B7FFFBCF1A
:10E630008091F2038093CE0015C09091AA01892F9A
:10E640008150833020F4822F0E9455680BC0943093
:10E6500021F4822F0E94F16C05C0983019F4822FAA
:10E660000E94F46BFF91EF91BF91AF919F918F91B9
:10E670007F916F915F914F913F912F910F900FBEBE
:10E680000F901F901895FB01DC0102C005900D92C0
:10E6900041505040D8F70895FC014150504030F0AF
:10E6A00001900616D1F73197CF0108958827992751
:10E6B0000895A0E0B0E0EFE5F3E70C9487756C01F6
:10E6C0007B01EA01590121978FEFCF3FD80789F0ED
:10E6D00086010894C11CD11CC7010894E11CF11CDF
:10E6E000F5010995F80180832197FFEFCF3FDF0700
:10E6F00079F7EAE0CDB7DEB70C94A375CF92DF923D
:10E70000EF92FF920F931F937C016B01FB01099520
:10E71000082FC7010196F6010995182FC8011F910E
:10E720000F91FF90EF90DF90CF900895A0E0B0E0C0
:10E73000ECE9F3E70C9489758C017B01EA0169012E
:10E7400021978FEFCF3FD80771F0F70121917F011B
:10E75000C8010F5F1F4F622FF60109952197FFEF48
:10E76000CF3FDF0791F7E8E0CDB7DEB70C94A57592
:10E77000CF92DF92EF92FF920F931F936C018B0168
:10E780007A01FA010995812F9927682FC601019610
:10E79000F70109951F910F91FF90EF90DF90CF90B7
:10E7A00008955058BB27AA270ED0E0C0D1D030F032
:10E7B000D6D020F031F49F3F11F41EF4C6C00EF401
:10E7C000E095E7FBBCC0E92FE2D080F3BA176207FF
:10E7D00073078407950718F071F49EF5FAC00EF4DC
:10E7E000E0950B2EBA2FA02D0B01B90190010C0161
:10E7F000CA01A0011124FF27591B99F0593F50F479
:10E80000503E68F11A16F040A22F232F342F4427D0
:10E81000585FF3CF469537952795A795F0405395C8
:10E82000C9F77EF41F16BA0B620B730B840BBAF098
:10E830009150A1F0FF0FBB1F661F771F881FC2F703
:10E840000EC0BA0F621F731F841F48F48795779517
:10E850006795B795F7959E3F08F0B3CF9395880FCE
:10E8600008F09927EE0F97958795089598D088F02E
:10E870009F5790F0B92F9927B751A0F0D1F0660FAC
:10E88000771F881F991F1AF0BA95C9F712C0B130C7
:10E8900081F09FD0B1E008959CC0672F782F882722
:10E8A000B85F39F0B93FCCF3869577956795B39506
:10E8B000D9F73EF490958095709561957F4F8F4F75
:10E8C0009F4F0895E89409C097FB3EF4909580957A
:10E8D000709561957F4F8F4F9F4F9923A9F0F92F26
:10E8E00096E9BB279395F695879577956795B795A4
:10E8F000F111F8CFFAF4BB0F11F460FF1BC06F5F8A
:10E900007F4F8F4F9F4F16C0882311F096E911C09B
:10E91000772321F09EE8872F762F05C0662371F0BC
:10E9200096E8862F70E060E02AF09A95660F771FD0
:10E93000881FDAF7880F9695879597F9089597F9C4
:10E940009F6780E870E060E008959FEF80EC089595
:10E9500000240A94161617061806090608950024BE
:10E960000A9412161306140605060895092E039438
:10E97000000C11F4882352F0BB0F40F4BF2B11F4AC
:10E9800060FF04C06F5F7F4F8F4F9F4F089557FD0B
:10E990009058440F551F59F05F3F71F04795880F0D
:10E9A00097FB991F61F09F3F79F0879508951216A4
:10E9B00013061406551FF2CF4695F1DF08C0161650
:10E9C00017061806991FF1CF869571056105089401
:10E9D0000895E894BB2766277727CB0197F9089518
:10E9E000629FD001739FF001829FE00DF11D649F33
:10E9F000E00DF11D929FF00D839FF00D749FF00DBF
:10EA0000659FF00D9927729FB00DE11DF91F639F5F
:10EA1000B00DE11DF91FBD01CF0111240895991B0F
:10EA200079E004C0991F961708F0961B881F7A9505
:10EA3000C9F780950895AA1BBB1B51E107C0AA1F07
:10EA4000BB1FA617B70710F0A61BB70B881F991F8F
:10EA50005A95A9F780959095BC01CD01089597FB33
:10EA6000092E07260AD077FD04D0E5DF06D0002066
:10EA70001AF4709561957F4F0895F6F790958195FA
:10EA80009F4F0895A1E21A2EAA1BBB1BFD010DC0CA
:10EA9000AA1FBB1FEE1FFF1FA217B307E407F5074E
:10EAA00020F0A21BB30BE40BF50B661F771F881F2A
:10EAB000991F1A9469F760957095809590959B01C0
:10EAC000AC01BD01CF01089597FB092E05260ED09C
:10EAD00057FD04D0D7DF0AD0001C38F4509540957C
:10EAE000309521953F4F4F4F5F4F0895F6F7909522
:10EAF0008095709561957F4F8F4F9F4F08952F920E
:10EB00003F924F925F926F927F928F929F92AF92BD
:10EB1000BF92CF92DF92EF92FF920F931F93CF930A
:10EB2000DF93CDB7DEB7CA1BDB0B0FB6F894DEBFA1
:10EB30000FBECDBF09942A88398848885F846E84C7
:10EB40007D848C849B84AA84B984C884DF80EE8011
:10EB5000FD800C811B81AA81B981CE0FD11D0FB61A
:10EB6000F894DEBF0FBECDBFED010895EE0FFF1F7D
:0AEB70000590F491E02D0994FFCF09
:10EB7A0004035E0A010164FF010020FFFFC01FC0F9
:10EB8A001F0101F40101737373FF03007D0000C4C8
:10EB9A0009C4099600124167696C65005175616480
:10EBAA00726F0000000000000064000CD201012016
:10EBBA000B050000ECFF0002040607080808070618
:10EBCA00040200FEFCFAF9F8F8F8F9FAFCFE000271
:10EBDA0004060708086440415A4655326464640AC8
:10EBEA0002969696960840403A1030380132FF0352
:10EBFA007F0090D0030090D0030032002064FFFF12
:10EC0A0064200B0A0D0B0E100B0A0C0F0B1110FAD5
:0EEC1A002068010101F7FFFCFF70FF010F648D
:00000001FF
